:100000000C94660F0C94970F0C94970F0C94970F09
:100010000C94970F0C94970F0C94970F0C94970FC8
:100020000C94970F0C94970F0C94970F0C94970FB8
:100030000C94970F0C94F8AD0C94970F0C94970FA9
:100040000C94970F0C94D18C0C94970F0C94970FE1
:100050000C94970F0C94970F0C947A260C94BEA9CD
:100060000C94970F0C94DC890C94970F0C94970FB9
:100070000C94970F0C94970F0C94970F0C94970F68
:100080000C94970F0C94970F0C94970F0C94970F58
:100090000C94970F0C94970F0C94970F0C94F0A658
:1000A0000C94970F0C94970F0C94970F0C94970F38
:1000B0000C94970F0C94970F0C94970F0C94970F28
:1000C0000C94970F0C94970F0C94970F0C94970F18
:1000D0000C94970F0C94970F0C94970F0C94970F08
:1000E0000C94970FC726D526F126FF261927272718
:1000F0004127452747274B27532742A847A84CA805
:1001000056A8CFA860A868A870A87AA884A88EA8C6
:100110009DA8A7A8CFA8B1A8BBA8C5A8EDA8F0A87E
:10012000E3A8E7A827A9F4A8F8A8FEA802A906A9A9
:100130000CA910A914A927A91AA91EA922A9084A1D
:10014000D73B3BCE016E84BCBFFDC12F3D6C7431EB
:100150009ABD56833DDA3D00C77F11BED9E4BB4C42
:100160003E916BAAAABE000000803F05A84CCDB20C
:10017000D44EB93836A9020C50B9918688083CA6ED
:10018000AAAA2ABE000000803F007C3C3E5E2B3DB8
:100190003F2F5B5D3B2C2A225C004572723A204D5A
:1001A000415854454D50204245440054656D70659A
:1001B000726174757265206865617465642062653A
:1001C00064207377697463686564206F66662E20A7
:1001D0004D415854454D502074726967676572658A
:1001E00064202121004572723A204D494E54454DFC
:1001F00050003A204578747275646572207377698F
:100200007463686564206F66662E204D494E5445C0
:100210004D502074726967676572656420210045DE
:1002200072723A204D415854454D50003A2045785D
:10023000747275646572207377697463686564208D
:100240006F66662E204D415854454D50207472699A
:10025000676765726564202100202D20496E7661F4
:100260006C6964206578747275646572206E756D52
:10027000626572202100504944204175746F747585
:100280006E652066696E69736865642120507574B7
:1002900020746865206C617374204B702C204B694E
:1002A00020616E64204B6420636F6E7374616E74A2
:1002B000732066726F6D2061626F766520696E745F
:1002C0006F20436F6E66696775726174696F6E2E19
:1002D0006800504944204175746F74756E652066DE
:1002E00061696C6564212074696D656F75740020A7
:1002F000403A006F6B20543A006F6B20423A005036
:100300004944204175746F74756E65206661696C2F
:100310006564212054656D70657261747572652025
:10032000746F6F206869676800204B643A20002072
:100330004B693A2000204B703A200020436C6173D7
:100340007369632050494420002054753A200020EE
:100350004B753A2000206D61783A2000206D696E5F
:100360003A200020643A200020626961733A20003C
:100370001000C90210012C01400122017001180176
:10038000B0010E01F00104015002FA00B002F000C9
:100390003003E600D003DC009004D2007005C800F2
:1003A000A006BE000008B400B009AA00D00BA0004F
:1003B000600E960060118C000015820020197800F4
:1003C000C01D6E00A0226400B0275A00902C50007F
:1003D00000314600E0343C0010383200903A2800EA
:1003E000603C1E00A03D1400803E0A00203F00003B
:1003F00070012C0190012701B0012201C0011D01F3
:10040000F00118011002130130020E01600209010F
:1004100090020401C002FF000003FA004003F5004F
:100420008003F000D003EB002004E6007004E1003C
:10043000E004DC004005D700C005D2004006CD0036
:10044000D006C8008007C3003008BE00F008B9001D
:10045000C009B400B00AAF00B00BAA00D00CA500D0
:10046000000EA000500F9B00C0109600501291008B
:1004700000148C00C0158700B0178200B0197D00F1
:10048000D01B7800001E730040206E00902269008F
:10049000F024640040275F0090295A00E02B5500AB
:1004A000102E500020304B0010324600E033410047
:1004B00090353C001037370070383200A0392D00DD
:1004C000B03A2800A03B2300603C1E00103D1900FC
:1004D000903D1400103E0F00703E0A00C03E050023
:1004E000003F00004D383420582059205A20450044
:1004F00043616E6E6F7420656E74657220737562F1
:100500006469723A20004D3234004D323320257335
:10051000006175746F25692E67006572726F7220B5
:1005200077726974696E6720746F2066696C650004
:100530004E6F74207072696E74696E67000A002FC6
:10054000005344207072696E74696E67206279741A
:100550006520000A002E0044656C6574696F6E208A
:100560006661696C65642C2046696C653A200046BA
:10057000696C652064656C657465643A002E006F73
:1005800070656E206661696C65642C2046696C65D7
:100590003A200057726974696E6720746F2066692B
:1005A0006C653A20002E006F70656E206661696C84
:1005B00065642C2046696C653A20002E006F7065DA
:1005C0006E206661696C65642C2046696C653A2012
:1005D0000046696C652073656C6563746564002012
:1005E00053697A653A200046696C65206F70656EC4
:1005F00065643A20002E006F70656E206661696C3C
:1006000065642C2046696C653A20004E6F77206641
:10061000726573682066696C653A20004E6F7720BA
:10062000646F696E672066696C653A2000222070ED
:100630006F73002220706172656E743A2200535508
:1006400042524F5554494E452043414C4C20746111
:10065000726765743A2200747279696E6720746FEC
:100660002063616C6C207375622D67636F64652015
:1006700066696C6573207769746820746F6F206D8C
:10068000616E79206C6576656C732E204D41582023
:100690006C6576656C2069733A005344206361721F
:1006A00064206F6B006F70656E526F6F74206661AF
:1006B000696C656400766F6C756D652E696E697422
:1006C000206661696C656400534420696E6974201A
:1006D0006661696C0000002110422063308440A5EF
:1006E00050C660E770088129914AA16BB18CC1ADF9
:1006F000D1CEE1EFF13112100273325222B5529491
:1007000042F772D662399318837BB35AA3BDD39C48
:10071000C3FFF3DEE36224433420040114E664C71C
:1007200074A44485546AA54BB528850995EEE5CF98
:10073000F5ACC58DD55336722611163006D776F630
:10074000669556B4465BB77AA719973887DFF7FEE8
:10075000E79DD7BCC7C448E5588668A778400861BC
:100760001802282338CCC9EDD98EE9AFF948896938
:10077000990AA92BB9F55AD44AB77A966A711A50D0
:100780000A333A122AFDDBDCCBBFFB9EEB799B5888
:100790008B3BBB1AABA66C877CE44CC55C222C035C
:1007A0003C600C411CAEED8FFDECCDCDDD2AAD0BD8
:1007B000BD688D499D977EB66ED55EF44E133E3270
:1007C0002E511E700E9FFFBEEFDDDFFCCF1BBF3A28
:1007D000AF599F788F8891A981CAB1EBA10CD12D17
:1007E000C14EF16FE18010A100C230E3200450251A
:1007F0004046706760B9839893FBA3DAB33DC31C8E
:10080000D37FE35EF3B1029012F322D23235421469
:100810005277625672EAB5CBA5A89589856EF54FD9
:10082000E52CD50DC5E234C324A0148104667447B9
:100830006424540544DBA7FAB79987B8975FE77E2D
:10084000F71DC73CD7D326F2369106B01657667609
:1008500076154634564CD96DC90EF92FE9C899E979
:10086000898AB9ABA94458654806782768C018E159
:10087000088238A3287DCB5CDB3FEB1EFBF98BD8CD
:100880009BBBAB9ABB754A545A376A167AF10AD0A9
:100890001AB32A923A2EFD0FED6CDD4DCDAABD8B19
:1008A000ADE89DC98D267C076C645C454CA23C83F9
:1008B0002CE01CC10C1FEF3EFF5DCF7CDF9BAFBA6D
:1008C000BFD98FF89F176E367E554E745E932EB249
:1008D0003ED10EF01E53544F505045442E20005030
:1008E00072696E7465722073746F707065642064D1
:1008F000756520746F206572726F72732E20466961
:100900007820746865206572726F7220616E642051
:10091000757365204D39393920746F207265737491
:100920006172742E202854656D70657261747572E1
:10093000652069732072657365742E205365742079
:100940006974206166746572207265737461727473
:10095000696E6729004B494C4C45442E200050726B
:10096000696E7465722068616C7465642E206B69B1
:100970006C6C28292063616C6C656421006F6B00CE
:10098000526573656E643A20002200556E6B6E6F7F
:10099000776E20636F6D6D616E643A2022004D3278
:1009A000323020532569005A204F666673657420E3
:1009B0003A20007A5F6D61783A20007A5F6D696E47
:1009C0003A20005A204F6666736574005A204F66BD
:1009D00066736574206F6B002200556E6B6E6F77C7
:1009E0006E20636F6D6D616E643A2022007A5F6DD8
:1009F00061783A20007A5F6D696E3A2000795F6D08
:100A000061783A2000795F6D696E3A2000785F6DF9
:100A100061783A2000785F6D696E3A2000205A3A7A
:100A20000020593A0020436F756E7420583A200018
:100A300020453A00205A3A0020593A00583A0046D8
:100A400049524D574152455F4E414D453A4D6172B5
:100A50006C696E2056312E302E323B2053707269F5
:100A60006E7465722F6772626C206D617368757049
:100A700020666F722067656E36204649524D574199
:100A800052455F55524C3A68747470733A2F2F6711
:100A900069746875622E636F6D2F4D61726C696E3B
:100AA0004669726D776172652F4D61726C696E2057
:100AB00050524F544F434F4C5F56455253494F4E3F
:100AC0003A312E30204D414348494E455F545950EC
:100AD000453A507275736120693320455854525518
:100AE0004445525F434F554E543A31205555494481
:100AF0003A30303030303030302D303030302D30F2
:100B00003030302D303030302D30303030303030EB
:100B100030303030300A00507275736120693320F4
:100B20004F66662E005072757361206933207265BE
:100B30006164792E0042656420646F6E652E00202A
:100B4000423A0020453A00543A0042656420486524
:100B50006174696E672E0048656174696E67206410
:100B60006F6E652E0020573A0020453A00543A0037
:100B700048656174696E672E2E2E002042403A004F
:100B800020403A00202F003A00205400202F00205F
:100B9000423A00202F006F6B20543A002569206DE7
:100BA000696E2C2025692073656300456E6420669C
:100BB000696C65206C69737400426567696E2066B4
:100BC000696C65206C697374004E6F206D6F76657B
:100BD0002E005072757361206933207265616479EB
:100BE0002E00526573756D696E67207072696E7440
:100BF000005761697420666F7220757365722E2EBE
:100C00002E00536C6565702E2E2E00256920686FAE
:100C1000757273202569206D696E75746573004463
:100C20006F6E65207072696E74696E672066696C9C
:100C3000650053544F505045442E20005072696E49
:100C40007465722073746F707065642064756520BC
:100C5000746F206572726F72732E204669782074EB
:100C60006865206572726F7220616E6420757365AD
:100C7000204D39393920746F207265737461727434
:100C80002E202854656D70657261747572652069D7
:100C9000732072657365742E205365742069742007
:100CA00061667465722072657374617274696E67CF
:100CB00029004E6F204C696E65204E756D6265721D
:100CC000207769746820636865636B73756D2C2089
:100CD0004C617374204C696E653A20004E6F20435E
:100CE0006865636B73756D2077697468206C696ED5
:100CF00065206E756D6265722C204C617374204C9A
:100D0000696E653A2000636865636B73756D206D6D
:100D100069736D617463682C204C617374204C6935
:100D20006E653A20004C696E65204E756D62657285
:100D3000206973206E6F74204C617374204C696E4F
:100D400065204E756D6265722B312C204C61737479
:100D5000204C696E653A20004D31313000446F6E91
:100D60006520736176696E672066696C652E006F19
:100D70006B004D3239002020506C616E6E657242FE
:100D8000756666657242797465733A200020467212
:100D90006565204D656D6F72793A20004A616E205D
:100DA0003236203230313600436F6D70696C6564C5
:100DB0003A2000286E6F6E652C2064656661756C44
:100DC0007420636F6E6669672900207C204175740A
:100DD000686F723A20004A616E203236203230311C
:100DE000362031393A33373A353400204C61737448
:100DF00020557064617465643A2000312E302E32C3
:100E0000004D61726C696E0020536F667477617279
:100E10006520526573657400205761746368646F60
:100E200067205265736574002042726F776E206F81
:100E30007574205265736574002045787465726E10
:100E4000616C20526573657400506F7765725570E0
:100E5000007374617274002200656E717565696E4D
:100E6000672022002200656E717565696E67202219
:100E700000FFFFFF0000A0400000A0400000004075
:100E800000005643000046431FC5484300000000D1
:100E9000000000001F856B3E0000564300004643E3
:100EA0000000494300000000000000001F856B3E69
:100EB0006563686F3A004572726F723A00436172FF
:100EC000642072656D6F76656400436172642069A9
:100ED0006E73657274656400473120453430204676
:100EE0003130300047312045373020463430300033
:100EF0004D383300473120452D38302046343030CE
:100F0000004D3833002D2D3A2D2D002D2D2D005361
:100F100044000120000120004D363030004368615C
:100F20006E67652066696C616D656E7400466C6FF6
:100F30007700466C6F770046616E2073706565645C
:100F40000046616E2073706565640042656400420E
:100F50006564004E6F7A7A6C65004E6F7A7A6C65C4
:100F6000005370656564005370656564004D616988
:100F70006E00436F6F6C646F776E00464C4558206F
:100F80002D20203233302F35300050502020202D9E
:100F900020203235342F3130300048495053202D35
:100FA00020203232302F3130300050455420202D57
:100FB00020203234302F393000504C4120202D2059
:100FC000203231302F35300041425320202D202057
:100FD0003235352F313030004D61696E004D383477
:100FE000004D383420582059205A2045004D3234C5
:100FF000004D323320257300052E2E004D61696EA1
:101000000046616E2073706565640046616E2073F2
:10101000706565640042656400426564004E6F7AE5
:101020007A6C65004E6F7A7A6C65005365747469EA
:101030006E677300580059005A00457874727564E1
:101040006572004578747275646572004D6F7665DF
:10105000205A004D6F76652059004D6F76652058F7
:101060000053657474696E677300473238004175C8
:10107000746F20686F6D65004D383400446973618A
:10108000626C6520737465707065727300473238E6
:10109000205A0043616C696272617465205A004D88
:1010A0006F766520617869730054656D7065726153
:1010B00074757265004D61696E005265763A203133
:1010C00037352D326200686F77746F2E70727573CA
:1010D0006133642E636F6D00666F72756D2E707272
:1010E00075736133642E636F6D0070727573613355
:1010F000642E636F6D004669726D77617265202D95
:1011000020322E322E32004D61696E0053757070A0
:101110006F72740053657474696E677300556E6CFA
:101120006F61642066696C616D656E74004C6F61FF
:10113000642066696C616D656E74004E6F20534467
:101140002063617264005072696E742066726F6D04
:101150002053440053746F70207072696E74005293
:101160006573756D65207072696E7400506175737A
:1011700065207072696E74005072656865617400F4
:1011800054756E6500496E666F2073637265656E97
:101190000048617264636F646564204465666175CC
:1011A0006C742053657474696E6773204C6F61644E
:1011B00065640046696C616D656E74207365747456
:1011C000696E67733A2044697361626C65640020DC
:1011D00020204D32303020440046696C616D656ED0
:1011E000742073657474696E67733A002020204D13
:1011F0003230392053004175746F2D52657472611D
:1012000063743A20533D3020746F206469736162C7
:101210006C652C203120746F20696E746572707259
:10122000657420657874727564652D6F6E6C7920B5
:101230006D6F76657320617320726574726163747B
:1012400073206F72207265636F76657269657300D3
:101250002046002020204D32303820530052656354
:101260006F7665723A20533D4578747261206C65E3
:101270006E67746820286D6D2920463A5370656545
:101280006420286D6D2F6D2900205A002046002013
:1012900020204D32303720530052657472616374E0
:1012A0003A20533D4C656E67746820286D6D292087
:1012B000463A537065656420286D6D2F6D29205A5C
:1012C0003A205A4C69667420286D6D29002044002C
:1012D0002049002020204D33303120500050494417
:1012E0002073657474696E67733A00205A00205940
:1012F0000020204D323036205800486F6D65206F39
:10130000666673657420286D6D293A0020450020BB
:101310005A0020580020420020540020204D323036
:1013200035205300416476616E6365642076617296
:101330006961626C65733A20533D4D696E20666544
:1013400065647261746520286D6D2F73292C20549B
:101350003D4D696E2074726176656C2066656564CA
:101360007261746520286D6D2F73292C20423D6DAC
:10137000696E696D756D207365676D656E74207437
:10138000696D6520286D73292C20583D6D61786941
:101390006D756D205859206A65726B20286D6D2F10
:1013A00073292C20205A3D6D6178696D756D205A26
:1013B000206A65726B20286D6D2F73292C202045C3
:1013C0003D6D6178696D756D2045206A65726B2091
:1013D000286D6D2F73290020540020204D323034A9
:1013E000205300416363656C65726174696F6E3A86
:1013F00020533D616363656C65726174696F6E2C27
:1014000020543D7265747261637420616363656C1E
:1014100065726174696F6E00204500205A00205982
:101420000020204D3230312058004D6178696D75B3
:101430006D20416363656C65726174696F6E20280D
:101440006D6D2F7332293A00204500205A00205933
:101450000020204D3230332058004D6178696D7581
:101460006D2066656564726174657320286D6D2FEB
:1014700073293A00204500205A0020590020204DB1
:10148000393220580053746570732070657220756E
:101490006E69743A0045303A20005A3A2000593AB1
:1014A0002000583A20004D53312C4D5332205069C2
:1014B0006E730A00656E6473746F7073206869746C
:1014C0003A205A00205A3A00656E6473746F707344
:1014D000206869743A20590020593A00656E647397
:1014E000746F7073206869743A20580020583A006D
:1014F000656E6473746F7073206869743A20002499
:10150000F4D43050C38E20C2A24017828B701112C7
:101510007A910D816CD90AA861E108C75866076104
:101520005143061E4B5D05C145A7041A411104092C
:101530003D9803713931034036DB0265339102D4A3
:10154000305402802E1D02632CEE01752AC501B0B5
:1015500028A001102781018F2564012B244B01E075
:10156000223401AC211F018D200D01801FFC00845D
:101570001EED00971DDF00B81CD200E61BC6002040
:101580001BBC00641AB200B219A8000A19A0006AB4
:10159000189900D117910040178B00B516840031BF
:1015A000167E00B31579003A157300C7146F005802
:1015B000146A00EE1366008813630025135E00C7EB
:1015C000125B006C12570015125400C111510070CB
:1015D000114F0021114B00D61049008D10470046D5
:1015E00010440002104200C00F4000800F3E004235
:1015F0000F3C00060F3B00CB0E3800930E37005C0B
:101600000E3500270E3400F30D3200C10D3100906D
:101610000D3000600D2E00320D2D00050D2C00D96F
:101620000C2B00AE0C2900850C29005C0C27003522
:101630000C27000E0C2600E80B2400C40B2400A08D
:101640000B23007D0B23005A0B2100390B210018BE
:101650000B2000F80A1F00D90A1E00BB0A1E009DBD
:101660000A1D00800A1D00630A1C00470A1B002C8B
:101670000A1B00110A1A00F7091A00DD091900C433
:10168000091900AB091900920917007B09180063BA
:101690000917004C09160036091600200916000A21
:1016A000091500F5081500E0081400CC081400B86E
:1016B000081400A4081400900813007D0812006BA1
:1016C00008130058081200460812003408110023BD
:1016D0000811001208110001081100F0071000E0C5
:1016E000071000D0071000C0071000B0070F00A1BE
:1016F00007100091070E0083070F0074070F0065A5
:10170000070E0057070E0049070E003B070D002E7D
:10171000070E0020070D0013070D0006070D00F946
:10172000060C00ED060D00E0060C00D4060C00C807
:10173000060C00BC060C00B0060C00A4060B0099B9
:10174000060C008D060B0082060B0077060B006C62
:10175000060B0061060A0057060B004C060A004201
:10176000060A0038060A002E060A0024060A001A95
:10177000060A001006090007060A00FD050900F424
:10178000050900EB050900E2050900D9050900D0AB
:10179000050900C7050900BE050900B5050800AD2B
:1017A000050800A50509009C050800940508008CA3
:1017B000050800840508007C050800740508006C15
:1017C000050700650508005D050700560508004E81
:1017D00005070047050700400508003805070031E8
:1017E0000507002A050700230507001C050600164B
:1017F0000507000F0507000805060002050700FBA6
:10180000040600F5040700EE040600E8040600E202
:10181000040700DB040600D5040600CF040600C957
:10182000040600C3040600BD040600B7040600B1A8
:10183000040500AC040600A6040600A00405009BF5
:1018400004060095040500900406008A040500853E
:10185000040500800406007A040500750405007084
:101860000405006B04050066040500610405005CC6
:1018700004050057040500520405004D0405004806
:10188000040500430405003E0404003A0405003545
:10189000040500300404002C040500270404002380
:1018A0000405001E0404001A0404001604050011B7
:1018B0000404000D040400090405000404040000ED
:1018C000040400FC030400F8030400F4030400F023
:1018D000030400EC030400E8030400E4030400E054
:1018E000030400DC030400D8030400D4030400D084
:1018F000030400CC030400C8030300C50303002451
:10190000F404D9201BC40C5C0E9804C4095F026562
:10191000077101F405F900FB04B30048048700C116
:101920000369005803550003034500BE023A0084D2
:1019300002310053022A002902250004022000E49B
:10194000011C00C8011900AF0117009801140084A0
:10195000011300710110006101100051010E0043DC
:10196000010D0036010B002B010B0020010B0015AF
:101970000109000C01090003010800FB000800F345
:10198000000800EB000700E4000600DE000600D8B7
:10199000000600D2000600CC000500C7000500C20A
:1019A000000500BD000400B9000400B5000400B14A
:1019B000000400AD000400A9000400A5000300A27B
:1019C0000003009F0004009B0003009800030095A3
:1019D00000020093000300900003008D0002008BC2
:1019E00000030088000200860002008400030081DA
:1019F0000002007F0002007D0002007B00020079EF
:101A000000020077000100760002007400020072FC
:101A1000000100710002006F0002006D0001006C07
:101A20000002006A00010069000200670001006610
:101A30000001006500010064000200620001006115
:101A4000000100600001005F0002005D0001005C19
:101A50000001005B0001005A00010059000100581C
:101A6000000100570001005600010055000100541C
:101A7000000100530000005300010052000100511A
:101A8000000100500001004F0001004E0000004E18
:101A90000001004D0001004C0001004B0000004B14
:101AA0000001004A00010049000100480000004810
:101AB000000100470001004600000046000100450B
:101AC0000000004500010044000100430000004305
:101AD00000010042000000420001004100000041FE
:101AE000000100400001003F0000003F0001003EF7
:101AF0000000003E0001003D0000003D0001003CF0
:101B00000000003C0000003C0001003B0000003BE6
:101B10000001003A0000003A0001003900000039DD
:101B200000010038000000380000003800010037D4
:101B300000000037000100360000003600000036CB
:101B400000010035000000350000003500010034C0
:101B500000000034000000340001003300000033B6
:101B600000000033000100320000003200000032AB
:101B700000010031000000310000003100010030A0
:101B800000000030000000300001002F0000002F96
:101B90000000002F0000002F0001002E0000002E8A
:101BA0000000002E0001002D0000002D0000002D7F
:101BB0000000002D0001002C0000002C0000002C73
:101BC0000000002C0001002B0000002B0000002B67
:101BD0000000002B0001002A0000002A0000002A5B
:101BE0000000002A0001002900000029000000294F
:101BF0000000002900000029000100280000002842
:101C00000000002800000028000000280001002734
:101C10000000002700000027000000270000002728
:101C2000000100260000002600000026000000261B
:101C3000000000260001002500000025000000250E
:101C40000000002500000025000000250001002400
:101C500000000024000000240000002400000024F4
:101C600000010023000000230000002300000023E7
:101C700000000023000000230000002300010022D8
:101C800000000022000000220000002200000022CC
:101C900000000022000100210000002100000021BE
:101CA00000000021000000210000002100000021B0
:101CB00000010020000000200000002000000020A3
:101CC0000000002000000020000000200000002094
:101CD0000001001F0000001F0000001F0000001F87
:101CE0000000001F0000001F0000001F0001001E78
:101CF0000000001E0000001E0000001E000000206A
:101D0000746F6F206C6F6E6720657874727573697D
:101D10006F6E2070726576656E7465640020636F07
:101D20006C6420657874727573696F6E207072656B
:101D300076656E746564000000090A02080B0C0DDC
:101D4000070603040100000000000000000000007E
:101D50000000000000000000000000000000000083
:101D600000000011100F0000000000000000000043
:101D70000000000000000000000000000000000063
:101D80000000000000000000000000000001021040
:101D90002020080810204010204080020102010885
:101DA0000402010102040810204080804020100835
:101DB000040201800402018040201008040201088E
:101DC00004020101020408102040800102040810EE
:101DD000204080100804088010204004408010201B
:101DE00040048005050505070508080808020202E9
:101DF000020A0A08080404040401010101010101A6
:101E0000010303030303030303040707070C0C0C7C
:101E10000C0C0C0C0C020202020606060606060654
:101E2000060B0B0B0B0B0B0B0B07070A0A0A0A0A14
:101E30000A05050504040408080000200023002604
:101E40000029002C002F00320000010000030106D1
:101E500001090100002200250028002B002E00317E
:101E600000340002010000050108010B01000021FF
:101E700000240027002A002D00300033000101005B
:101E800000040107010A01024E414E494E495459CE
:101E9000494E46CDCCCC3D0AD7233C17B7D1387735
:101EA000CC2B329595E6241FB14F0A00002041004B
:101EB00000C84200401C4620BCBE4CCA1B0E5AAE95
:101EC000C59D74008B64D07EC4A68F6411241FBE90
:101ED000CFEFD1E2DEBFCDBF00E00CBF15E0A0E048
:101EE000B2E0E0E1F4E701E00BBF02C007900D9221
:101EF000A23EB107D9F724E1A2EEB5E001C01D92E0
:101F0000AD3BB207E1F71EE1CAECDEE100E006C03E
:101F100022970109FE010BBF0E94AFB3C43CD10759
:101F200080E00807A9F70E94C8AA0C94F7B90C949E
:101F30000000CF93DF93EC019C012C5F3F4F41E009
:101F400050E060E070E0898D9A8D0E943B1A8823F2
:101F500099F04D895E896F89788D452B462B472BEB
:101F600059F44C815D816E817F814D8B5E8B6F8BCF
:101F7000788F998190689983DF91CF910895CF925E
:101F8000DF92EF92FF920F931F93CF93DF93EC01B9
:101F900089899A89AB89BC89803E9F4FAF41B10541
:101FA00010F080E06BC0CE01C4DF8823D1F30E9423
:101FB0004F18182F8823A9F3E98DFA8DCC80DD8086
:101FC000EE80FF8032E0C31AD108E108F1080584F1
:101FD00004C0CC0CDD1CEE1CFF1C0A94D2F78685D5
:101FE0009785A089B189C80ED91EEA1EFB1E81E023
:101FF0008093E805C092EB07D092EC07E092ED07E2
:10200000F092EE0780E092E0EBEEF5E0DF019C015C
:102010001D9221503040E1F701E0E98DFA8D848175
:10202000081790F42BEE35E0B701A601400F511DC3
:10203000611D711D8091E9059091EA050E94D53CD2
:102040008823E1F00F5FE9CFC12C82E0D82EE12C8C
:10205000F12C058404C0CC0CDD1CEE1CFF1C0A9482
:10206000D2F749895A896B897C894C0D5D1D6E1D9B
:102070007F1D498B5A8B6B8B7C8B812FDF91CF918E
:102080001F910F91FF90EF90DF90CF900895CF9325
:10209000DF93EC0141E0611101C040E06C857D857A
:1020A0008E859F850E948F18882341F0888920E2C1
:1020B000829FC001112485519A4F02C080E090E0B8
:1020C000DF91CF91089530E020E04EE2DC015C9199
:1020D000503271F0383029F4FB01E20FF11D4083DA
:1020E0002F5FFB01E20FF11DDC015C9150832F5F3C
:1020F0003F5F01963B3051F7FB01E20FF11D10826B
:102100000895CF93DF93EB01FC012381211102C0DD
:1021100080E00EC02250223020F48FE288831982A2
:1021200006C060E0B4DF009799F3BE01CCDF81E028
:10213000DF91CF910895FB012BE030E231932150E4
:10214000E9F7DC0190E027E03A2FEB2F8D91811128
:102150000AC0DA013C931196EC9381E0FB01908177
:10216000903239F525C08F32A1F38E3219F0EAE8AA
:10217000F1E008C02A30E1F098E02AE0E5CF31969E
:102180003817B1F034913111FACF291788F03FEDAB
:10219000380F3E3568F431E0390FFB01E90FF11DCE
:1021A0009FE9980F9A3108F480528083932FCCCF07
:1021B00080E008950F931F93CF93DF93EC018B0181
:1021C0008B81882311F080E042C0FB018789803138
:1021D00039F18032C1F783E08B83F801428D538D52
:1021E000648D758D4D8B5E8B6F8B788F9E012F5E0E
:1021F0003F4FC8010E944619882329F31A8F098F7F
:1022000081E089831C821D821E821F8218861986A6
:102210001A861B861C861D861E861F86188A17C076
:1022200082E08B831D8A1E8A1F8A188EFB01408DD7
:10223000518D60E070E095E0440F551F661F771FD9
:102240009A95D1F7498B5A8B6B8B7C8BD7CFDF91CB
:10225000CF911F910F9108952F923F924F925F92CD
:102260006F927F928F929F92AF92BF92CF92DF92A6
:10227000EF92FF920F931F93CF93DF93EC015B01DB
:102280006A018B81811103C08FEF9FEFC7C08981E5
:1022900080FFFACF49895A896B897C89888599851D
:1022A000AA85BB852601612C712C8A019B01081B24
:1022B000190B2A0B3B0B401651066206730618F0E9
:1022C0006A01C81AD90A76013E0124E0620E711C27
:1022D000E114F10409F476C0488559856A857B8547
:1022E0004A0181E098222B811A012B01E9E05694E2
:1022F000479437942794EA95D1F7898D9A8DFC01FC
:10230000223049F4628D738D848D958D620D731D1D
:10231000841D951D3CC0148111501221811491041B
:10232000C1F4111116C0452B462B472B49F48D895A
:102330009E89AF89B88D8C839D83AE83BF8309C08E
:102340004C815D816E817F81930121D7882309F4BF
:102350009BCFE98DFA8D6C817D818E819F8162504A
:10236000710981099109058404C0660F771F881FD0
:10237000991F0A94D2F72685378540895189620FC3
:10238000731F841F951F610F711D811D911D20E01A
:1023900032E02819390987012E153F0508F4890113
:1023A0000115F2E01F0769F52091EB073091EC076A
:1023B0004091ED075091EE07621773078407950768
:1023C00019F41FC0C6012AC09501AB01BC01809160
:1023D000E9059091EA050E94603C882309F454CFF6
:1023E000A00EB11E88859985AA85BB85800F911F97
:1023F000A11DB11D88879987AA87BB87E01AF10ABA
:1024000067CF40E08CD6882309F43ECFB4016551F4
:102410007A4FA801C5010E94CCB6E2CFDF91CF91DF
:102420001F910F91FF90EF90DF90CF90BF90AF90F2
:102430009F908F907F906F905F904F903F902F90E4
:102440000895CF93DF931F92CDB7DEB741E050E000
:10245000BE016F5F7F4F00DF019719F4898190E023
:1024600002C08FEF9FEF0F90DF91CF910895CF9231
:10247000DF92EF92FF920F931F93CF93DF936C0144
:10248000EB017A01FC018381823060F000851185C7
:10249000228533850F71112722273327012B022B29
:1024A000032B11F08FEF5CC04115510511F0F701BE
:1024B00010821DE040E250E0BE01C601CDDE803258
:1024C000910539F021E0892B09F420E0822F8195D4
:1024D00047C028812223C1F0253E61F32E3251F3FB
:1024E0003B853F733F3061F4E114F10449F04A8DBC
:1024F0005B8D452B29F42F713FEF320F343030F0D4
:102500002B8523FDD7CF2CC080E02AC030E021509E
:102510003109129FC001139F900D1124F701E80F9C
:10252000F91F298120832B8121832D8122832F81F3
:102530002383298524832E852583288926832A8938
:1025400027832C8920872E892187288D22872C8D0F
:1025500023872E8D2487288126FFD2CF1586D0CFC2
:10256000DF91CF911F910F91FF90EF90DF90CF906F
:1025700008951F93CF93DF93EC018B81823018F481
:1025800080E090E023C0488559856A857B85A5E079
:102590007695679557954795AA95D1F7142F1F7093
:1025A000CE014FDF97FDECCF488559856A857B8545
:1025B000415E5F4F6F4F7F4F488759876A877B87A0
:1025C00020E2129FC001112485519A4FDF91CF91D3
:1025D0001F9108954F925F926F927F92AF92BF9238
:1025E000CF92DF92EF92FF920F931F93CF93DF93DF
:1025F000EC016A017B012B81222349F089899A89A8
:10260000AB89BC8984179507A607B70710F480E04B
:102610006BC0223009F463C0C114D104E104F10499
:1026200049F41C821D821E821F82188619861A8612
:102630001B8659C088859985AA85BB85E98DFA8D49
:10264000E585F0E03996AC01BD01415051096109C1
:1026500071090E2E04C076956795579547950A9493
:10266000D2F797018601015011092109310904C0EF
:102670003695279517950795EA95D2F7041715070C
:102680002607370720F0892B8A2B8B2B49F48D895D
:102690009E89AF89B88D8C839D83AE83BF8304C030
:1026A000041B150B260B370B280139015E0184E052
:1026B000A80EB11C411451046104710481F04C81D5
:1026C0005D816E817F819501898D9A8D60D591E0C4
:1026D000491A5108610871088111ECCF05C0C886FC
:1026E000D986EA86FB8681E0DF91CF911F910F9119
:1026F000FF90EF90DF90CF90BF90AF907F906F9062
:102700005F904F9008950F931F93CF93DF93EC0149
:102710008B818823D1F1898187FF32C061E0CE01AE
:10272000B6DC8C01009789F1FC018081853E69F15E
:102730008B81823040F449895A896B897C89448F26
:10274000558F668F778F4D895E896F89788DF801F7
:10275000538F428F758B648BE091E205F091E30516
:10276000309759F0B8016A5E7F4FC80148961995B5
:10277000F801808D918D938B828B89818F778983EE
:10278000DF91CF911F910F918AC481E0888380E00F
:10279000DF91CF911F910F910895CF93DF93EC01BB
:1027A000B2DF1B82DF91CF910895FC0123812111BB
:1027B000F4CF08954F925F926F927F92AF92BF9243
:1027C000CF92DF92EF92FF920F931F93CF93DF93FD
:1027D00000D01F92CDB7DEB75C016A017B01FC011E
:1027E00083818130E9F4818181FF1AC0F5018189FB
:1027F0009289A389B48984179507A607B70780F043
:10280000892B8A2B8B2B09F472C0F50140845184EB
:1028100062847384B701A601C501DCDE811102C0A8
:1028200080E066C0F501818D928DC114D104E10470
:10283000F10469F4458956896789708D25D7882305
:1028400079F3F501158A168A178A108E37C0F501BB
:1028500044815581668177819E012F5F3F4F97D4D8
:102860008823F1F249815A816B817C81F501818D48
:10287000928DFC012789203139F4483FFFEF5F0733
:1028800061057105D8F407C0483F2FEF5207620772
:102890002FE0720798F4F8D6882309F4C1CFF50128
:1028A00044815581668177810FEF1FEF2FEF3FE065
:1028B000818D928D51D5882309F4B2CFF501C18A5B
:1028C000D28AE38AF48A818180688183C5011BDF13
:1028D000882309F4A5CFB701A6014C145D046E044A
:1028E0007F0410F4B301A201C50174DE01C081E0D0
:1028F0000F900F900F900F90DF91CF911F910F913C
:10290000FF90EF90DF90CF90BF90AF907F906F904F
:102910005F904F900895FF920F931F93CF93DF9393
:10292000EC01F42E80E2689FF0011124E551FA4F8A
:102930008385817121F0842F827109F04EC08091CE
:10294000EB079091EC07A091ED07B091EE078C8713
:102950009D87AE87BF87688B4489558960E070E0AA
:10296000BA0155274427028D138D20E030E0402B1B
:10297000512B622B732B4D8B5E8B6F8B788F8385E6
:10298000887151F4048D158D268D378D098B1A8B26
:102990002B8B3C8B81E00BC08031F9F49E012F5EC4
:1029A0003F4F898D9A8D72D48823B9F084E08B8350
:1029B0008F2D8F7089831C821D821E821F82188634
:1029C00019861A861B86F4FE0BC040E050E0BA015F
:1029D000CE01F0DE811104C011C01B8280E00EC068
:1029E000F5FE0BC049895A896B897C89CE01DF913C
:1029F000CF911F910F91FF90EDCD81E0DF91CF91AD
:102A00001F910F91FF900895AF92BF92CF92DF92E6
:102A1000EF92FF920F931F93CF93DF937C01EB0113
:102A20006A01B22E898D9A8DF701928F818F40E0D5
:102A300050E0BA01CE01CEDDA12C088519852A858A
:102A40003B8589899A89AB89BC89081719072A07A8
:102A50003B07A0F585E036952795179507958A954C
:102A6000D1F70F70CE0185DD009709F481C0FC011C
:102A70002081222311F0253EB9F4A1100EC040910F
:102A8000EB075091EC076091ED077091EE07F701AD
:102A90004487558766877787008BFC018081AA244D
:102AA000A3948111CACF0AC04BE050E0BC01C6011B
:102AB0000E94BFB6892B09F0C0CF58C08B2D8274FD
:102AC000823409F055C0AA2049F0F701008961E07D
:102AD000C701DDDAEC01009769F44AC08B818230CE
:102AE00009F446C0CE014BDA882309F441C0CBEE8D
:102AF000D5E000E080E2FE0111928A95E9F78BE0D3
:102B0000F601DE0101900D928A95E1F7E091E20570
:102B1000F091E305309739F0BE01625F7F4FCE013F
:102B20004096199508C081E298E2998B888B80E0E5
:102B300098E09F878E87888999899B8B8A8B998F4C
:102B4000888F8E859F859F8B8E8BA9D2882381F05D
:102B50004B2D602FC701DF91CF911F910F91FF90F7
:102B6000EF90DF90CF90BF90AF90D5CEB7FEF0CF73
:102B700080E0DF91CF911F910F91FF90EF90DF9058
:102B8000CF90BF90AF9008953F924F925F926F9217
:102B90007F928F929F92AF92BF92CF92DF92EF92ED
:102BA000FF920F931F93CF93DF93CDB7DEB7C3543C
:102BB000D1090FB6F894DEBF0FBECDBF5C016B012B
:102BC00024965FAF4EAF2497522E1C8E1F8E198213
:102BD0001C826115710511F410E073C0FC01838142
:102BE0008111FACF2496EEADFFAD249780818F320C
:102BF00011F076011DC02496EEADFFAD24978081C3
:102C00008F3231F431962496FFAFEEAF2497F3CF95
:102C1000F60183818250823060F3F601618D728DFE
:102C2000CE010196C7DA8823B9F2CE0101967C0164
:102C30008E01045E1F4F3801FE0131964F01402E78
:102C4000312E19C08823A9F121E0AE01495C5F4F04
:102C5000B701C801D9DE882309F4BECFEC14FD0406
:102C600011F0C7019ADD0615170501F1942D832D8A
:102C70007801092F182FAE014E5B5F4FBE01695CD2
:102C80007F4F24968EAD9FAD249755DA882309F4A3
:102C9000A3CF2496EEADFFAD249780818F3291F6BD
:102CA00031962496FFAFEEAF2497F3CF982D892D60
:102CB000DFCF252DAE01495C5F4FB701C501A4DE12
:102CC000182FCE01019671DDCE014C966EDD812F5D
:102CD000CD5BDF4F0FB6F894DEBF0FBECDBFDF91E7
:102CE000CF911F910F91FF90EF90DF90CF90BF9009
:102CF000AF909F908F907F906F905F904F903F909C
:102D00000895CF93DF93EC0140E050E0BA0152DD2B
:102D1000882361F061E0CE01BAD9009739F025EE41
:102D2000FC0120831B82DF91CF91B9C180E0DF914C
:102D3000CF9108951F93CF93DF93CDB7DEB76B97F5
:102D40000FB6F894DEBF0FBECDBFAB0119821C8257
:102D500022E0BC01CE01019617DF182F882321F055
:102D6000CE010196CEDF182FCE0101961EDD812FF8
:102D70006B960FB6F894DEBF0FBECDBFDF91CF913B
:102D80001F9108952F923F924F925F926F927F9280
:102D90008F929F92AF92BF92CF92DF92EF92FF926B
:102DA0000F931F93CF93DF9300D01F921F92CDB745
:102DB000DEB78C015B013A01DC0113968C9113970D
:102DC0008130C1F411968C9181FF14C082FF18C02C
:102DD000F801418952896389748980859185A2852A
:102DE000B38584179507A607B70751F0C801F2DB32
:102DF000811106C081E0F80180838FEF9FEF37C11A
:102E0000630183C0D80159968D919C915A97FC011A
:102E1000F481F1501A012B0169E0569447943794DC
:102E200027946A95D1F7F221FD834A0121E092228D
:102E3000FF2309F476C080E092E0881999097601B1
:102E40008C159D0508F47C01D8015996ED91FC91F3
:102E50005A9714962D903D904D905C901797B2E044
:102E60002B1A310841085108058404C0220C331C78
:102E7000441C551C0A94D2F786859785A089B18990
:102E8000280E391E4A1E5B1EED812E0E311C411C80
:102E9000511CE114F2E0FF0609F089C08091EB07B4
:102EA0009091EC07A091ED07B091EE078215930584
:102EB000A405B50569F41092E8058FEF9FEFDC01DA
:102EC0008093EB079093EC07A093ED07B093EE0788
:102ED0009501B201A1018091E9059091EA050E9456
:102EE000D53C882309F486CFF80180859185A28599
:102EF000B3858E0D9F1DA11DB11D80879187A2876F
:102F0000B387AE0CBF1CCE18DF08D80118964D91C0
:102F10005D916D917C911B97C114D10409F072CF22
:102F20007AC08114910409F086CF14964D915D9179
:102F30006D917C911797411551056105710559F403
:102F400055968D919D910D90BC91A02D0097A10556
:102F5000B10539F520C09E012F5F3F4F18D188235E
:102F600009F448CF89819A81AB81BC81F801218D18
:102F7000328DF9012789203139F4883FFFEF9F070F
:102F8000A105B10540F40DC0883F2FEF9207A207BD
:102F90002FE0B20730F0C8010E94990F81114BCF8A
:102FA00029CFF80184839583A683B78344CF811406
:102FB000910411F5D80118964D915D916D917C9118
:102FC0001B9751968D919D910D90BC91A02D481706
:102FD00059076A077B0780F062D0882309F40ACF7B
:102FE00081E08093E8052092EB073092EC07409255
:102FF000ED075092EE0707C041E0C201B1018FD04A
:10300000882309F4F7CEA701B501C40185519A4F71
:103010000E94CCB669CF51968D919D910D90BC9137
:10302000A02DF801218184179507A607B70738F46A
:10303000418B528B638B748B206821830CC08091F1
:10304000E2059091E305892B31F06114710419F0C8
:103050002068F8012183D80111968C9183FD02C06C
:10306000C30105C0C8014FDB8111FACFC3CE0F9059
:103070000F900F900F900F90DF91CF911F910F91B4
:10308000FF90EF90DF90CF90BF90AF909F908F9088
:103090007F906F905F904F903F902F900895CF93C7
:1030A0008091E8058823B9F14091EB075091EC0736
:1030B0006091ED077091EE072BEE35E08091E90508
:1030C0009091EA050E94D53CC82F811102C0C0E052
:1030D00023C04091E4055091E5056091E6057091AB
:1030E000E705411551056105710591F02BEE35E0BD
:1030F0008091E9059091EA050E94D53C882339F337
:103100001092E4051092E5051092E6051092E7058D
:103110001092E80501C0C1E08C2FCF910895CF92A5
:10312000DF92EF92FF92CF936B017C01C42F8091CD
:10313000EB079091EC07A091ED07B091EE078C158D
:103140009D05AE05BF05C9F0AADF811102C080E070
:1031500018C02BEE35E0B701A6018091E9059091EA
:10316000EA050E94603C882391F3C092EB07D0925D
:10317000EC07E092ED07F092EE0781E0C111809339
:10318000E805CF91FF90EF90DF90CF9008958F9258
:103190009F92AF92BF92CF92DF92EF92FF920F93E6
:1031A0001F93CF93DF93EC016A017B01890189852D
:1031B0009A85AB85BC850196A11DB11D8417950725
:1031C000A607B70710F480E054C08F89803129F436
:1031D0009927872F762F652F0BC08032A1F7CB015F
:1031E000BA0127E096958795779567952A95D1F747
:1031F0008B889C88AD88BE88680D791D8A1D9B1DB3
:103200008090EB079090EC07A090ED07B090EE0750
:10321000681579058A059B0581F48F89803191F4C1
:10322000DD24EE24FF24F601EE0FFF1FE551FA4FD7
:1032300080819181A0E0B0E016C040E070DF811194
:10324000ECCFC1CFE894C7F8DD24EE24FF24F601CB
:10325000EE0FFF1FEE0FFF1FE551FA4F80819181A6
:10326000A281B381BF70F80180839183A283B3836D
:1032700081E0DF91CF911F910F91FF90EF90DF9050
:10328000CF90BF90AF909F908F9008954F925F9294
:103290006F927F92AF92BF92CF92DF92EF92FF92A6
:1032A0000F931F93CF93DF9300D01F92CDB7DEB75C
:1032B0008C0149835A836B837C835901C12CD12CA7
:1032C0007601412C42E0542E612C712C49815A81A7
:1032D0006B817C819E012F5F3F4FC80158DF88239F
:1032E00041F1D301C201F801058404C0880F991F80
:1032F000AA1FBB1F0A94D2F7C80ED91EEA1EFB1ED6
:1033000049815A816B817C818789803139F481E0E0
:10331000483F5F4F6105710538F4D8CF81E0483FE1
:103320005F4F6F4F7F4090F2F501C082D182E28201
:10333000F3820F900F900F900F90DF91CF911F911C
:103340000F91FF90EF90DF90CF90BF90AF907F9064
:103350006F905F904F9008954F925F926F927F921F
:103360008F929F92AF92BF92CF92DF92EF92FF9295
:103370000F931F93CF93DF93EC014A015B01280168
:103380003901423051056105710508F462C0498573
:103390005A856B857C854F5F5F4F6F4F7F4F481518
:1033A00059056A057B0508F454C08F89803129F4DA
:1033B000FF24EB2CDA2CC92C0CC0803209F049C058
:1033C0007501640177E0F694E794D794C7947A95F1
:1033D000D1F74B895C896D897E89C40ED51EE61EA6
:1033E000F71E41E0C701B6019ADE882391F19F895B
:1033F000903159F49924AA24BB24F401EE0FFF1F45
:10340000E551FA4F5182408210C0E89487F8992420
:10341000AA24BB24F401EE0FFF1FEE0FFF1FE5519E
:10342000FA4F40825182628273829A89923090F080
:103430004D815E816F8178854C0D5D1D6E1D7F1DF8
:103440004093E4055093E5056093E6057093E70526
:1034500001C080E0DF91CF911F910F91FF90EF901D
:10346000DF90CF90BF90AF909F908F907F906F90A4
:103470005F904F9008952F923F924F925F926F927C
:103480007F928F929F92AF92BF92CF92DF92EF92F4
:10349000FF920F931F93CF93DF93CDB7DEB72F9794
:1034A0000FB6F894DEBF0FBECDBF1C014C875D8701
:1034B0006E877F873B872A87DC0119960D911D91C6
:1034C0002D913C911C970F5F1F4F2F4F3F4F0D8346
:1034D0001E832F833887EA85FB8580809180A280B8
:1034E000B38081149104A104B10431F0FFEF8F1A6D
:1034F0009F0AAF0ABF0A10C0DC018D909D90AD906D
:10350000BC90B1E0B9870C851D852E853F850130C3
:1035100011052105310509F0198675016401412C59
:10352000512C3201F10181859285A385B48548161D
:1035300059066A067B0608F04EC00D811E812F8158
:1035400038850C151D052E053F0550F4F2E0CF2EF1
:10355000D12CE12CF12CA2E08A2E912CA12CB12CA3
:103560009E012F5F3F4FB701A601C10110DE8823E6
:1035700091F149815A816B817C81D701C601019605
:10358000A11DB11D452B462B472B19F04C015D01A8
:103590000FC0AC01BD01481959096A097B090C85A6
:1035A0001D852E853F85401751076207730741F03F
:1035B0001FEF411A510A610A710A6C017D01B2CFF5
:1035C0000FEF1FEF2FEF3FE0B701A601C101C4DEEF
:1035D0008D83811113C01D823DC02601370121E07A
:1035E000421A51086108710897018601B301A201CE
:1035F000C101B2DE882379F3730162018C149D044A
:10360000AE04BF0450F3AA85BB854D915D916D91C9
:103610007C914115510561057105A9F4EA85FB8589
:1036200080829182A282B382F985FF2399F00FEF05
:10363000801A900AA00AB00AD1018D929D92AD9293
:10364000BC92139707C095018401C10185DE8111E9
:10365000E5CFC1CF8D812F960FB6F894DEBF0FBE98
:10366000CDBFDF91CF911F910F91FF90EF90DF9031
:10367000CF90BF90AF909F908F907F906F905F9012
:103680004F903F902F900895AF92BF92CF92DF92CC
:10369000EF92FF920F931F93CF93DF9300D01F926F
:1036A000CDB7DEB75C016A017B0182E090E0A0E06B
:1036B000B0E0F50180839183A283B3839E012F5FE5
:1036C0003F4FB701A601C50162DD811102C080E054
:1036D00023C000E010E09801B701A601C5013CDE5F
:1036E0008823A9F3C980DA80EB80FC80F501878903
:1036F000803149F481E0F8EFCF16FFEFDF06E104F7
:10370000F10450F4DBCF81E098EFC9169FEFD906A2
:10371000E9069FE0F90690F20F900F900F900F903E
:10372000DF91CF911F910F91FF90EF90DF90CF909D
:10373000BF90AF9008957F928F929F92AF92BF9269
:10374000CF92DF92EF92FF920F931F93CF93DF936D
:10375000EC01142F7093EA056093E9051F8A82E05B
:1037600090E0A0E0B0E088839983AA83BB831092A5
:10377000E8051092E4051092E5051092E605109216
:10378000E7058FEF9FEFDC018093EB079093EC0749
:10379000A093ED07B093EE07442349F1453008F0BC
:1037A000DEC040E060E070E0CB01B9DC882309F4C2
:1037B000D6C020E1129FF0011124E756F84F808116
:1037C0008F7709F0CCC084859585A685B78584362A
:1037D0009105A105B10508F4C2C0C084D184E2847A
:1037E000F384C114D104E104F10421F4B8C0C12C64
:1037F000D12C760140E0C701B60191DC782E8823F8
:1038000009F4ADC08091F6059091F70581159240BD
:1038100009F0A5C03091FB05332309F4A0C08091C5
:10382000F9059091FA05892B09F499C02091F805C2
:10383000222309F494C03A8B2C831D8630E041E0AA
:1038400050E06D85062FCA01062E02C0880F991F11
:103850000A94E2F72817390731F081E0860F8D8747
:10386000683078F37CC02091010630910206211562
:10387000310519F040E050E008C020910F0630916A
:10388000100640911106509112062D833E834F83FE
:1038900058878091F9059091FA0546015701880EE5
:1038A000991EA11CB11C8B8A9C8AAD8ABE8AE091AC
:1038B000FC05F091FD05F98FE88FA091FB05B0E0C4
:1038C0000E949FB3680D791D8A1D9B1D6A8F7B8F97
:1038D0008C8F9D8FB5E0EE0FFF1FBA95E1F7E15099
:1038E000FE4FEF2FFF27E695DC01CB018E0F9F1FC8
:1038F000A11DB11D8E879F87A88BB98B8090FE0577
:103900009090FF058114910419F0A12CB12C08C0EE
:1039100080900B0690900C06A0900D06B0900E06BD
:10392000A7019601281B390B4A0B5B0BDA01C90171
:10393000880D991DAA1DBB1D04C0B695A795979526
:1039400087950A95D2F789879A87AB87BC87853F89
:103950003FE09307A105B10520F48CE08F8B712C1B
:1039600015C0853F9F4FA105B10510F480E10DC042
:103970008091170690911806A0911906B0911A0629
:103980008A8F9B8FAC8FBD8F80E28F8B872DDF91CD
:10399000CF911F910F91FF90EF90DF90CF90BF904C
:1039A000AF909F908F907F9008954F925F926F920B
:1039B0007F928F929F92AF92BF92CF92DF92EF92BF
:1039C000FF920F931F93CF93DF932C0124EF33E0EB
:1039D00081E090E0F90145915491441655060CF0B0
:1039E00062C0AC0141505109DA01AA0FBB1FAA0FF6
:1039F000BB1FAE50BC4FFD0165917491440F551F24
:103A0000440F551F40515C4FFA0165907490FC01C2
:103A1000EE0FFF1FEE0FFF1FEE50FC4FA590B4906E
:103A2000FD0105911491F901C591D491FA01859098
:103A30009490882777FD8095982F0E9419B06B018C
:103A40007C01B20166197709882777FD8095982F48
:103A50000E9419B02B013C01B501601B710B882736
:103A600077FD8095982F0E9419B09B01AC01C3018E
:103A7000B2010E944CB22B013C01BE0168197909C8
:103A8000882777FD8095982F0E9419B09B01AC0183
:103A9000C301B2010E947EAF9B01AC01C701B60118
:103AA0000E949EAE11C001962C5F3F4F8D33910551
:103AB00009F090CFE2EEF4E065917491882777FDEC
:103AC0008095982F0E9419B0DF91CF911F910F918F
:103AD000FF90EF90DF90CF90BF90AF909F908F902E
:103AE0007F906F905F904F9008954F925F926F928A
:103AF0007F928F929F92AF92BF92CF92DF92EF927E
:103B0000FF920F931F93CF93DF932C01662371F1E4
:103B1000E6EBFEE08491882341F09091C00095FF90
:103B2000FCCF8093C6003196F5CF70E04AE050E0BC
:103B30008CE99DE00E94318BE9E5F2E084918823D5
:103B400041F09091C00095FFFCCF8093C600319664
:103B5000F5CF8091C00085FFFCCF8AE08093C6003E
:103B60000E94104660E070E0CB017EC024E733E0A5
:103B700081E090E0F90145915491441655060CF00E
:103B800062C0AC0141505109DA01AA0FBB1FAA0F54
:103B9000BB1FAE58BC4FFD0165917491440F551F7A
:103BA000440F551F40595C4FFA0165907490FC0119
:103BB000EE0FFF1FEE0FFF1FEE58FC4FA590B490C5
:103BC000FD0105911491F901C591D491FA018590F7
:103BD0009490882777FD8095982F0E9419B06B01EB
:103BE0007C01B20166197709882777FD8095982FA7
:103BF0000E9419B02B013C01B501601B710B882795
:103C000077FD8095982F0E9419B09B01AC01C301EC
:103C1000B2010E944CB22B013C01BE016819790926
:103C2000882777FD8095982F0E9419B09B01AC01E1
:103C3000C301B2010E947EAF9B01AC01C701B60176
:103C40000E949EAE11C001962C5F3F4F80329105BD
:103C500009F090CFEEEEF3E065917491882777FD3F
:103C60008095982F0E9419B0DF91CF911F910F91ED
:103C7000FF90EF90DF90CF90BF90AF909F908F908C
:103C80007F906F905F904F90089560E0809144081E
:103C9000909145082ADF6093400870934108809313
:103CA00042089093430880913E0890913F087DDE42
:103CB00060933A0870933B0880933C0890933D08CA
:103CC0008FB7F894109232088FBF08952091140294
:103CD00030911502409116025091170260E070E099
:103CE0008FE793E40E947EAF6093120870931308ED
:103CF0008093140890931508089597FF03C080914E
:103D0000390804C0FC01E45FF74F808190E008951A
:103D1000CF93DF93D82FC62FC19561E00E9428A9C9
:103D20006C2F8D2F0E9461A96C2F70E08D2FDF9179
:103D3000CF910C941EA8CF93C1E020E030E048E47E
:103D400052E460914008709141088091420890913E
:103D500043080E947AB118160CF0C0E06C2F88E07E
:103D600090E0CF91D5CF2F923F924F925F926F927A
:103D70007F928F929F92AF92BF92CF92DF92EF92FB
:103D8000FF920F931F93CF93DF93CDB7DEB72897A2
:103D90000FB6F894DEBF0FBECDBF809132088823E6
:103DA00009F4F8C172DF8090400890904108A0901B
:103DB0004208B09043080091480810914908B801A2
:103DC000882777FD8095982F0E9419B0A50194014E
:103DD0000E949DAE6B017C0160931A0870931B08D2
:103DE00080931C0890931D0820E030E040E251E4ED
:103DF0000E947AB1181624F481E080931108F7C06C
:103E000020E030E040E251ECC701B6010E9477AFFC
:103E100087FD02C0012B21F481E0809311080CC1C1
:103E200080911108882351F010922E0810922F08CB
:103E30001092300810923108109211082091180247
:103E40003091190240911A0250911B02C701B6012C
:103E50000E944CB269837A838B839C83609326088B
:103E600070932708809328089093290820912E08A2
:103E700030912F084091300850913108C701B601A8
:103E80000E949EAE2B013C0120901608309017082E
:103E900010911808009119089101412F502F0E948C
:103EA00077AF87FD14C0209012083090130810914E
:103EB0001408009115089101412F502FB201C30140
:103EC0000E947AB118161CF01201162D072DC1019F
:103ED000A12FB02F80932E0890932F08A093300825
:103EE000B0933108209114023091150240911602CE
:103EF00050911702B101812F902F0E944CB26D8317
:103F00007E838F8398876093220870932308809321
:103F100024089093250820912A0830912B0840917D
:103F20002C0850912D08C501B4010E949DAE20912E
:103F300010023091110240911202509113020E941E
:103F40004CB220ED3CEC4CE45DE30E944CB22B0102
:103F50003C0123E333E343E75FE360911E08709184
:103F60001F0880912008909121080E944CB29B016B
:103F7000AC01C301B2010E949EAE2B013C016093D3
:103F80001E0870931F0880932008909321082D81AC
:103F90003E814F81588569817A818B819C810E9405
:103FA0009EAEA30192010E949DAE2B013C0120E038
:103FB00030E04FE753E40E947AB120E030E0A901FD
:103FC0001816E4F4C701B6010E947AB118167CF401
:103FD000A7019601B101812F902F0E949DAE6093A1
:103FE0002E0870932F088093300890933108412C4D
:103FF000512C9FE7692E93E4792E21C0C301B201B1
:104000000E9477AF87FF1BC020E030E0A901C70105
:10401000B6010E9477AF87FF0FC0A7019601B101DB
:10402000812F902F0E949DAE60932E0870932F08D1
:104030008093300890933108412C512C32018092AA
:104040002A0890922B08A0922C08B0922D0860911B
:10405000040870910508882777FD8095982F0E94A5
:1040600019B09B01AC01C501B4010E947AB11816C8
:10407000DCF46091080270910902882777FD809531
:10408000982F0E9419B09B01AC01C501B4010E9498
:1040900077AF87FF09C0C301B2010E94E6AF7595F3
:1040A000679560930C0802C010920C080E9408AA41
:1040B000009108081091090820910A0830910B0816
:1040C000601B710B820B930B653C79408105910558
:1040D00058F031DE0E9408AA60930808709309081E
:1040E00080930A0890930B080E9408AA00910D087B
:1040F00010910E0820910F0830911008601B710B71
:10410000820B930B683873418105910508F442C016
:104110000E9408AA60930D0870930E0880930F0800
:1041200090931008C0903A08D0903B08E0903C086B
:10413000F0903D0820E030E040E751E4C701B601CF
:104140000E947AB118161CF520E030E046E153E4F5
:10415000C701B6010E9477AF87FF19C0609146087A
:1041600070914708882777FD8095982F0E9419B095
:104170009B01AC01C701B6010E947AB187FD03C063
:104180001092390807C08FE78093390803C0109256
:104190003908A59828960FB6F894DEBF0FBECDBF9C
:1041A000DF91CF911F910F91FF90EF90DF90CF9013
:1041B000BF90AF909F908F907F906F905F904F9047
:1041C0003F902F900895CF93DF931092160810928E
:1041D00017081092180810921908209114023091B3
:1041E0001502409116025091170260E070E08FE7CF
:1041F00093E40E947EAF609312087093130880933B
:104200001408909315086D9A809101018061809344
:1042100001019D9A8091010188608093010187EDE1
:1042200080937A0010927E0010927D0080917E0033
:10423000816080937E0080917E00826080937E000A
:1042400080917E00846080937E0080E888BD8091AC
:104250006E00846080936E006AEF70E080E090E012
:104260000E9437AA8FE090E090930508809304089D
:1042700060E080910A0290910B0237DC20E030E090
:1042800040E751E40E9477AF87FF0AC080910A029D
:1042900090910B02409790930B0280930A02E8CF13
:1042A00086E391E0909309028093080260E0809198
:1042B00006089091070819DC20E030E04BE953E450
:1042C0000E947AB1181654F480910608909107085C
:1042D00040969093070880930608E8CFC0910208A3
:1042E000D0910308CE0161DB20E030E046E153E4E9
:1042F0000E947AB1181634F46096D0930308C093E4
:104300000208ECCFDF91CF910895089510924908EB
:1043100010924808109247081092460810920C0814
:104320007598109247081092460810923908A5987F
:1043300008952F923F924F925F926F927F928F9249
:104340009F92AF92BF92CF92DF92EF92FF920F9324
:104350001F93CF93DF93CDB7DEB7AE970FB6F89428
:10436000DEBF0FBECDBF6B8F7C8F8D8F292E5A87FE
:1043700049873CA72BA70E9408AA6F8F78A389A31F
:104380009AA30E9408AA6FA378A789A79AA729854C
:104390003A85121613061CF0E4E2F3E017C0E7E3D7
:1043A000F3E08191882339F09091C00095FFFCCF14
:1043B0008093C600F6CF8091C00085FFFCCF1BC262
:1043C0009091C00095FFFCCF8093C6008191811130
:1043D000F7CF8091C00085FFFCCF8AE08093C600B4
:1043E00095DF49855A858FE7452B99F180933908E8
:1043F0008F8D98A1A9A1BAA1898B9A8BAB8BBC8B0D
:104400008D879E87AF87B88B1D8290E4988FACE133
:10441000A98FB6E4BA8F1DA61D8A1E8A1F8A2FE7B0
:1044200030E040E050E029833A834B835C83EFE740
:104430004E2E512C612C712C1BA21CA21DA21EA25F
:1044400031E03E8F1C861B86312C00E010E01EA65A
:1044500005C080930C08CCCF0E94767780913208FB
:10446000882309F4F6C011DC49855A85452B51F0A3
:1044700030903A0800913B0810913C0850913D085B
:104480005EA709C030904008009141081091420891
:10449000809143088EA7232D302F412F5EA56DA557
:1044A0007D898E899F890E947AB118162CF03DA6CD
:1044B0000D8B1E8B9EA59F8B232D302F412F5EA52C
:1044C0006D81788D898D9A8D0E9477AF87FD05C0AB
:1044D0003D82088F198FAEA5AA8F0E9408AA2FA12E
:1044E00038A549A55AA5621B730B840B950B653C37
:1044F00079408105910538F01EDC0E9408AA6FA35F
:1045000078A789A79AA74E8D442309F44FC02B8D15
:104510003C8D4D8D522D632D702F812F9EA50E94B5
:104520007AB118160CF095C00E9408AA29893A8918
:104530004B895C89621B730B840B950B6938734143
:104540008105910508F485C0D301C20129813A8112
:104550004B815C81821B930BA40BB50B49855A855B
:10456000B595A79597958795452B19F080933908B0
:1045700002C080930C080E9408AA6D877E878F87EF
:10458000988BDC01CB0129893A894B895C89821B94
:10459000930BA40BB50B8BA39CA3ADA3BEA33B8D28
:1045A0003DA74C8D4D8B5D8D5E8B2F8A2B8D3C8D69
:1045B0004D8D522D632D702F812F9EA50E9477AFB8
:1045C00087FFEEC20E9408AA2D853E854F85588937
:1045D000621B730B840B950B693873418105910540
:1045E00008F4DEC20E9408AA698B7A8B8B8B9C8BA5
:1045F000DC01CB012D853E854F855889821B930BAD
:10460000A40BB50B4B855C85452B09F010C1898146
:104610009A81AB81BC81840D951DA61DB71D29858E
:104620003A85B595A79597958795232B09F4B5C23B
:10463000809339084B855C854F5F5F4F5C874B8764
:104640005B8D5D838C8D888F9D8D998F2A8EA1E0E7
:10465000AE8F20E030E040EA51E46B8D7C8D8D8D93
:10466000922D0E949EAE9B01AC01632D702F812F75
:104670009EA50E947AB1181694F4EFEFF2E08491AF
:10468000882341F09091C00095FFFCCF8093C60035
:104690003196F5CF8091C00085FFFCCFACC00E9461
:1046A00008AA2F8D38A149A15AA1621B730B840B54
:1046B000950B613D77408105910508F44FC0498510
:1046C0005A85452B81F0E0903908F12CE9EFF2E0B2
:1046D00084918823C1F09091C00095FFFCCF809316
:1046E000C6003196F5CFE0900C08F12CE3EFF2E034
:1046F0008491882341F09091C00095FFFCCF809376
:10470000C6003196F5CF22E030E0432D502F612FC7
:104710007EA58CE99DE00E94078CEFEEF2E084918B
:10472000882341F09091C00095FFFCCF8093C60094
:104730003196F5CF4AE050E0B7018CE99DE00E9448
:10474000318B8091C00085FFFCCF8AE08093C6004A
:104750000E9408AA6F8F78A389A39AA30E9408AA2F
:104760006B017C010E9408AA89889A88AB88BC8862
:104770002D853E854F855889820E931EA41EB51E39
:10478000C818D908EA08FB08C60ED71EE81EF91E8D
:1047900031E8C3163FE4D30632E1E306F10490F0BA
:1047A000E2EDF2E08491882341F09091C00095FF02
:1047B000FCCF8093C6003196F5CF8091C00085FF75
:1047C000FCCF19C04B855C858BA59CA584179507EC
:1047D0000CF042CEE6E7F2E08491882341F090911C
:1047E000C00095FFFCCF8093C6003196F5CF809135
:1047F000C00085FFFCCF8AE08093C600AE960FB65E
:10480000F894DEBF0FBECDBFDF91CF911F910F9106
:10481000FF90EF90DF90CF90BF90AF909F908F90E0
:104820007F906F905F904F903F902F9008958BA056
:104830009CA0ADA0BEA0880E991EAA1EBB1E2BA1D7
:104840003CA14DA15EA1281B390B4A0B5B0BCA0191
:10485000B90129813A814B815C810E9412B3A50183
:1048600094010E9477B3240D351D461D571D243138
:1048700031054105510504F129013A013CEE431689
:104880005104610471042CF06BEE462E512C612C06
:10489000712C40E84416510461047104DCF08EEF81
:1048A00090E0A0E0B0E084199509A609B7098983D2
:1048B0009A83AB83BC8312C054E1452E512C612CEA
:1048C000712C24E130E040E050E029833A834B83AF
:1048D0005C8304C049825A826B827C82E8E6F3E002
:1048E0008491882341F09091C00095FFFCCF809384
:1048F000C6003196F5CF2AE030E0B301A2018CE981
:104900009DE00E94068BE3E6F3E08491882341F06A
:104910009091C00095FFFCCF8093C6003196F5CFF3
:104920002AE030E049815A816B817C818CE99DE0ED
:104930000E94068BECE5F3E08491882341F090918E
:10494000C00095FFFCCF8093C6003196F5CF22E0E2
:1049500030E04D81588D698D7A8D8CE99DE00E9403
:10496000078CE5E5F3E08491882341F09091C00045
:1049700095FFFCCF8093C6003196F5CF22E030E062
:104980004DA55D896E897F898CE99DE00E94078C29
:104990008091C00085FFFCCF8AE08093C6002B8504
:1049A0003C85233031050CF432CE69817A818B81CC
:1049B0009C810E9419B020E030E040E850E40E9461
:1049C0004CB26B017C012D81388D498D5A8D6DA5BE
:1049D0007D898E899F890E949DAE20ED3FE049E44C
:1049E00050E40E944CB220E030E040E05FE30E94DF
:1049F0004CB29B01AC01C701B6010E947EAF6B01B6
:104A00007C01C501B4010E9419B020E030E04AE702
:104A100054E40E947EAF4B015C01EFE4F3E084912B
:104A2000882341F09091C00095FFFCCF8093C60091
:104A30003196F5CF22E030E0B701A6018CE99DE088
:104A40000E94078CE9E4F3E08491882341F090917F
:104A5000C00095FFFCCF8093C6003196F5CF22E0D1
:104A600030E0B501A4018CE99DE00E94078C8091A3
:104A7000C00085FFFCCF8AE08093C6002AE939E9AF
:104A800049E15FE3C701B6010E944CB26B017C01B2
:104A90009B01AC010E949EAEA50194010E947EAFD5
:104AA0006D837E838F839887A5019401C701B6012A
:104AB0000E944CB220E030E040E05EE30E944CB245
:104AC0004B015C01EBE3F3E08491882341F090918A
:104AD000C00095FFFCCF8093C6003196F5CF809142
:104AE000C00085FFFCCF8AE08093C600E5E3F3E0D9
:104AF0008491882341F09091C00095FFFCCF809372
:104B0000C6003196F5CF22E030E0B701A6018CE96E
:104B10009DE00E94078C8091C00085FFFCCF8AE059
:104B20008093C600EFE2F3E08491882341F09091F6
:104B3000C00095FFFCCF8093C6003196F5CF22E0F0
:104B400030E04D815E816F8178858CE99DE00E9427
:104B5000078C8091C00085FFFCCF8AE08093C6005F
:104B6000E9E2F3E08491882341F09091C00095FF41
:104B7000FCCF8093C6003196F5CF22E030E0B5013E
:104B8000A4018CE99DE00E94078C8091C00085FF04
:104B9000FCCF8AE08093C6003ACD80930C084ACDC2
:104BA0001E8E57CDCF93C82FB1DB0E94D74A8111FB
:104BB00034C0E6EBFEE09491992341F08091C0006F
:104BC00085FFFCCF9093C6003196F5CF6C2F70E037
:104BD0004AE050E08CE99DE00E94318B8091C0005A
:104BE00085FFFCCF8AE08093C600ECE2F2E084917E
:104BF000882341F09091C00095FFFCCF8093C600C0
:104C00003196F5CF8091C00085FFFCCF8AE080937C
:104C1000C6008FE192E00E94D476CF910C94984A1E
:104C2000CF93C82F73DB0E94D74A811134C0E6EBC3
:104C3000FEE09491992341F08091C00085FFFCCF64
:104C40009093C6003196F5CF6C2F70E04AE050E0AB
:104C50008CE99DE00E94318B8091C00085FFFCCFE4
:104C60008AE08093C600E2EFF1E08491882341F06E
:104C70009091C00095FFFCCF8093C6003196F5CF90
:104C80008091C00085FFFCCF8AE08093C60085EE4E
:104C900091E00E94D476CF910C94984AA5980E94F6
:104CA000D74A811125C0E6EBFEE08491882341F0CC
:104CB0009091C00095FFFCCF8093C6003196F5CF50
:104CC000EBEAF1E08491882341F09091C00095FFD8
:104CD000FCCF8093C6003196F5CF8091C00085FF50
:104CE000FCCF8AE08093C6008AE991E00E94D476E6
:104CF0000C94984A1F920F920FB60F9211240BB684
:104D00000F920F931F932F933F934F935F936F9344
:104D10007F938F939F93AF93BF93CF93DF93EF9343
:104D2000FF9380910702811112C080910C0880933B
:104D30000108882311F0759A01C07598809139088F
:104D400080930008882311F0A59A01C0A59890913E
:104D5000010880910702981708F47598909100084F
:104D600080910702981708F4A598809107028F5F39
:104D70008F77809307028091060290E08B30910537
:104D800008F093C0FC01EE58FF4F0C9493B31092BF
:104D90007B0080E480937C0080917A008064809323
:104DA0007A000E94DD7681E019C020917800309170
:104DB00079008091FC079091FD07A091FE07B091CA
:104DC000FF07820F931FA11DB11D8093FC079093D5
:104DD000FD07A093FE07B093FF0782E080930602D1
:104DE00064C010927B0082E480937C0080917A0002
:104DF000806480937A000E94DD7683E0EFCF20917B
:104E00007800309179008091F8079091F907A0918E
:104E1000FA07B091FB07820F931FA11DB11D80936C
:104E2000F8079093F907A093FA07B093FB0784E083
:104E3000D5CF10927B0081E480937C0080917A0032
:104E4000806480937A000E94DD7685E0C7CF209150
:104E50007800309179008091F4079091F507A09146
:104E6000F607B091F707820F931FA11DB11D809324
:104E7000F4079093F507A093F607B093F70786E041
:104E8000ADCF0E94DD7687E0A9CF88E0A7CF0E9452
:104E9000DD7689E0A3CF109206028091F3078F5F41
:104EA0008093F30702C0109206028091F3078031CD
:104EB00008F463C080913208811110C08091FC0712
:104EC0009091FD0790934508809344088091F807DE
:104ED0009091F90790933F0880933E0881E080937A
:104EE00032081092F3071092FC071092FD071092FF
:104EF000FE071092FF071092F4071092F507109228
:104F0000F6071092F7071092EF071092F007109231
:104F1000F1071092F2071092F8071092F907109219
:104F2000FA071092FB0720914408309145088091C0
:104F30000608909107088217930714F080E032DE8C
:104F4000209144083091450880910A0290910B020B
:104F50002817390714F080E063DE20913E08309175
:104F60003F088091020890910308821793072CF064
:104F7000109247081092460891DE00E010E0E80128
:104F8000CC0FDD1FCD5CD74F88819981181619068B
:104F900044F461E0802F0E94AC948881998101974C
:104FA00009C0892B49F060E0802F0E94AC94888171
:104FB00099810196998388830F5F1F4F03301105F4
:104FC000F1F6FF91EF91DF91CF91BF91AF919F915A
:104FD0008F917F916F915F914F913F912F911F9191
:104FE0000F910F900BBE0F900FBE0F901F90189552
:104FF0002CEA35EC47E25EE30C944CB22CEA35EC3B
:1050000047E25EE30C947EAF2CEA35EC47E25EE3C8
:105010000C947EAF2CEA35EC47E25EE30C944CB284
:10502000CF93DF93EC0160E08E810E9461A981E063
:1050300090E00E945BAA61E08E810E9461A981E0FC
:1050400090E00E945BAA60E08E810E9461A984E6E4
:1050500090E0DF91CF910C945BAACF92DF92EF9218
:10506000FF920F931F93CF93DF937C01C0E0D0E0BA
:10507000C62ED12C87010C0F1D1F61E0F80187811E
:105080000E9428A9B6010C2E02C0759567950A9456
:10509000E2F76170F80187810E9461A92196C4300E
:1050A000D10541F7C701DF91CF911F910F91FF907B
:1050B000EF90DF90CF90B4CFCF92DF92EF92FF923C
:1050C0000F931F93CF93DF937C01C0E0D0E0C62EF7
:1050D000D12C87010C0F1D1F61E0F80187810E9410
:1050E00028A9B6010C2E02C0759567950A94E2F7BF
:1050F0006170F80187810E9461A92196C830D105AD
:1051000041F7C701DF91CF911F910F91FF90EF9071
:10511000DF90CF9085CF1F93CF93DF93EC01162FB5
:10512000642F8C810E9461A98D818F3F19F060E00E
:105130000E9461A98F85612F84FF05C0CE01DF9198
:10514000CF911F91B9CF70E084E0759567958A95EE
:10515000E1F7CE0182DF612FCE01DF91CF911F9168
:105160007CCF40E0D8CF61E0FCDF80E496E00C9497
:105170005BAA62E0F6DF80E496E00C945BAACF9332
:10518000DF93CDB7DEB728970FB6F894DEBF0FBE1A
:10519000CDBF28E0E7EAF2E0DE01119601900D9222
:1051A0002A95E1F7FC012389421710F04FEF420FD7
:1051B000FE013196E40FF11DE40FF11D2081260F51
:1051C0002068622F28960FB6F894DEBF0FBECDBFC1
:1051D000DF91CF91C6CFFC016089262F2460208B00
:1051E0006C60BFCFCF93DF93EC01423018F08F8516
:1051F00088608F874B8B1C8A222329F0413019F459
:105200008F8584608F8780E593EC0E945BAA60E0C5
:105210008C810E9461A960E08E810E9461A98D81CC
:105220008F3F19F060E00E9461A96F8564FD19C08D
:1052300063E0CE0112DF84E991E10E945BAA63E0A2
:10524000CE010BDF84E991E10E945BAA63E0CE010D
:1052500004DF86E990E00E945BAA62E0CE01FDDEF9
:1052600013C06062CE017DDF84E991E10E945BAAF8
:105270006F856062CE0175DF86E990E00E945BAACF
:105280006F856062CE016DDF6F856062CE0169DF80
:105290008CE390E00E945BAA84E0888BCE019BDFC8
:1052A0008CE390E00E945BAACE015DDF88EB9BE07F
:1052B0000E945BAA82E0898B66E0CE0152DF8CE31C
:1052C00090E0DF91CF910C945BAA6F927F928F92C6
:1052D000AF92CF92EF920F931F93CF93DF93CDB7FF
:1052E000DEB73C01162F842F5E854F85388999895A
:1052F000F301848325830683E782C086A1868286A4
:10530000538744873587968761E00E9428A9F30177
:1053100085818F3F19F061E00E9428A961E0F301C7
:1053200086810E9428A9112319F0F301178603C072
:1053300080E1F301878720E041E060E1C301DF9174
:10534000CF911F910F91EF90CF90AF908F907F9062
:105350006F9048CF8F92AF92CF92EF920F93DC0174
:1053600013961C921E921297E5E6F3E0ED93FC93E0
:105370001F921F921F921F928C2CAE2CC02EE22ED9
:10538000042F2FEF462F61E0A0DF0F900F900F90BA
:105390000F900F91EF90CF90AF908F900895CF9393
:1053A000DF93EC01423018F08F8588608F874B8B3C
:1053B0001C8A222329F0413019F48F8584608F875D
:1053C00080E593EC0E945BAA60E08C810E9461A959
:1053D00060E08E810E9461A98D818F3F19F060E0AD
:1053E0000E9461A96F8564FD19C063E0CE0135DEBE
:1053F00084E991E10E945BAA63E0CE012EDE84E99C
:1054000091E10E945BAA63E0CE0127DE86E990E08D
:105410000E945BAA62E0CE0120DE13C06062CE0172
:10542000A0DE84E991E10E945BAA6F856062CE01F3
:1054300098DE86E990E00E945BAA6F856062CE01EB
:1054400090DE6F856062CE018CDE8CE390E00E947E
:105450005BAA84E0888BCE01BEDE8CE390E00E94E4
:105460005BAACE0186DE80E496E00E945BAA82E021
:10547000898B66E0CE0175DE8CE390E00E945BAA2A
:1054800040E068E0CE017BDE6EE873E0CE010E9472
:1054900095AE41E068E0CE0172DE6EE873E0CE01C9
:1054A0000E9495AE42E066E0CE0169DE6CE873E0F2
:1054B000CE01DF91CF910C9495AECF92DF92EF9217
:1054C000FF920F931F93CF93DF931F921F92CDB73D
:1054D000DEB78C01677088E0689FB00111246064BA
:1054E000C80149835A833DDE4981C42E5A81D52E95
:1054F000E12CF12CD6016D916D01D801ED91FC915B
:105500000190F081E02DC8011995BFEFEB1AFB0A5D
:10551000E8E0EE16F10471F70F900F90DF91CF9154
:105520001F910F91FF90EF90DF90CF90089541E091
:10553000F2DD81E090E008952F923F924F925F92CA
:105540006F927F928F929F92AF92BF92CF92DF9293
:10555000EF92FF920F931F93CF93DF93CDB7DEB7F8
:10556000CF54D1090FB6F894DEBF0FBECDBF1C01DA
:105570007E8F6D8F4A012FAB09AF2896EFAE28972B
:105580002C96ACAEBDAECEAEDFAE2C9734E0239FF2
:1055900050011124FC01EA0DFB1D80819181A28143
:1055A000B381898F9A8FAB8FBC8FDA01AA0DBB1D97
:1055B000BCAFABAF4D905D906D907C90A30192011C
:1055C000698D7A8D8B8D9C8D0E949EAE21966CAFDD
:1055D0007DAF8EAF9FAF2197B4E00B9F8001112468
:1055E000F101E00FF11F20813181428153812F8F22
:1055F00038A349A35AA3A401400F511F23965FAFBC
:105600004EAF2397DA01CD90DD90ED90FC90A7018D
:1056100096016F8D78A189A19AA10E949EAE2796CE
:105620006CAF7DAF8EAF9FAF27972896EFAD2897D1
:10563000B4E0EB9FC0011124F101E80FF91F2081B4
:105640003181428153812BA33CA34DA35EA3ED8DF9
:10565000FE8DE80FF91F60817181828193810E9424
:105660009DAE6FA378A789A79AA7AD8DBE8D1C9616
:105670008D919D910D90BC91A02D60968CAF9DAFAA
:10568000AEAFBFAF6097D1011C962D913D914D916A
:105690005C911F972BA73CA74DA75EA7A301920182
:1056A00050582D8B3E8B4F8B588FD701C601B05869
:1056B000898B9A8BAB8BBC8BED8DFE8DEA0DFB1D20
:1056C00020813181428153812FA738AB49AB5AAB3E
:1056D00021962CAD3DAD4EAD5FAD21976FA578A95C
:1056E00089A99AA90E949DAE6B017C01ED8DFE8D6A
:1056F000E00FF11F80819181A281B3818BAB9CABC4
:10570000ADABBEAB27962CAD3DAD4EAD5FAD279793
:10571000BC01CD010E949DAE4B015C01A701960129
:105720006D897E898F89988D0E944CB22B013C0136
:10573000A501940169897A898B899C890E944CB260
:105740009B01AC01C301B2010E949EAE2B013C0142
:10575000A50194016D897E898F89988D0E944CB234
:105760004B015C01A701960169897A898B899C8923
:105770000E944CB29B01AC01C501B4010E949DAED8
:10578000A30192010E9411AF6B017C0120E030E087
:10579000A9010E9477AF87FF0AC02BED3FE049ECDB
:1057A00050E4C701B6010E949EAE6B017C01AA962F
:1057B0008FADAA97882351F02BED3FE049EC50E4E0
:1057C000C701B6010E949DAE6B017C012FA538A9CF
:1057D00049A95AA9698D7A8D8B8D9C8D0E9477AFCE
:1057E00081111FC02BA93CA94DA95EA96F8D78A17D
:1057F00089A19AA10E9477AF811113C020E030E007
:10580000A901C701B6010E9477AF81110AC02BED33
:105810003FE049EC50E4C701B6010E949EAE6B0127
:105820007C01A9962CAD3DAD4EAD5FADA997C701EA
:10583000B6010E944CB22FA138A549A55AA55F77A1
:105840000E9487B14B015C012FE632E143E85AE345
:105850000E9477AF87FDC8C1C501B4010E9454B052
:105860000E94EBAF7A8F698FDB01AB2B21F4E1E073
:10587000F0E0FA8FE98F298D3A8DB90180E090E050
:105880000E9417B04B015C019B01AC01C701B6013E
:105890000E947EAF2B013C01A50194016FA178A568
:1058A00089A59AA50E947EAF6FA778AB89AB9AAB0A
:1058B0002BA53CA54DA55EA560966CAD7DAD8EADCE
:1058C0009FAD60970E949DAEA50194010E947EAF9E
:1058D0006BAB7CAB8DAB9EAB20E030E040E05FE398
:1058E000C301B2010E944CB2A30192010E944CB2CA
:1058F0009B01AC0160E070E080E89FE30E949DAEF8
:105900006FA378A789A79AA7CE010196FC012896D4
:105910004FAD289734E0439FE00DF11D11242BA1DA
:105920003CA14DA15EA120833183428353832BA5EB
:105930003CA54DA55EA52D873E874F87588BB12C82
:1059400041E050E058A34F8F1C01BFA9A4E0BA9FCB
:10595000800D911D112498AF8FAB910159AD44E09A
:10596000549F200D311D11243AAF29AFFCA7EBA79E
:105970004F8D58A1898D9A8D4817590708F01AC183
:1059800088E18B150CF444C02FA138A549A55AA570
:1059900069897A898B899C890E944CB26B017C0150
:1059A000A30192016D897E898F89988D0E944CB2E6
:1059B000A70196010E949EAEA62E172F982E892E23
:1059C0002FA138A549A55AA56D897E898F89988D03
:1059D0000E944CB26B017C01A301920169897A8912
:1059E0008B899C890E944CB29B01AC01C701B60116
:1059F0000E949DAE6D8B7E8B8F8B988FB3948A2D7A
:105A0000912FA92DB82D898B9A8BAB8BBC8B6CC039
:105A1000AF8DB8A1BD0180E090E00E9417B0A30156
:105A200092010E944CB26B017C010E947BAF698B9A
:105A30007A8B8B8B9C8BC701B6010E94AFB24B0156
:105A40005C01EBADFCADC080D180E280F380F7FA61
:105A5000F094F7F8F0942396AEADBFAD23972D9157
:105A60003D914D915C912BA33CA34DA35EA329894D
:105A70003A894B895C89C701B6010E944CB26D8B93
:105A80007E8B8F8B988FA50194016BA17CA18DA13A
:105A90009EA10E944CB29B01AC016D897E898F89C9
:105AA000988D0E949EAE6D8B7E8B8F8B988FA501FB
:105AB0009401C701B6010E944CB26B017C01298997
:105AC0003A894B895C896BA17CA18DA19EA10E9422
:105AD0004CB29B01AC01C701B6010E949DAE698B1F
:105AE0007A8B8B8B9C8BB12C2D893E894F89588D5D
:105AF00021966CAD7DAD8EAD9FAD21970E949EAE7F
:105B0000EFA9F8AD608371838283938329893A89F1
:105B10004B895C8927966CAD7DAD8EAD9FAD279787
:105B20000E949EAEA9ADBAAD6D937D938D939C936B
:105B300013972FA538A949A95AA9EBA5FCA56081FF
:105B40007181828193810E949EAEABA5BCA56D93AD
:105B50007D938D939C9313972BA93CA94DA95EA986
:105B60006D857E858F8598890E949EAE6D877E8724
:105B70008F87988BC1010E945842FE01E659FF4F62
:105B80006F012C96ECACFDAC0EAD1FAD2C979E01B9
:105B9000235F3F4FAE01475F5F4FBE016B5F7F4F9B
:105BA000C1010E944E9B2F8D38A12F5F3F4F38A31C
:105BB0002F8FDECE2D8D3E8D245F3F4F4D8D5E8D20
:105BC000485F5F4F6D8D7E8D6C5F7F4FDE01A65904
:105BD000BF4F6D012C96ECACFDAC0EAD1FAD2C97FC
:105BE0008D8D9E8D0E944E9BC15BDF4F0FB6F8944A
:105BF000DEBF0FBECDBFDF91CF911F910F91FF9000
:105C0000EF90DF90CF90BF90AF909F908F907F905C
:105C10006F905F904F903F902F900895FC011482F9
:105C20001782138212828AEB95E091838083089514
:105C30002AEB35E0FC01318320832781222319F0F0
:105C400004960C94CD130895CF92DF92EF92FF92B9
:105C50000F931F93CF93DF93EC01875B9F4FDEDFA2
:105C6000CE0186599F4FDADF7E0129E8E20EF11C52
:105C700087016E0131E4C31A3EEFD30AC801CEDFBB
:105C8000015E1F4F0C151D05C9F7FE01EF53FE4FB6
:105C900089E1818314823596178ACE018C519E4FFB
:105CA000BDDFFE01EB56FD4F10821182128213827E
:105CB000389610821182128213821A821B821882F5
:105CC00019826E0187E6C81A8DEFD80AF601108294
:105CD000118212821382F80111821082FE01ED5F9F
:105CE000FD4F108286E391E0F7019C011192215053
:105CF0003040E1F7FE01EF55FD4F81E08083C95B45
:105D0000DF4F198218820E9408AA68577C4E8F4F75
:105D10009F4FF6016083718382839383DF91CF91DC
:105D20001F910F91FF90EF90DF90CF900895FC01AD
:105D300020E03EE2DB014C91403241F0283011F48A
:105D400030833196DB014C91408331962F5F6F5F3A
:105D50007F4F2B3079F7108208952F923F924F9208
:105D60005F926F927F928F929F92AF92BF92CF92EB
:105D7000DF92EF92FF920F931F93CF93DF93CDB7F4
:105D8000DEB7CA58D1090FB6F894DEBF0FBECDBF3B
:105D90008C016B017A014901CA57DF4F1882C6583E
:105DA000D04084E0E80EF11C180191E1290E311C6D
:105DB000F801EA5BFF4FC957DF4FF983E883C75803
:105DC000D0403801FEE56F1AFDEF7F0A58018CE5DF
:105DD000A81A8DEFB80A80E4482E512C4C0E5D1E97
:105DE00094E0490E511CA101BE016F5F7F4FC701B6
:105DF0000E94371218160CF03CC12C85322F3871D6
:105E0000303109F09EC0F3018081918101970297A2
:105E100008F497C0BE016F5F7F4FCE0187589F4F38
:105E200086DFA0961FAEA097F6018081811107C082
:105E300069E673E0CE01815A9F4F0E94EFB6B6012A
:105E4000CE01815A9F4F0E94EFB6BE0167587F4F27
:105E5000CE01815A9F4F0E94EFB669E673E0CE01F2
:105E6000815A9F4F0E94EFB6CE01805C9F4FD6DED5
:105E700021E0AE0147585F4FB701C2010E94C4152F
:105E8000811139C0F30180819181892BA1F5E0EB6B
:105E9000FEE08491882341F09091C00095FFFCCFF3
:105EA0008093C6003196F5CFEBE6F3E0819188232D
:105EB00039F09091C00095FFFCCF8093C600F6CFDB
:105EC0008091C00085FFFCCF8AE08093C600FE0170
:105ED000E758FF4F8191882339F09091C00095FFDA
:105EE000FCCF8093C600F6CF8091C00085FFFCCF29
:105EF0008AE08093C6008BE1FE01EC5BFF4FDE0180
:105F0000959601900D928A95E1F724968EAD9FADFE
:105F100024979CA38BA38AEB95E09AA389A320E006
:105F200030E0AE014F5D5F4FBE01615A7F4FC80147
:105F300014DFCE0181967CDECE01805C9F4F78DE3F
:105F400052CF8981882309F494C08E3209F44BCF53
:105F50008F3509F448CFF80181898E3209F443CF97
:105F60008F3509F440CF23FD3ECF81E0303109F079
:105F700080E0C957DF4FE881F981C758D04080835E
:105F8000811108C08985873409F02DCF8A858E3725
:105F900009F429CF98012C5F3F4FBE016F5F7F4FFF
:105FA000C901C757DF4F2883C958D040C657DF4FB4
:105FB0003883CA58D040BBDEF30180819181C75736
:105FC000DF4F2881C958D040C657DF4F3881CA58A3
:105FD000D0400097F1F4F6018191882339F0909137
:105FE000C00095FFFCCF8093C600F6CFF9018191E8
:105FF000882339F09091C00095FFFCCF8093C600B4
:10600000F6CF8091C00085FFFCCF8AE08093C60068
:10601000EACE8130910539F4F501808191810196B4
:1060200091838083E0CE029709F0DDCE8114910444
:1060300039F0B901C4010E94DCB6892B71F419C092
:10604000CA57DF4FF881C658D0402F2F30E0F501F6
:10605000808191812817390761F0CA57DF4FF88195
:10606000C658D040FF5FCA57DF4FF883C658D040AC
:10607000BACEC657DF4F0FB6F894DEBF0FBECDBF06
:10608000DF91CF911F910F91FF90EF90DF90CF9014
:10609000BF90AF909F908F907F906F905F904F9048
:1060A0003F902F9008950F931F93CF93DF93CDB719
:1060B000DEB76F970FB6F894DEBF0FBECDBF8C0171
:1060C000FC01EE55FD4F1182108240E050E0BA0114
:1060D000835B9F4F0E94EA12C801875B9F4F2BE1B1
:1060E000FC013496DE01159601900D922A95E1F798
:1060F000FC01828193819C838B838AEB95E09A8358
:10610000898320E030E0AE014F5F5F4F62E973E0CA
:10611000C80123DECE0101968BDD6F960FB6F89491
:10612000DEBF0FBECDBFDF91CF911F910F910895BC
:106130002BE1FB013496DC01149601900D922A9517
:10614000E1F7FB0122813381FC013383228308952F
:10615000EF92FF920F931F93CF93DF93EC011B827B
:10616000FC01E05BFF4F8081882329F0CE01835B37
:106170009F4F0E94CD137E018FE3E81A8EEFF80A3D
:1061800045E360E0C7010E94AD3B81111FC0E0EB19
:10619000FEE08491882341F09091C00095FFFCCFF0
:1061A0008093C6003196F5CFE8ECF6E08491882321
:1061B00041F09091C00095FFFCCF8093C6003196CE
:1061C000F5CF8091C00085FFFCCF77C08E010A53C8
:1061D0001E4F41E0B701C8010E949B1B811126C0E0
:1061E00040E0B701C8010E949B1B81111FC0E6EB74
:1061F000FEE08491882341F09091C00095FFFCCF90
:106200008093C6003196F5CFE5EBF6E084918823C4
:1062100041F09091C00095FFFCCF8093C60031966D
:10622000F5CF8091C00085FFFCCF47C0B801CE01FB
:10623000835B9F4F0E94DA1081111FC0E6EBFEE0E6
:106240008491882341F09091C00095FFFCCF80930A
:10625000C6003196F5CFE5EAF6E08491882341F057
:106260009091C00095FFFCCF8093C6003196F5CF8A
:106270008091C00085FFFCCF20C081E08B83E0EBE4
:10628000FEE08491882341F09091C00095FFFCCFFF
:106290008093C6003196F5CFEAE9F6E08491882331
:1062A00041F09091C00095FFFCCF8093C6003196DD
:1062B000F5CF8091C00085FFFCCF8AE08093C600B7
:1062C0008E01075B1F4FB801CE0186599F4F30DF0B
:1062D000C859DF4F19830883DF91CF911F910F9128
:1062E000FF90EF900895FC01128213820895FC0143
:1062F0002381222311F021E022830895FC012281D1
:10630000211112820895AF92BF92CF92DF92EF9245
:10631000FF920F931F93CF93DF931F92CDB7DEB7FA
:106320008C018FE2FB0181935F01D12C41E0780168
:10633000F1E4EF1AFEEFFF0A9FE1C92E2D2D30E0A8
:10634000F7018081918128173907D8F4C29EC001D6
:10635000C39E900D112483579F4FB501800F911F4D
:1063600049830E948110C50149815C010196F501B4
:106370002081222321F04D3810F44F5FF6CFD394C3
:10638000DDCF47FD11C0B501C80188519E4F0F9068
:10639000DF91CF911F910F91FF90EF90DF90CF9001
:1063A000BF90AF900C948110F50110820F90DF9197
:1063B000CF911F910F91FF90EF90DF90CF90BF9002
:1063C000AF9008953F924F925F926F927F928F921B
:1063D0009F92AF92BF92CF92DF92EF92FF920F9374
:1063E0001F93CF93DF93CDB7DEB7AC970FB6F8947A
:1063F000DEBF0FBECDBF7C015B01FC018381882322
:1064000009F408C1C70188519E4F0E94CD13F701BE
:106410001282CE0101966C0101DC270198E6490E3B
:10642000511CC701875B9F4FF20191838083F50167
:1064300080818F3209F084C06FE270E0C5010E9454
:10644000FAB68C010F5F1F4F2AE0322E011511059D
:1064500009F47CC06FE270E0C8010E94FAB64C01FA
:10646000009709F474C00817190708F070C03C01C0
:10647000601A710AA301B801CE0180960E9423B769
:10648000E0E2F0E0EC0FFD1FE60DF71D1082FE01CB
:10649000B0968191882339F09091C00095FFFCCF90
:1064A0008093C600F6CF8091C00085FFFCCF30926C
:1064B000C600F201608171816115710519F06C5F90
:1064C0007F4F02C060E070E021E0AE01405E5F4FB0
:1064D000CE0105960E94C41581112BC0EFE7F5E0AF
:1064E0008491882341F09091C00095FFFCCF809368
:1064F000C6003196F5CFFE01B0968191882339F020
:106500009091C00095FFFCCF8093C600F6CFEDE7D9
:10651000F5E08491882341F09091C00095FFFCCF75
:106520008093C6003196F5CF8091C00085FFFCCFE7
:106530006CC0F201D182C08284010F5F1F4F86CFF1
:10654000C70186599F4FF201918380838501F20133
:1065500080819181009711F0049602C080E090E064
:10656000B8010E949A16882339F1EFE6F5E084918C
:10657000882341F09091C00095FFFCCF8093C60026
:106580003196F5CFF8018191882339F09091C000C0
:1065900095FFFCCF8093C600F6CF8091C00085FFA9
:1065A000FCCF8AE08093C600F701E356FD4F1082CE
:1065B0001182128213822CC0E7E5F5E084918823D2
:1065C00041F09091C00095FFFCCF8093C6003196BA
:1065D000F5CFF8018191882339F09091C00095FFA3
:1065E000FCCF8093C600F6CFE5E5F5E084918823E3
:1065F00041F09091C00095FFFCCF8093C60031968A
:10660000F5CF8091C00085FFFCCF8AE08093C60063
:10661000C6010EDBAC960FB6F894DEBF0FBECDBF41
:10662000DF91CF911F910F91FF90EF90DF90CF906E
:10663000BF90AF909F908F907F906F905F904F90A2
:106640003F9008958F929F92AF92BF92CF92DF9228
:10665000EF92FF92CF93DF931F92CDB7DEB77C010D
:10666000FC018281882309F4AFC07196819188234F
:1066700039F09091C00095FFFCCF8093C600F6CF13
:10668000E3E5F5E08491882341F09091C00095FF07
:10669000FCCF8093C6003196F5CFE1E4F5E084911C
:1066A000882341F09091C00095FFFCCF8093C600F5
:1066B0003196F5CFF701E356FD4F4081518162815C
:1066C00073812AE030E08CE99DE00E945D8BEFE36E
:1066D000F5E08491882341F09091C00095FFFCCFB4
:1066E0008093C6003196F5CFF701EB56FD4F408100
:1066F0005181628173812AE030E08CE99DE00E9443
:106700005D8B8091C00085FFFCCF8AE08093C6003E
:106710000E9408AA30E6C32E3AEED32EE12CF12CCB
:10672000A70196010E9455B349015A016091520890
:10673000709153088091540890915508A7019601D3
:106740000E9455B3821A930AC4016CE370E00E9460
:106750002EB36983CE0101960E940779FC01219135
:10676000CF01222339F03091C00035FFFCCF2093B8
:10677000C600F4CF40E050E06AE38CE99DE00E945F
:10678000158BC4016CE370E00E942EB38983CE01A7
:1067900001960E940779FC012191CF01222339F053
:1067A0003091C00035FFFCCF2093C600F4CFEDE35D
:1067B000F5E084918823E1F09091C00095FFFCCF33
:1067C0008093C6003196F5CFE0E3F5E0849188230D
:1067D00041F09091C00095FFFCCF8093C6003196A8
:1067E000F5CF8091C00085FFFCCF8AE08093C60082
:1067F0000F90DF91CF91FF90EF90DF90CF90BF90FF
:10680000AF909F908F900895AF92BF92CF92DF92FA
:10681000EF92FF920F931F93CF93DF935C01EB01F5
:10682000FB0101900020E9F78F0101501109061BBF
:10683000170B6C01F8E1CF1AFEEFDF0AF6011082A8
:106840006EE470E0CE010E94FAB67C01009729F454
:10685000F8013197EC0FFD1F0DC060E270E00E945F
:10686000FAB6EC0121966AE270E0C7010E94FAB61E
:10687000FC0131978DE081838AE082831382BE011F
:10688000C5018C519E4F0E941A8CF601808188238D
:1068900009F1E6EBFEE08491882341F09091C0007D
:1068A00095FFFCCF8093C6003196F5CFEAE1F5E085
:1068B0008491882341F09091C00095FFFCCF809394
:1068C000C6003196F5CF8091C00085FFFCCF8AE0ED
:1068D0008093C600DF91CF911F910F91FF90EF90B1
:1068E000DF90CF90BF90AF9008952F923F924F923C
:1068F0005F926F927F928F929F92AF92BF92CF9250
:10690000DF92EF92FF920F931F93CF93DF93CDB758
:10691000DEB7CC55D1090FB6F894DEBF0FBECDBFA0
:106920004C018C010F551D4F662339F0F801108280
:10693000F401838181111DC015C0F8018081882375
:1069400009F4AFC0F401E756FD4FC080D180E2806A
:10695000F3800E9408AAC616D706E806F90608F4CE
:10696000A0C0E4CFC401F4DBF4018381882309F4DF
:1069700098C07401F7E4EF0EF11CF70181818F9349
:1069800080818F9381E195E09F938F938E01015CCD
:106990001F4F1F930F930E9432B70F900F900F90CD
:1069A0000F900F900F90B12CF80101900020E9F7A3
:1069B0003197E01BF10BBE1684F46801CB0CD11C9F
:1069C000B7FCDA94F6018081992787FD90950E94A3
:1069D0006FB6F6018083B394E7CFFDE48F0E911C70
:1069E00040E050E0BA01C4010E94EA12512CCE01ED
:1069F00001966C014AE0642E45E0742E5E0191E23E
:106A0000A90EB11C40E050E0B601C4010E9437124B
:106A10001816DCF5412CF60101900020E9F73197BA
:106A2000EC19FD094E1674F41601240C311C47FCB8
:106A30003A94F101808190E00E946FB6F101808369
:106A40004394E9CF8A858E37E9F245E050E0B801FA
:106A5000C6010E9415B7892BA9F61F930F937F9249
:106A60006F92BF92AF920E9432B7C5010E94AE3EB4
:106A700086E095E00E94213F0F900F900F900F90BD
:106A80000F900F9055245394BDCF511004C08FEF39
:106A90009FEFF70104C0F7018081918101969183F6
:106AA0008083C45ADF4F0FB6F894DEBF0FBECDBF50
:106AB000DF91CF911F910F91FF90EF90DF90CF90DA
:106AC000BF90AF909F908F907F906F905F904F900E
:106AD0003F902F9008950F931F93CF93DF93EC0176
:106AE0008C0108511E4FC8010E948313C8010E94E7
:106AF000CD1318821982DF91CF911F910F910895C4
:106B0000CF92DF92EF92FF920F931F93CF93DF9379
:106B1000CDB7DEB76F970FB6F894DEBF0FBECDBF0F
:106B20008C016A017C0188E6E80EF11CC8018659D7
:106B30009F4FF70191838083E65CFD4F22E030E0B8
:106B40003183208332967183608340E050E0BA0144
:106B500004960E94EA12F701808191812BE1FC01E9
:106B60003496DE01159601900D922A95E1F7FC010D
:106B7000828193819C838B838AEB95E09A838983BE
:106B80009601AE014F5F5F4F62E973E0C801E5D83F
:106B9000CE0101964DD86F960FB6F894DEBF0FBEAA
:106BA000CDBFDF91CF911F910F91FF90EF90DF90BC
:106BB000CF9008952F923F924F925F926F927F9263
:106BC0008F929F92AF92BF92CF92DF92EF92FF92FD
:106BD0000F931F93CF93DF93CDB7DEB7AC970FB66C
:106BE000F894DEBF0FBECDBF8C016B01342EDC01EB
:106BF00013968C91882309F4EEC2F801E551FE4FFB
:106C00008081882309F4F5C02111C1C07801BDEF4E
:106C1000EB1AFB0AF7018081882361F1E6EBFEE0C5
:106C20008491882341F09091C00095FFFCCF809320
:106C3000C6003196F5CFE7E5F6E08491882341F070
:106C40009091C00095FFFCCF8093C6003196F5CFA0
:106C50004AE050E061E070E08CE99DE00E94318BF9
:106C60008091C00085FFFCCF8AE08093C6000E941F
:106C70001046B1C2E0EBFEE08491882341F0909190
:106C8000C00095FFFCCF8093C6003196F5CFEEE3B0
:106C9000F6E08491882341F09091C00095FFFCCFED
:106CA0008093C6003196F5CFF6018191882339F0A3
:106CB0009091C00095FFFCCF8093C600F6CFE3E330
:106CC000F6E08491882341F09091C00095FFFCCFBD
:106CD0008093C6003196F5CFD7018C916DE8B62E22
:106CE000B801B89E600D711D1124685F7D4FC80109
:106CF0000ADBF7018081F801B89EE00DF11D112437
:106D0000E85FFD4F8191882339F09091C00095FF95
:106D1000FCCF8093C600F6CFEDE2F6E084918823A5
:106D200041F09091C00095FFFCCF8093C600319652
:106D3000F5CF5801F3E6AF1AFDEFBF0AD5014D912B
:106D40005D916D917C912AE030E08CE99DE00E949C
:106D50005D8B8091C00085FFFCCF8AE08093C600E8
:106D6000F7012081F80184E0289FE00DF11D112436
:106D7000EC5FFD4FD5014D915D916D917C9140830C
:106D80005183628373832F5FF70120832CC0E0EB74
:106D9000FEE08491882341F09091C00095FFFCCFE4
:106DA0008093C6003196F5CFECE1F6E0849188231C
:106DB00041F09091C00095FFFCCF8093C6003196C2
:106DC000F5CFF6018191882339F09091C00095FFAD
:106DD000FCCF8093C600F6CF8091C00085FFFCCF2A
:106DE0008AE08093C600C80188519E4F0E94CD134F
:106DF00030C0F801ED5FFD4F1082E0EBFEE08491C2
:106E0000882341F09091C00095FFFCCF8093C6008D
:106E10003196F5CFEBE0F6E08491882341F0909134
:106E2000C00095FFFCCF8093C6003196F5CFF601E8
:106E30008191882339F09091C00095FFFCCF809319
:106E4000C600F6CF8091C00085FFFCCF8AE080931A
:106E5000C600D80112961C92FE0131965F01CF0147
:106E60000E940E2E2801F8E64F0E511CC801875BC8
:106E70009F4FD2018D939C93F60180818F3209F050
:106E800084C06FE270E0C6010E94FAB601967C01F0
:106E90005AE0252EE114F10409F47DC06FE270E0A0
:106EA000C7010E94FAB64C01009709F475C0E816B4
:106EB000F90608F071C03C016E187F08A301B70104
:106EC000CE0180960E9423B7E0E2F0E0EC0FFD1FB8
:106ED000E60DF71D1082FE01B0968191882339F0EE
:106EE0009091C00095FFFCCF8093C600F6CF8091B3
:106EF000C00085FFFCCF2092C600D2016D917C912D
:106F00006115710519F06C5F7F4F02C060E070E0A1
:106F100021E0AE01405E5F4FCE0105960E94C41590
:106F200081112BC0E7EFF5E08491882341F0909127
:106F3000C00095FFFCCF8093C6003196F5CFFE01CF
:106F4000B0968191882339F09091C00095FFFCCFD5
:106F50008093C600F6CFE5EFF5E08491882341F0F9
:106F60009091C00095FFFCCF8093C6003196F5CF7D
:106F70008091C00085FFFCCF02C1F201B182A082E6
:106F80007401FFEFEF1AFF0A85CFC80186599F4FA2
:106F9000D2018D939C937601F801E851FE4F4F0189
:106FA000332009F4B1C0D2016D917C916115710556
:106FB00019F06C5F7F4F02C060E070E021E0A70134
:106FC000C4010E94C415882309F474C0F4018189A6
:106FD0009289A389B489F801EB56FD4F8083918390
:106FE000A283B383E7EEF5E08491D801AB56BD4FA1
:106FF000882349F09091C00095FFFCCF8093C60094
:1070000031968491F5CFF7018191882339F09091E1
:10701000C00095FFFCCF8093C600F6CFEFEDF5E002
:107020008491882341F09091C00095FFFCCF80931C
:10703000C6003196F5CF4D915D916D917C912AE01E
:1070400030E08CE99DE00E945D8B8091C00085FF5F
:10705000FCCF8AE08093C600F801E356FD4F108212
:10706000118212821382E1EDF5E08491882341F0D0
:107070009091C00095FFFCCF8093C6003196F5CF6C
:107080008091C00085FFFCCF8AE08093C600A701F5
:1070900060E070E0C80134DDD80151968C918823FE
:1070A00019F0C801419601C0C7010E940F738EE715
:1070B00093E08CC0EDEBF5E08491882341F0909152
:1070C000C00095FFFCCF8093C6003196F5CFF70145
:1070D0008191882339F09091C00095FFFCCF809377
:1070E000C600F6CFEBEBF5E08491882341F0909158
:1070F000C00095FFFCCF8093C6003196F5CF8091FC
:10710000C00085FFFCCF3BC0F20160817181611539
:10711000710519F06C5F7F4F02C060E070E026E5FA
:10712000A701C4010E94C41581112DC0E7EAF5E052
:107130008491882341F09091C00095FFFCCF80930B
:10714000C6003196F5CFF7018191882339F09091EF
:10715000C00095FFFCCF8093C600F6CFE5EAF5E0CE
:107160008491882341F09091C00095FFFCCF8093DB
:10717000C6003196F5CF8091C00085FFFCCF8AE034
:107180008093C60025C081E0D8018C93E3E9F5E047
:107190008491882341F09091C00095FFFCCF8093AB
:1071A000C6003196F5CFF6018191882339F0909190
:1071B000C00095FFFCCF8093C600F6CF8091C00041
:1071C00085FFFCCF8AE08093C600C7010E940F7341
:1071D000C5010E94182EAC960FB6F894DEBF0FBE04
:1071E000CDBFDF91CF911F910F91FF90EF90DF9076
:1071F000CF90BF90AF909F908F907F906F905F9057
:107200004F903F902F90089521E0FC01218340E0B2
:10721000D1CCCF92DF92EF92FF920F931F93CF9337
:10722000DF93CDB7DEB76F970FB6F894DEBF0FBE12
:10723000CDBF8C016C0128E6C20ED11C86599F4F30
:10724000F60191838083E65CFD4F21E030E03183DD
:1072500020837801FCE5EF1AFDEFFF0AF7011182A8
:10726000108240E050E0BA0104960E94EA12F60152
:10727000808191812BE1FC013496DE01159601900D
:107280000D922A95E1F7FC01828193819C838B8387
:107290008AEB95E09A83898320E030E0AE014F5F6E
:1072A0005F4F62E973E0C8010E94AD2ECE010196E6
:1072B0000E94182EF701808191816F960FB6F89485
:1072C000DEBF0FBECDBFDF91CF911F910F91FF9019
:1072D000EF90DF90CF900895AF92BF92CF92DF9260
:1072E000EF92FF920F931F93CF93DF93CDB7DEB74B
:1072F0006F970FB6F894DEBF0FBECDBF8C017B0138
:10730000CE0101960E940E2EF801EF58FF4F8081AA
:107310006801811104C029E4C20ED11C03C08AE6B1
:10732000C80ED11C21E0A701B6016C5F7F4FCE01D2
:1073300005960E94C41581112DC0E0EBFEE08491FA
:10734000882341F09091C00095FFFCCF8093C60048
:107350003196F5CFE0EFF4E08491882341F09091ED
:10736000C00095FFFCCF8093C6003196F5CFF701A2
:107370008191882339F09091C00095FFFCCF8093D4
:10738000C600F6CF8091C00085FFFCCF8AE08093D5
:10739000C60036C0F801E154FE4F808191818A30E9
:1073A000910530F59C012F5F3F4F318320832FE102
:1073B000289F7001299FF00C112429E8E20EF11C8E
:1073C000E00EF11E5C01B701C7014F960E94983094
:1073D00081E0A81AB1082FE1E21AF1088FEFA81690
:1073E000B80689F7B601C80187579F4F0E949830A9
:1073F000BE016F5F7F4FC80186599F4F0E94983032
:10740000CE0101960E94182E6F960FB6F894DEBF3B
:107410000FBECDBFDF91CF911F910F91FF90EF90E5
:10742000DF90CF90BF90AF900895EF92FF920F93AF
:107430001F93CF93DF93EC01C154DE4F2881398134
:1074400021153105F9F021503109398328838C0148
:1074500007571F4FB80186599F4F0E949830C801A7
:1074600000E010E07C012FE1E20EF11C288139815F
:107470000217130738F40F5F1F4FB7010E949830AF
:10748000C701F0CFDF91CF911F910F91FF90EF9047
:107490000895EF92FF920F931F93CF93DF93EC0128
:1074A0000E9414948E010D5F1D4FF80180819E0192
:1074B00028513E4F79018823A1F1C9010E94CD13C3
:1074C000F801808181508083BE01FDE88F9F600DAF
:1074D000711D1124685F7D4F21E041E0CE016ADB20
:1074E000F8018081FE0124E0829FE00DF11D11244E
:1074F000EC5FFD4F4081518162817381FE01E35653
:10750000FD4F4083518362837383C7010E94EA1257
:10751000CE01DF91CF911F910F91FF90EF900C94CE
:1075200077310E948A94C7010E94CD131A8284EE9B
:1075300094E0DF91CF911F910F91FF90EF9081C464
:107540008FEF8EBD0DB407FEFDCF8EB508958EBDB5
:107550000DB407FEFDCF089561E0FC0180810C941D
:1075600061A9FC012281322F306A36953CBD20FD95
:1075700006C031E0263009F430E0232F01C020E0BE
:107580002DBD60E0FC0180810C9461A9CF92DF9257
:10759000EF92FF920F931F93CF93DF93EC018B0138
:1075A0007A010E9408AA6B01CBDF8B838F3F49F4DD
:1075B0000E9408AA6C197D096D327140A8F381E11F
:1075C00044C08E3F11F08FE040C0E114F104D9F0C7
:1075D000C70101972FEF2EBDF8014FEF9F01201B30
:1075E000310B2817390738F40DB407FEFDCF2EB53F
:1075F00021934EBDF3CF0DB407FEFDCF2EB5F8019C
:10760000E80FF91F2083D801E00EF11EC12CD12C08
:10761000AE15BF0579F08D91ED2DFF27E827EE0F10
:10762000FF1FEB52F94F85919491DC2CCC24C82696
:10763000D926EECF85DF082F10E0102F002780DF3E
:10764000082BC016D10631F080E28983CE0184DF99
:1076500080E003C0CE0180DF81E0DF91CF911F91F8
:107660000F91FF90EF90DF90CF9008950F931F93AD
:10767000CF93DF93EB010E9408AA8B0161DF8F3F5C
:1076800049F00E9408AA601B710B6C177D07B0F3CC
:1076900080E001C081E0DF91CF911F910F910895AB
:1076A000CF92DF92FF920F931F93CF93DF9300D07F
:1076B0001F92CDB7DEB76C01F62E29833A834B8338
:1076C0005C834FDF6CE271E0C601D0DF8F2D8064F8
:1076D0003EDF08E110E05C814B813A812981DA01CB
:1076E000C901002E04C0B695A795979587950A9471
:1076F000D2F729833A834B835C8329DF0850110931
:1077000029813A814B815C81083F8FEF180739F757
:10771000FF2029F0E8E0FE1621F08FEF03C085E995
:1077200001C087E814DFFCE0FF1201C009DF10E0B0
:1077300007DFF601838387FF04C01F3F11F01F5F3F
:10774000F7CF0F900F900F900F90DF91CF911F9177
:107750000F91FF90DF90CF900895BF92CF92DF926C
:10776000EF92FF920F931F93CF93DF93EC01B62E0E
:107770001C82198248830E9408AA8B0161E08881DB
:107780000E9428A9CE01E8DE60E082E30E9428A9D9
:1077900061E083E30E9428A961E084E30E9428A9B4
:1077A00061E085E30E9428A961E085E30E9461A968
:1077B00085E08A8382E58CBD1DBC6AE0F62E8FEFE2
:1077C000C6DEFA94E1F720E030E0A90160E0CE01E6
:1077D00067DFF82E8B8381E0F81649F00E9408AA33
:1077E000601B710B613D774070F381E046C02AEA6F
:1077F00031E040E050E068E0CE0152DF82FF02C09D
:10780000FC820CC054E0F52E9BDE8B83FA94E1F7EA
:107810008A3A11F082E031C082E08C838C81823020
:1078200031F4C12CD12CE12C40E4F42E03C0C12C46
:10783000D12C760120E030E0A90167E3CE0130DFF2
:10784000A701960169E2CE012BDF8B83882349F0E3
:107850000E9408AA601B710B613D774058F38AE0D3
:107860000CC08C818230B1F420E030E0A9016AE3E1
:10787000CE0116DF882329F088E08983CE016CDEF3
:1078800014C05EDE807C803C11F483E08C8358DE83
:1078900057DE56DECE0160DE86E08B1518F488E1F7
:1078A000898303C0BA8281E001C080E0DF91CF917B
:1078B0001F910F91FF90EF90DF90CF90BF900895B0
:1078C000AF92BF92CF92DF92EF92FF920F931F93EE
:1078D000CF93DF93EC016A017B0189018C818330B6
:1078E00039F0F9E0CC0CDD1CEE1CFF1CFA95D1F749
:1078F00073E0B72EE4E0AE2EBA94A701960161E1E1
:10790000CE01CEDE882311F0A98207C040E052E00C
:10791000B801CE013BDE81110EC0CE01BB2049F083
:107920001BDE20E030E0A9016CE0CE01B9DE198257
:10793000E3CF12DE80E0DF91CF911F910F91FF9096
:10794000EF90DF90CF90BF90AF900895CF93DF93EB
:10795000EC016EBD20E030E00DB407FEFDCFFA0172
:10796000E20FF31F80818EBD0DB407FEFDCF818134
:107970008EBD2E5F3F4F211582E0380769F70DB4A9
:1079800007FEFDCF8FEFE3DD8FEFE1DDD9DD8B83E8
:107990008F71853031F083E18983CE01DDDD80E0B8
:1079A00001C081E0DF91CF9108950F931F93CF9392
:1079B000DF93EC0189018C81833039F0B9E0440F09
:1079C000551F661F771FBA95D1F79A01AB0168E181
:1079D000CE0166DE882311F086E01EC0A8016EEF9E
:1079E000CE01B4DF8823C9F068E572E0CE013EDE47
:1079F000182F811102C087E10FC020E030E0A901FB
:107A00006DE0CE014DDE811106C09ADD811103C00B
:107A1000CE01A2DD05C086E18983CE019DDD10E0A7
:107A2000812FDF91CF911F910F910895FC016591F6
:107A300075918591949108952F923F924F925F9204
:107A40006F927F928F929F92AF92BF92CF92DF926E
:107A5000EF92FF920F931F93CF93DF9300D000D04C
:107A6000CDB7DEB71C01FC01EF58F14F14919C011A
:107A7000220F331F220F331F3E832D832C5B354F84
:107A80004901F901108211821282138220E53AE045
:107A90004CE45AE068E47AE084E49AE00E9415A598
:107AA0008D819E818058914FC1DF6B017C01612FD8
:107AB000772767FD7095872F972F0E9419B02B01AC
:107AC0003C012D813E81215F354F590120E030E09E
:107AD00040EC5FE3C701B6010E944CB2A3019201E2
:107AE0000E944CB2F50160837183828393832D8160
:107AF0003E81215A3D4F3C832B83F9016081718186
:107B000082819381609321027093220280932302E9
:107B10009093240220E030E040E752E40E947EAFE0
:107B200020E3C22E2AE0D22E7B018C012BE13AE029
:107B300047E15AE063E17AE08FE09AE00E944E9BD1
:107B40000E941494F401108211821282138220E5A3
:107B50003AE04CE45AE068E47AE084E49AE00E9477
:107B600015A52D813E812C58314F3A832983C901B7
:107B70005DDF9058A30192010E944CB2F501608331
:107B800071838283938320E030E040E752E4609188
:107B900021027091220280912302909124020E947E
:107BA0007EAF7B018C012BE13AE047E15AE063E1D3
:107BB0007AE08FE09AE00E944E9B0E9414948981A3
:107BC0009A8134DF9B01AC010E949EAEA301920119
:107BD0000E944CB2F501608371838283938320E01D
:107BE00030E040E05FE3EB81FC8160817181828164
:107BF00093810E944CB26093210270932202809381
:107C000023029093240220E030E040E752E40E94F7
:107C10007EAF7B018C012BE13AE047E15AE063E162
:107C20007AE08FE09AE00E944E9B0E9414948D812E
:107C30009E818457914FFADE0D811E81085C154F9D
:107C4000F80120813181428153810E949EAEF4016E
:107C500060837183828393838D819E818C55914F44
:107C6000E5DE2D813E812D5B3D4F7901F8012081BC
:107C70003181428153810E949EAEF70160837183FE
:107C8000828393838D819E818856914FCFDE2D8193
:107C90003E81295C3D4F7901F8012081318142818B
:107CA00053810E949EAEF701608371838283938328
:107CB000F40180819181A281B381F5018083918358
:107CC000A283B38310922102109222021092230207
:107CD000109224020E94C18CF101EB5CF54F81E00F
:107CE000808326960FB6F894DEBF0FBECDBFDF911E
:107CF000CF911F910F91FF90EF90DF90CF90BF90A9
:107D0000AF909F908F907F906F905F904F903F903B
:107D10002F900895FC012491222341F03091C0005E
:107D200035FFFCCF2093C6000196F4CF22E030E06F
:107D30008CE99DE00C94078CFC012491222341F0F6
:107D40003091C00035FFFCCF2093C6000196F4CFE0
:107D50002AE030E08CE99DE00C945D8B2091640872
:107D600030916508243031050CF06AC040916608F6
:107D70005091670860E6649F9001659F300D112463
:107D8000BC01C9018259974F0E940EB7E0EBFEE09B
:107D90008491882341F09091C00095FFFCCF80939F
:107DA000C6003196F5CFE6E6FEE08491882341F0E7
:107DB0009091C00095FFFCCF8093C6003196F5CF1F
:107DC000809166089091670820E6289FF001299F1E
:107DD000F00D1124E259F74F8191882339F09091E9
:107DE000C00095FFFCCF8093C600F6CFE4E6FEE02E
:107DF0008491882341F09091C00095FFFCCF80933F
:107E0000C6003196F5CF8091C00085FFFCCF8AE097
:107E10008093C6008091660890916708019664E09F
:107E200070E00E9442B39093670880936608809147
:107E300064089091650801969093650880936408A2
:107E400008952091640830916508243031050CF0C4
:107E50006AC0409166085091670860E6649F90018F
:107E6000659F300D1124BC01C9018259974F0E94B2
:107E700077B6E0EBFEE08491882341F09091C0005A
:107E800095FFFCCF8093C6003196F5CFE9E5FEE083
:107E90008491882341F09091C00095FFFCCF80939E
:107EA000C6003196F5CF809166089091670820E66C
:107EB000289FF001299FF00D1124E259F74F81917D
:107EC000882339F09091C00095FFFCCF8093C600C5
:107ED000F6CFE7E5FEE08491882341F09091C00061
:107EE00095FFFCCF8093C6003196F5CF8091C000FE
:107EF00085FFFCCF8AE08093C60080916608909150
:107F00006708019664E070E00E9442B390936708AE
:107F1000809366088091640890916508019690931B
:107F200065088093640808959B9AA3980895FCDFE0
:107F300040E052EC61E070E08CE99DE00E94158A1F
:107F4000E1E5FEE08491882341F09091C00095FF27
:107F5000FCCF8093C6003196F5CF8091C00085FF9D
:107F6000FCCF8AE08093C60080EB9EE0FC01249168
:107F7000222341F03091C00035FFFCCF2093C60092
:107F80003196F5CF24B720FF14C0E9E4FEE0349128
:107F9000332341F04091C00045FFFCCF3093C60031
:107FA0003196F5CF3091C00035FFFCCF3AE03093E9
:107FB000C60021FF14C0E9E3FEE03491332341F011
:107FC0004091C00045FFFCCF3093C6003196F5CFFD
:107FD0003091C00035FFFCCF3AE03093C60022FF5D
:107FE00014C0E8E2FEE03491332341F04091C00038
:107FF00045FFFCCF3093C6003196F5CF3091C000DD
:1080000035FFFCCF3AE03093C60023FF14C0E8E10F
:10801000FEE03491332341F04091C00045FFFCCF96
:108020003093C6003196F5CF3091C00035FFFCCFBC
:108030003AE03093C60025FF14C0E8E0FEE024914A
:10804000222341F03091C00035FFFCCF2093C600C1
:108050003196F5CF2091C00025FFFCCF2AE0209378
:10806000C60014BEE1E0FEE02491222341F03091ED
:10807000C00035FFFCCF2093C6003196F5CFEBEF63
:10808000FDE02491222341F03091C00035FFFCCF68
:108090002093C6003196F5CF2091C00025FFFCCF7C
:1080A0002AE02093C600FC012491E0EBFEE02223AD
:1080B00049F03091C00035FFFCCF2093C6003196C7
:1080C0002491F5CFEBEEFDE02491222341F0309195
:1080D000C00035FFFCCF2093C6003196F5CFE6ED0A
:1080E000FDE02491222341F03091C00035FFFCCF08
:1080F0002093C6003196F5CFEAECFDE024912223CF
:1081000041F03091C00035FFFCCF2093C60031967E
:10811000F5CFE3EBFDE02491222341F03091C00044
:1081200035FFFCCF2093C6003196F5CF2091C000DB
:1081300025FFFCCF2AE02093C600E8EAFDE0249169
:10814000222341F03091C00035FFFCCF2093C600C0
:108150003196F5CFECE9FDE02491222341F03091F6
:10816000C00035FFFCCF2093C6003196F5CF20919B
:10817000C00025FFFCCF2AE02093C600FC018491BB
:10818000E0EBFEE0882349F09091C00095FFFCCF22
:108190008093C60031968491F5CFEDE8FDE084919F
:1081A000882341F09091C00095FFFCCF8093C600DA
:1081B0003196F5CF0E942F974AE050E0BC018CE940
:1081C0009DE00E94318BE6E7FDE08491882341F039
:1081D0009091C00095FFFCCF8093C6003196F5CFFB
:1081E0004AE050E060ED74E08CE99DE00E94318B44
:1081F0008091C00085FFFCCF8AE08093C60010927A
:108200006A0810926B0810926C0810926D080E9418
:1082100038880E940A840E94E3200E94FE9A0E94ED
:108220001D960E943B77FFEF23ED80E3F150204045
:108230008040E1F700C00000089580915E089091B1
:108240005F0860E070E001960C94CEB380915E0808
:1082500090915F084AE050E060E070E001960C9475
:1082600036B5682F772767FD7095209168083091A3
:10827000690840E6429FC001439F900D1124825936
:10828000974F0E94FAB690935F0880935E0821E0B2
:10829000892B09F420E0822F08950E9408AA609398
:1082A0005A0870935B0880935C0890935D0808956A
:1082B0000E9408AA60935A0870935B0880935C0838
:1082C00090935D08E0916808F0916908E659F74FCE
:1082D0008081811114C0EDE7F9E08491882341F099
:1082E0009091C00095FFFCCF8093C6003196F5CFEA
:1082F0008091C00085FFFCCF8AE08093C60008957E
:108300008CE99DE00E94678AE0E8F9E08491882387
:1083100041F09091C00095FFFCCF8093C60031964C
:10832000F5CF4091F3095091F4096091F5097091EE
:10833000F6094F5F5F4F6F4F7F4F2AE030E08CE9C7
:108340009DE00E94068B8091C00085FFFCCF8AE0F3
:108350008093C600ADCF8F929F92AF92BF92CF9283
:10836000DF92EF92FF920F931F93CF93DF9337EC3F
:10837000E32E34E0F32E04E41AE0CFE0DAE049E53E
:10838000C42E4AE0D42EF70181917F016ADF882351
:1083900011F153DF4B015C01F6018081811103C0B3
:1083A0006091EE0901C061E070E080E090E00E9421
:1083B00019B0F80120813181428153810E944CB271
:1083C0009B01AC01C501B4010E949EAE6883798314
:1083D0008A839B8309C0F80180819181A281B38146
:1083E00088839983AA83BB830C5F1F4F2496FFEF7A
:1083F000CF1ADF0A8BECE81684E0F80621F686E453
:1084000030DF8823D1F019DF6B017C016093FF0915
:108410007093000A8093010A9093020A20E030E0F2
:10842000A9010E947AB1181644F4C0922102D09298
:108430002202E0922302F0922402DF91CF911F9159
:108440000F91FF90EF90DF90CF90BF90AF909F90F3
:108450008F90089580DF89E404DF882351F0EDDEFA
:108460006093030A7093040A8093050A9093060AA6
:1084700008C01092030A1092040A1092050A109282
:10848000060A8AE4EEDE882351F0D7DE6093070AFD
:108490007093080A8093090A90930A0A089510922B
:1084A000070A1092080A1092090A10920A0A0895FF
:1084B000CF92DF92EF92FF92CF93DF93EC01C090C7
:1084C0004302D0904402E0904502F0904602A7019A
:1084D0009601688179818A819B810E9477AF87FFAD
:1084E00004C0C882D982EA82FB82C0904702D09041
:1084F0004802E0904902F0904A02A70196016C817F
:108500007D818E819F810E9477AF87FF04C0CC82DE
:10851000DD82EE82FF8220E030E0A90160914B0213
:1085200070914C0280914D0290914E020E949EAE3D
:108530006B017C019B01AC01688579858A859B85EF
:108540000E9477AF87FF04C0C886D986EA86FB867B
:10855000C0903702D0903802E0903902F0903A0291
:10856000A7019601688179818A819B810E947AB1F5
:10857000181624F4C882D982EA82FB82C0903B029A
:10858000D0903C02E0903D02F0903E02A70196019F
:108590006C817D818E819F810E947AB1181624F4AE
:1085A000CC82DD82EE82FF82C0903F02D0904002FA
:1085B000E0904102F0904202A7019601688579851A
:1085C0008A859B850E947AB1181624F4C886D986BC
:1085D000EA86FB86DF91CF91FF90EF90DF90CF90FE
:1085E0000895CF92DF92EF92FF920F931F938FE047
:1085F0009AE05EDF0E9408AA60935A0870935B08B5
:1086000080935C0890935D0820910F0A3091100AC6
:108610004091110A5091120A6091440A7091450AE2
:108620008091460A9091470A0E9477AF811179C0E4
:108630002091130A3091140A4091150A5091160A9C
:108640006091480A7091490A80914A0A90914B0AB8
:108650000E9477AF811165C020E030E040E752E42E
:108660006091210270912202809123029091240254
:108670000E947EAF50E3C52E5AE0D52E7B018C01BF
:108680002BE13AE047E15AE063E17AE08FE09AE0DB
:108690000E944E9B80910F0A9091100AA091110A9E
:1086A000B091120A8093440A9093450AA093460A17
:1086B000B093470A8091130A9091140AA091150A69
:1086C000B091160A8093480A9093490AA0934A0AE7
:1086D000B0934B0A8091170A9091180AA091190A39
:1086E000B0911A0A80934C0A90934D0AA0934E0AB7
:1086F000B0934F0A80911B0A90911C0AA0911D0A09
:10870000B0911E0A8093500A9093510AA093520A86
:10871000B093530A1F910F91FF90EF90DF90CF908D
:10872000089560915D0270915E02882777FD8095C3
:10873000982F0E9419B0209121023091220240917D
:108740002302509124020E944CB220E030E040E726
:1087500052E40E947EAF20E030E048EC52E488CF43
:10876000CF92DF92EF92FF92CF93C62FE091300A23
:10877000F0E0882309F4C2C0DF01A45DB54F8C91FD
:10878000811196C18091440A9091450AA091460AB0
:10879000B091470A80930F0A9093100AA093110A90
:1087A000B093120A8091480A9091490AA0914A0A0E
:1087B000B0914B0A8093130A9093140AA093150A60
:1087C000B093160A80914C0A90914D0AA0914E0ADE
:1087D000B0914F0A8093170A9093180AA093190A30
:1087E000B0931A0AC090500AD090510AE090520AF1
:1087F000F090530AC0921B0AD0921C0AE0921D0A04
:10880000F0921E0AEE0FFF1FEE0FFF1FE15BFD4F00
:108810002081318142815381CC2349F060912F0224
:1088200070913002809131029091320208C06091C3
:1088300033027091340280913502909136020E9489
:108840007EAF9B01AC01C701B6010E949EAE609352
:10885000500A7093510A8093520A9093530A80E50C
:108860009AE00E94BAA5C0902102D0902202E09026
:108870002302F090240220E030E040E752E46091CF
:108880002B0270912C0280912D0290912E020E9459
:108890004CB2609321027093220280932302909342
:1088A0002402E091300AF0E0E45DF54F81E080833E
:1088B00098DE2091280A3091290A40912A0A509185
:1088C0002B0A60914C0A70914D0A80914E0A90914A
:1088D0004F0A0E949DAE60934C0A70934D0A80939C
:1088E0004E0A90934F0A20E53AE04CE45AE068E4DF
:1088F0007AE084E49AE00E9415A5D1C0E45DF54FCA
:108900008081882309F4D4C08091440A9091450A5B
:10891000A091460AB091470A80930F0A9093100ADB
:10892000A093110AB093120A8091480A9091490AC3
:10893000A0914A0AB0914B0A8093130A9093140AAB
:10894000A093150AB093160A60914C0A70914D0AD3
:1089500080914E0A90914F0A6093170A7093180AFB
:108960008093190A90931A0AC090500AD090510A25
:10897000E090520AF090530AC0921B0AD0921C0A4F
:10898000E0921D0AF0921E0A2091280A3091290ACD
:1089900040912A0A50912B0A0E949EAE60934C0A85
:1089A00070934D0A80934E0A90934F0A20E53AE067
:1089B0004CE45AE068E47AE084E49AE00E9415A569
:1089C000F090300ACC2389F02091200A3091210ABE
:1089D0004091220A5091230A60912F027091300237
:1089E000809131029091320210C02091240A30917E
:1089F000250A4091260A5091270A6091330270910E
:108A0000340280913502909136020E949EAE24E09D
:108A1000F29EF0011124E15BFD4F20813181428102
:108A200053810E947EAF9B01AC016091500A70910E
:108A3000510A8091520A9091530A0E949DAE609310
:108A4000500A7093510A8093520A9093530A80E51A
:108A50009AE00E94BAA5C0902102D0902202E09034
:108A60002302F090240220E030E040E752E46091DD
:108A70002702709128028091290290912A020E9477
:108A80004CB2609321027093220280932302909350
:108A90002402E091300AF0E0E45DF54F1082A1DDA0
:108AA000C0922102D0922202E0922302F09224028C
:108AB000CF91FF90EF90DF90CF900895AF92BF924B
:108AC000CF92DF92EF92FF920F931F93CF93DF939A
:108AD000D82F2091070A3091080A4091090A509135
:108AE0000A0A6091030A7091040A8091050A909124
:108AF000060A0E9487B1C62F172F082FF92E609102
:108B00005D0270915E02882777FD8095982F0E9404
:108B100019B02091210230912202409123025091FC
:108B200024020E944CB220E030E040E752E40E9470
:108B30007EAF20E030E048EC52E40E947EAF20910E
:108B4000300A2F93DF93FF920F931F93CF935B0114
:108B50006C0172E0E72E01E020E043E05AE06FE0B4
:108B60007AE084E49AE00E949C2A80910F0A909116
:108B7000100AA091110AB091120A8093440A9093AE
:108B8000450AA093460AB093470A8091130A909130
:108B9000140AA091150AB091160A8093480A90937E
:108BA000490AA0934A0AB0934B0A8091170A909100
:108BB000180AA091190AB0911A0A80934C0A90934E
:108BC0004D0AA0934E0AB0934F0A80911B0A9091D0
:108BD0001C0AA0911D0AB0911E0A8093500A90931E
:108BE000510AA093520AB093530A0E9408AA6093B4
:108BF0005A0870935B0880935C0890935D080F900F
:108C00000F900F900F900F900F90DF91CF911F91C9
:108C10000F91FF90EF90DF90CF90BF90AF900895AD
:108C2000F8940E948621179A1092350A169A10928B
:108C3000360A159A1092370A149A60E087E40E9467
:108C400028A9E6EBFEE08491882341F09091C000D2
:108C500095FFFCCF8093C6003196F5CFEEE5F9E0A5
:108C60008491882341F09091C00095FFFCCF8093C0
:108C7000C6003196F5CF8091C00085FFFCCF8AE019
:108C80008093C60085E599E00E94D4767894C6E08A
:108C9000D0E02197209749F068EC70E080E090E008
:108CA0000E9437AA0E947677F4CFF894FFCF2F92D4
:108CB0003F924F925F926F927F928F929F92AF926C
:108CC000BF92CF92DF92EF92FF920F931F93CF93B9
:108CD000DF93CDB7DEB76E970FB6F894DEBF0FBE49
:108CE000CDBFB0E6BB2E14E0E12EF12C0CE3C02E7C
:108CF0000CE0D02E8AE0A82E9924939480911D0E2A
:108D000090911E0E20911F0E3091200E821B930B0E
:108D10008F779927892B09F41AC280916408909162
:108D2000650804970CF013C28CE99DE00E944B8A01
:108D30008093630820916108309162088A3061F065
:108D40008D3051F08A3321F490916008992321F0FD
:108D50002F3531050CF41DC12115310509F437C13A
:108D60008091660890916708B89E3001B99E700C9A
:108D70001124F301E20FF31FE259F74F1082209103
:108D80006008211101C110926008FC01E659F74FFB
:108D9000108283010259174F6EE470E0C8010E94EF
:108DA000FAB60097F1F190935F0880935E08801BFC
:108DB000910B860D971D4AE050E060E070E081590C
:108DC000974F0E9436B56093F7097093F809809326
:108DD000F9099093FA094090F3095090F4096090D2
:108DE000F5097090F6092FEF421A520A620A720AC8
:108DF000009166081091670864157505860597054A
:108E000009F4E8C0B09EC001B19E900D112468E540
:108E10007DE08259974F0E94A5B6892B09F0DAC0F0
:108E200069C16AE270E0C8010E94FAB6892B09F4B0
:108E300044C0E6EBFEE08491882341F09091C000AD
:108E400095FFFCCF8093C6003196F5CFE2EBFCE0B6
:108E50008491882341F09091C00095FFFCCF8093CE
:108E6000C6003196F5CF4091F3095091F409609115
:108E7000F5097091F6092AE030E08CE99DE00E9446
:108E8000068B8091C00085FFFCCF8AE08093C600EE
:108E90001092620810926108C0C28091F709909107
:108EA000F809A091F909B091FA098093F309909318
:108EB000F409A093F509B093F609809166089091A2
:108EC0006708B89E8001B99E100D1124C80182590F
:108ED000974F3C0167E470E00E94FAB6009781F179
:108EE00090935F0880935E0886199709800F911F01
:108EF00060E070E08159974F0E94CEB30E94E6AFC8
:108F000064307105E8F480914C088823C9F0F601BB
:108F10008491ECE3FCE0882349F09091C00095FF38
:108F2000FCCF8093C60031968491F5CF8091C0002C
:108F300085FFFCCFA092C60082E39CE00E94C7762A
:108F40000091660810916708B09EC001B19E900D17
:108F5000112463E973E08259974F0E9405B7892B6A
:108F600009F45EDEC8010196B7010E9442B39093F6
:108F7000670880936608809164089091650801965F
:108F800090936508809364081092620810926108BB
:108F9000B5CE8B3311F490926008909160089111D6
:108FA000ADCE4091660850916708B9016F5F7F4F61
:108FB0007093620860936108B49EF001B59EF00D55
:108FC0001124E20FF31FE259F74F808397CE1092DE
:108FD000600823C2B09E3001B19E700C1124C30101
:108FE0008259974F1C016AE270E00E94FAB600971E
:108FF00089F5E6EBFEE08491882341F09091C00072
:1090000095FFFCCF8093C6003196F5CFECEDFCE0E8
:109010008491882341F09091C00095FFFCCF80930C
:10902000C6003196F5CF4091F3095091F409609153
:10903000F5097091F6092AE030E08CE99DE00E9484
:10904000068B8091C00085FFFCCF8AE08093C6002C
:1090500057D91ECF20E010E0F301E20FF11DE259D5
:10906000F74F30813A3219F02F5F1327F5CF9093E5
:109070005F0880935E0882199309860D971D60E052
:1090800070E08159974F0E94CEB30E94E6AF212F26
:1090900030E02617370709F400CFE6EBFEE08491B5
:1090A000882341F09091C00095FFFCCF8093C600CB
:1090B0003196F5CFE6E0FDE08491882341F0909170
:1090C000C00095FFFCCF8093C6003196F5CF40914C
:1090D000F3095091F4096091F5097091F6092AE0BD
:1090E00030E08CE99DE00E94068B8091C00085FFF6
:1090F000FCCFABCFE6EBFEE08491882341F090916A
:10910000C00095FFFCCF8093C6003196F5CFE5E215
:10911000FDE08491882341F09091C00095FFFCCF41
:109120008093C6003196F5CF4091F3095091F40930
:109130006091F5097091F6092AE030E08CE99DE034
:109140000E94068B8091C00085FFFCCF7ECF80916E
:109150005F0A882309F461C18091610890916208D7
:10916000892B09F05AC18091640890916508892B78
:1091700011F410924A08F8EE2F2EF3E03F2E412C06
:10918000512CACE3CA2ED12CE12CF12C8E010F5FB7
:109190001F4FE0E66E2E772473944091FA0C5091A5
:1091A000FB0C6091FC0C7091FD0C8091F20C909185
:1091B000F30CA091F40CB091F50C481759076A070D
:1091C0007B0708F02AC18091640890916508049794
:1091D0000CF023C180914A0881111FC180914D0C70
:1091E00090914E0CA0914F0CB091500C8093FA0CC2
:1091F0009093FB0CA093FC0CB093FD0C85E49CE0D9
:109200000E942112482F809363088A30B9F04D30B4
:10921000A9F0433229F420916008222379F002C09A
:109220004A33C9F320916108309162082F35310526
:109230002CF48F3FFFEF9F0709F0D1C04091FA0C4B
:109240005091FB0C6091FC0C7091FD0C8091F20C24
:109250009091F30CA091F40CB091F50C48175907BC
:109260006A077B0708F481C0EFE1FCE08491882362
:1092700041F09091C00095FFFCCF8093C6003196DD
:10928000F5CF8091C00085FFFCCFFAE0F093C600D7
:109290000E9408AA60934E0870934F08809350086C
:1092A000909351088090520890905308A0905408D1
:1092B000B0905508681979098A099B09A2019101A2
:1092C0000E9455B349015A01CA01B901A70196018B
:1092D0000E9455B3CA01B901A70196010E9455B376
:1092E0007F936F93C501B40120E13EE040E050E080
:1092F0000E9455B33F932F93ABE0BCE0BF93AF9375
:109300001F930F930E9432B7E0EBFEE084910FB6FB
:10931000F894DEBF0FBECDBF882349F09091C00006
:1093200095FFFCCF8093C60031968491F5CFF8016C
:109330008191882339F09091C00095FFFCCF8093F4
:10934000C600F6CF8091C00085FFFCCF3AE0309395
:10935000C600C8010E940F738DE59AE00E94493A49
:1093600061E08DE59AE00E94753480916308833254
:1093700011F470924A082091610830916208211519
:10938000310509F424CE8091660890916708689EA3
:10939000F001699EF00D1124E20FF31FE259F74F1F
:1093A0001082FC01E659F74F7082209164083091D9
:1093B00065082F5F3F4F309365082093640801963E
:1093C00064E070E00E9442B390936708809366085F
:1093D000109260081092620810926108DECE4B3342
:1093E00011F470926008409160084111D2CE409112
:1093F000660850916708B9016F5F7F4F70936208EC
:1094000060936108649EF001659EF00D1124E20FE7
:10941000F31FE259F74F8083C0CE6E960FB6F894D3
:10942000DEBF0FBECDBFDF91CF911F910F91FF9097
:10943000EF90DF90CF90BF90AF909F908F907F90F4
:109440006F905F904F903F902F900895CF92DF9252
:10945000EF92FF920F931F93CF93C82F80916408D0
:109460009091650803970CF422DC0E9408AA0091F1
:109470005608109157082091580830915908C0900B
:109480005A08D0905B08E0905C08F0905D086C1979
:109490007D098E099F09061717072807390728F441
:1094A000012B022B032B09F0BBDB40911D025091D5
:1094B0001E0260911F0270912002452B462B472B04
:1094C00019F10E9408AA00915A0810915B08209196
:1094D0005C0830915D08601B710B820B930B00914F
:1094E0001D0210911E0220911F02309120020617CA
:1094F00017072807390740F490916D0E80916C0E84
:10950000981302C0CC2349F0CF911F910F91FF9087
:10951000EF90DF90CF900C94329B179A1092350AFF
:10952000169A1092360A159A1092370A149AECCFAE
:109530000E94862180914C08811138C081E080937F
:109540004C088091F3099091F409A091F509B0912C
:10955000F6098093EF099093F009A093F109B09375
:10956000F209E6EBFEE08491882341F09091C0007F
:1095700095FFFCCF8093C6003196F5CFEFEDF8E074
:109580008491882341F09091C00095FFFCCF809397
:10959000C6003196F5CF8091C00085FFFCCF8AE0F0
:1095A0008093C60085ED98E00C94C776089580916D
:1095B0004C080895CF93DF93EC018091300A80939B
:1095C0004D0884E50E943141811102C080E075C0E0
:1095D0000E941D410E94EBAF60934D086623B1F3DA
:1095E000E0EBFEE08491882341F09091C00095FF6C
:1095F000FCCF8093C6003196F5CFCD36D105B9F0BA
:1096000054F4C836D105B1F0C936D10509F045C0CA
:10961000EDEDF3E021C0CA3DD10531F0CD3DD105DE
:10962000E1F5E8E9F3E036C0EFEAF3E029C0E6EC63
:10963000F3E01CC0E4EFF3E08191882371F1909195
:10964000C00095FFFCCF8093C600F6CF9091C0007C
:1096500095FFFCCF8093C60081918111F7CF1DC08B
:109660009091C00095FFFCCF8093C600819181113D
:10967000F7CF13C09091C00095FFFCCF8093C60038
:1096800081918111F7CF09C09091C00095FFFCCF67
:109690008093C60081918111F7CF40E050E0609146
:1096A0004D088CE99DE00E94688B8091C00085FF89
:1096B000FCCF8AE08093C60081E0DF91CF910895CE
:1096C000CF92DF92EF92FF922091540A2223F1F081
:1096D00020E030E040E05FE30E944CB26B017C018F
:1096E00020E030E0A9010E9477AF882379F0A7013C
:1096F0009601C701B6010E944CB22BED3FE049E450
:1097000050E40E944CB29B01AC0104C020E030E068
:1097100040E85FE360E070E080E89FE30E947EAF96
:10972000FF90EF90DF90CF90089560915302709179
:1097300054028091550290915602C2DF60934F020D
:1097400070935002809351029093520208953F9279
:109750004F925F926F927F928F929F92AF92BF9241
:10976000CF92DF92EF92FF920F931F93CF93DF93ED
:10977000CDB7DEB7E9970FB6F894DEBF0FBECDBF09
:1097800081E40E9431418823B1F182E70E94314196
:109790008823A9F0EAE1F4E08191882339F09091DF
:1097A000C00095FFFCCF8093C600F6CF8091C0002B
:1097B00085FFFCCF8AE08093C6000C94E26186E7C7
:1097C0000E943141882311F40C94E261E0E2F4E05C
:1097D0008191882339F09091C00095FFFCCF809350
:1097E000C600F6CF8091C00085FFFCCF8AE0809351
:1097F000C6000C94E26187E40E943141882309F499
:109800004CC20E941D410E94E6AF6A30710509F406
:10981000AFC09CF46230710509F44CC024F477FFAA
:1098200025C00C94E2616330710509F44EC06430C8
:10983000710509F455C00C94E2616A35710509F4AB
:10984000D8C154F46B30710509F498C06C317105BE
:1098500009F49AC00C94E2616B35710509F4CDC12D
:109860006C35710509F4CEC10C94E26180914C080D
:1098700081110C94E2610E94AB4180912D0A8823F2
:10988000A9F088E50E943141811110C089E50E944C
:10989000314181110BC08AE50E943141811106C01E
:1098A00085E40E94314181110C94E5610E94F142EE
:1098B0000C94E26180914C0881110C94E2610E9449
:1098C0002A4281E0FBD80C94E26180914C0881111E
:1098D0000C94E2610E942A4280E0F0D80C94E2618C
:1098E00082E09CE00E94C77680E50E943141882397
:1098F00039F00E941D410E94EBAF4B015C0103C097
:10990000812C912C540183E50E943141882361F020
:109910000E941D4120E030E04AE754E40E944CB22E
:109920000E94EBAF4B015C010E9414940E9408AAB4
:109930006B017C01C80CD91CEA1CFB1C0E9408AA04
:1099400060935A0870935B0880935C0890935D085D
:109950000E9408AA6C157D058E059F0510F00C94D9
:10996000E2610E94B31E80E071DD0E947677F0CF45
:1099700060E081E00E94B0430C94E26160E080E02E
:109980000E94B0430C94E2618091210290912202E6
:10999000A0912302B09124028093FB099093FC09CB
:1099A000A093FD09B093FE0980915D0290915E0243
:1099B0009093580A8093570A84E690E090935E0251
:1099C00080935D020E9408AA60935A0870935B0816
:1099D00080935C0890935D0881E00E94C88C809120
:1099E000440A9091450AA091460AB091470A809393
:1099F0000F0A9093100AA093110AB093120A809153
:109A0000480A9091490AA0914A0AB0914B0A809362
:109A1000130A9093140AA093150AB093160A809122
:109A20004C0A90914D0AA0914E0AB0914F0A809332
:109A3000170A9093180AA093190AB0931A0A8091F2
:109A4000500A9091510AA091520AB091530A809302
:109A50001B0A90931C0AA0931D0AB0931E0A109231
:109A6000210210922202109223021092240288E511
:109A70000E943141882311F090E00AC089E50E94DC
:109A800031418111F9CF8AE50E94314191E0982757
:109A90009093250291110C94146288E50E94314143
:109AA00081110C9414628091250281110C941A6228
:109AB00089E50E94314181110C941A6288E50E9467
:109AC00031418823D1F00E942641672B682B692BF6
:109AD000A1F00E941D412091380A3091390A40912D
:109AE0003A0A50913B0A0E949EAE6093440A7093DA
:109AF000450A8093460A9093470A89E50E943141BE
:109B00008823D1F00E942641672B682B692BA1F096
:109B10000E941D4120913C0A30913D0A40913E0A2D
:109B200050913F0A0E949EAE6093480A7093490A82
:109B300080934A0A90934B0A8091250281110C94DC
:109B400020628AE50E94314181110C9420628AE5ED
:109B50000E9431418823D1F00E942641672B682B57
:109B6000692BA1F00E941D412091400A3091410AC9
:109B70004091420A5091430A0E949EAE60934C0A63
:109B800070934D0A80934E0A90934F0A20E53AE075
:109B90004CE45AE068E47AE084E49AE00E9415A577
:109BA00080E00E94C88C8091FB099091FC09A091F3
:109BB000FD09B091FE098093210290932202A093A7
:109BC0002302B09324028091570A9091580A9093EF
:109BD0005E0280935D020E9408AA60935A08709307
:109BE0005B0880935C0890935D080E94C18C0C9484
:109BF000E2611092EE090C94E26181E08093EE093B
:109C00000C94E26185E40E943141811102C00E94FE
:109C1000149457ECC52E54E0D52E68E3E62E6AE086
:109C2000F62E04E41AE0B12CF60181916F010E9436
:109C30003141882339F1F3E0BF120CC00E941D416D
:109C4000F801608371838283938380E59AE00E94A8
:109C5000BAA518C00E941D41F701208131814281BF
:109C600053810E949EAEF801608371838283938347
:109C700020E53AE04CE45AE068E47AE084E49AE0D3
:109C80000E9415A5B394F4E0EF0EF11C0C5F1F4F7A
:109C900024E0B212C9CF0C94E2618DE40E943141FC
:109CA000882311F40C9411610E941D410E94E6AFBB
:109CB0006537710511F40C94B7560CF0A6C06032EC
:109CC000710509F4F0C20CF056C06731710509F452
:109CD00045C254F56231710509F468C7BCF477FFD9
:109CE00002C00C94E261623071050CF461C1613113
:109CF000710511F00C94E26189EC9BE00E94C7763B
:109D000017981698159814980C94E26165317105AE
:109D100009F418C20CF01CC26431710511F00C94E6
:109D2000E261E9EBFBE0EAC16B31710509F442C283
:109D3000B4F46931710509F429C20CF02DC28DE526
:109D40009AE00E9477310E9408AA609352087093AB
:109D5000530880935408909355080C94E2616E3137
:109D6000710509F462C20CF03AC36C31710509F453
:109D700027C20C94E2616C35710509F46AC7ECF4F2
:109D80006235710509F409C764F46035710509F499
:109D9000DAC60CF0E5C66A32710509F47EC30C948C
:109DA000E2616435710509F401C70CF4FAC6653542
:109DB000710509F433C70C94E2616B36710509F43F
:109DC000BCC664F46936710509F4DEC30CF085C6BF
:109DD0006836710509F4A8C30C94E2616037710517
:109DE00009F4BFC334F46D36710509F4D9C40C9479
:109DF000E2616237710509F4CEC76337710511F06E
:109E00000C94E261EFE3FAE0ADC76D3D710511F42A
:109E10000C94C15A0CF04DC06B3C710511F40C94BC
:109E20003B5944F56C38710509F49DC39CF46837BF
:109E3000710511F40C94AB576937710511F40C944A
:109E4000B0576737710511F00C94E261E7E2F4E076
:109E50000C94BB57683C710511F40C94A558693CEF
:109E6000710511F40C941A596E3B710511F00C94A4
:109E7000E26120C56F3C710511F40C94F75954F45C
:109E80006D3C710511F40C947A5914F40C945859E2
:109E90000C94DA59613D710511F40C94525A14F482
:109EA0000C942C5A6C3D710511F40C94B25A0C941C
:109EB000E261603931E0730711F40C94845C54F56D
:109EC0006E3291E0790711F40C943E5C84F46C32AC
:109ED000F1E07F0711F40C94425B14F00C94785B72
:109EE000623E710511F40C94E75A0C94E2616E35F0
:109EF00031E0730711F40C947E606F3581E07807D0
:109F000011F40C94B5606F32714011F00C94E26161
:109F10000C944C5C6835E2E07E0711F40C94625DB1
:109F2000BCF4663F21E0720711F40C94875C673F34
:109F300031E0730711F40C948A5C653F714011F0B5
:109F40000C94E2610E9438880E940A840C94E261B9
:109F50006B3893E0790711F40C9458603CF4633546
:109F6000734011F40C948D5C0C94E261603A23E030
:109F7000720709F401C2673E734011F00C94E2616C
:109F800010924C080E94DA768091EF099091F009C6
:109F9000A091F109B091F2098093F3099093F4092B
:109FA000A093F509B093F6090E9480410C94E261F8
:109FB00000915E0810915F080E5F1F4F80E50E94C0
:109FC0003141882379F00E941D410E94EBAF6B0163
:109FD0007C01BB24B394611571058105910531F4B1
:109FE000B12C04C0B12CC12CD12C760183E50E9488
:109FF0003141882399F00E941D4120E030E04AE77A
:10A0000054E40E944CB20E94EBAF6B017C01AA2485
:10A01000A394611571058105910509F4A12C6AE2EB
:10A0200070E0C8010E94FAB6009711F0FC0110829E
:10A03000F801CF0121912032E1F3B11007C0A11046
:10A0400005C0222319F00E940F7304C081EF9BE02A
:10A050000E94C77681E00E94EF720E9414940E94D1
:10A0600008AA60935A0870935B0880935C089093E9
:10A070005D08C114D104E104F104A9F00E9408AA0A
:10A080004B015C018C0C9D1CAE1CBF1C0E9408AADD
:10A09000681579058A059B05B8F40E943878811106
:10A0A00013C00C9426620E943678882311F40C9415
:10A0B000E2610E94387881110AC00E94B31E80E0DC
:10A0C000C5D90E947677F5CF80E00E94EF7280912B
:10A0D0005F0A882331F082EE9BE00E94C7760C94E1
:10A0E000E26182ED9BE00E94C7760C94E261909160
:10A0F000C00095FFFCCF8093C600319684918111FA
:10A10000F6CF8091C00085FFFCCF8AE08093C60027
:10A110008DE59AE00E945330EBEAFBE084918823BE
:10A1200041F09091C00095FFFCCF8093C60031961E
:10A13000F5CF8091C00085FFFCCF8AE08093C600F8
:10A140000C94E2618DE59AE00E94A8300C94E261E3
:10A150008DE59AE00E9473310C94E26100915E08F3
:10A1600010915F080C5F1F4F6AE270E0C8010E9407
:10A17000FAB6009711F0FC01108221E041E0B8012D
:10A180008DE59AE00E94DA350C94E2618DE59AE063
:10A190000E947E310C94E2618091600A882311F460
:10A1A0000C94E26183E50E94314181110C942F628D
:10A1B0000C94E2618DE59AE00E9422330C94E261F6
:10A1C00080915E0890915F086AE270E004960E94B8
:10A1D000FAB68C010097D9F020916808309169088F
:10A1E00040E6429FC001439F900D11246EE470E051
:10A1F0008259974F0E94FAB660E270E00E94FAB668
:10A20000019690935F0880935E08F8011082609138
:10A210005E0870915F086C5F7F4F21E040E08DE544
:10A220009AE00E94DA350C94E2618091600A8823FA
:10A2300011F40C94E26160E08DE59AE00E946B35C8
:10A2400080915E0890915F086AE270E004960E9437
:10A25000FAB68C010097D9F020916808309169080E
:10A2600040E6429FC001439F900D11246EE470E0D0
:10A270008259974F0E94FAB660E270E00E94FAB6E7
:10A28000019690935F0880935E08F80110826091B8
:10A290005E0870915F086C5F7F4F8DE59AE00E94C9
:10A2A000E2310C94E26180915F0A81110E94149462
:10A2B00000915E0810915F080C5F1F4F6AE270E02A
:10A2C000C8010E94FAB67C0161E270E0C8010E94F8
:10A2D000FAB6009719F08C010F5F1F4FE114F104DB
:10A2E00011F0F701108280E50E943141F82E209193
:10A2F0005E0830915F080217130708F4F12C809173
:10A30000600A882311F40C94E26121E02F2541E0DA
:10A31000B8018DE59AE00E94DA3583E50E9431416B
:10A320008823B9F020915E0830915F08201731072B
:10A3300080F40E942641AB01BC014093FA0C50937B
:10A34000FB0C6093FC0C7093FD0C85E49CE00E9478
:10A35000EA128DE59AE00E947731F1100C94E261E7
:10A360000E9408AA6093520870935308809354087F
:10A37000909355080C94E26180915E0890915F087B
:10A380006AE270E005960E94FAB68C010097D9F057
:10A39000209168083091690840E6429FC001439FC0
:10A3A000900D11246EE470E08259974F0E94FAB626
:10A3B00060E270E00E94FAB6019690935F08809385
:10A3C0005E08F801108260915E0870915F086B5F13
:10A3D0007F4F8DE59AE00E9404390C94E2610E945F
:10A3E00008AA60934E0870934F088093500890938A
:10A3F000510800915208109153082091540830914F
:10A400005508601B710B820B930B28EE33E040E084
:10A4100050E00E9455B3CA01B9012CE330E040E09E
:10A4200050E00E9455B37F936F933F932F938CE935
:10A430009BE09F938F93CE0101969F938F930E94F1
:10A4400032B7E0EBFEE084910FB6F894DEBF0FBEAA
:10A45000CDBF882349F09091C00095FFFCCF809339
:10A46000C60031968491F5CFFE0131968191882303
:10A4700039F09091C00095FFFCCF8093C600F6CFD5
:10A480008091C00085FFFCCF8AE08093C600CE019A
:10A4900001960E940F730C94E26183E50E943141A2
:10A4A000882311F40C94E2610E941D410E94E6AFE2
:10A4B000F62EE72E862F9E2D8C0180E50E943141DD
:10A4C000882331F00F3F110509F010F40C9440621D
:10A4D0000DE010E0EFE8F4E0819191918017910791
:10A4E00011F40C94E26134E0E73CF307A9F706307D
:10A4F000110539F48F2D9E2D90932F0A80932E0AEB
:10A5000004C017FF02C00C94E26161E0802F0E943A
:10A5100028A96F2D802F0E9461A96F2D7E2D802F7D
:10A520000E941EA80C94E26188E690E043D8811155
:10A530000C94E26183E50E943141882371F000911F
:10A540004D080E941D4110E0000F111F085B174FBE
:10A550000E94E6AFF801718360830E9485210C940C
:10A56000E2610E94104683E50E943141882311F484
:10A570000C94E2610E941D410E94E6AF709347086F
:10A58000609346080C94E26189E690E013D881114B
:10A590000C94E261E6E9FBE08491882341F090911C
:10A5A000C00095FFFCCF8093C6003196F5CFE091B7
:10A5B0004D0824E0E29FF0011124E05CF74F408158
:10A5C00051816281738121E030E08CE99DE00E943D
:10A5D000078CE3E9FBE08491882341F09091C0006F
:10A5E00095FFFCCF8093C6003196F5CFE0914D08E2
:10A5F000F0E0EE0FFF1FE85BF74F60817181882765
:10A6000077FD8095982F0E9419B0AB01BC0121E025
:10A6100030E08CE99DE00E94078CEFE8FBE084913C
:10A62000882341F09091C00095FFFCCF8093C60035
:10A630003196F5CF40913A0850913B0860913C0823
:10A6400070913D0821E030E08CE99DE00E94078C8C
:10A65000ECE8FBE08491882341F09091C00095FFE5
:10A66000FCCF8093C6003196F5CF6091460870917B
:10A670004708882777FD8095982F0E9419B0AB0175
:10A68000BC0121E030E08CE99DE00E94078CE9E804
:10A69000FBE08491882341F09091C00095FFFCCFAE
:10A6A0008093C6003196F5CF4AE050E060E070E05C
:10A6B0008CE99DE00E94318BE7E8FBE084918823E0
:10A6C00041F09091C00095FFFCCF8093C600319679
:10A6D000F5CF409140085091410860914208709137
:10A6E000430821E030E08CE99DE00E94078CE4E81B
:10A6F000FBE08491882341F09091C00095FFFCCF4E
:10A700008093C6003196F5CF609148087091490852
:10A71000882777FD8095982F0E9419B0AB01BC0166
:10A7200021E030E08CE99DE00E94078CE0E8FBE04E
:10A730008491882341F09091C00095FFFCCF8093D5
:10A74000C6003196F5CF80914D0890E00E947D1EA5
:10A750004AE050E0BC018CE99DE00E94318BEBE7C0
:10A76000FBE08491882341F09091C00095FFFCCFDD
:10A770008093C6003196F5CF8FEF9FEF0E947D1E2C
:10A780004AE050E0BC018CE99DE00E94318B809151
:10A79000C00085FFFCCF8AE08093C6000C949E63C6
:10A7A0008DE690E00E94DA4A81110C94E26180E724
:10A7B0009BE00E94C77683E50E943141882391F097
:10A7C00000914D080E941D4110E0000F111F085B11
:10A7D000174F0E94E6AFF8017183608381E0809398
:10A7E0001C0215C082E50E943141882381F000914E
:10A7F0004D080E941D4110E0000F111F085B174F0C
:10A800000E94E6AFF8017183608310921C020E94DF
:10A8100085210E9408AA4B015C0100914D0810E0BF
:10A82000F801EE0FFF1FE85BF74F60817181882709
:10A8300077FD8095982F0E9419B0F801EE0FFF1F49
:10A84000EE0FFF1FE05CF74F11E020813181428164
:10A8500053810E947AB118160CF010E010934B0847
:10A8600010921F0ACC24CA94DC2C760148EE442EA8
:10A8700043E0542E612C712C5AE0352E80911F0A32
:10A8800081110C945B63FFEFCF16DF06EF06FF0626
:10A8900011F40C944762F7FE02C00C945B630E94B3
:10A8A00008AA6C197D09683B7B4010F40C94476240
:10A8B0000C945B638AE49BE00E94C77683E50E9468
:10A8C0003141882361F00E941D410E94E6AF7093E0
:10A8D00047086093460881E080931C020FC082E520
:10A8E0000E943141882351F00E941D410E94E6AF31
:10A8F000709347086093460810921C020E9408AAB1
:10A900004B015C0110921F0A609146087091470844
:10A91000882777FD8095982F0E9419B011E020912B
:10A920003A0830913B0840913C0850913D080E9404
:10A930007AB118160CF010E010934B0807E41BE0F6
:10A94000E3E4EE2EEBE0FE2EFFE3CF2EFBE0DF2E66
:10A95000AAE07A2E80914B086091460870914708D2
:10A96000882309F48BC080911F0A811187C0882732
:10A9700077FD8095982F0E9419B020913A08309168
:10A980003B0840913C0850913D080E947AB118164E
:10A990000CF08BC00E9408AA681979098A099B09E2
:10A9A000693E73408105910508F460C0E091300A6A
:10A9B00084E0E89FF0011124E05CF74F4081518171
:10A9C00062817381F8018491E7E4FBE0882349F018
:10A9D0009091C00095FFFCCF8093C6003196849182
:10A9E000F5CF22E030E08CE99DE00E94078CF70172
:10A9F0008491E3E4FBE0882349F09091C00095FF47
:10AA0000FCCF8093C60031968491F5CF6091300AD7
:10AA100070E04AE050E08CE99DE00E94318BF60145
:10AA20008491EFE3FBE0882349F09091C00095FF0B
:10AA3000FCCF8093C60031968491F5CF40913A08BF
:10AA400050913B0860913C0870913D0821E030E056
:10AA50008CE99DE00E94078C8091C00085FFFCCFAF
:10AA60007092C6000E9408AA4B015C010E94B31EAE
:10AA700080E00E94264A0E9476776CCF882777FD77
:10AA80008095982F0E9419B020913A0830913B0888
:10AA900040913C0850913D080E9477AF87FF05C068
:10AAA00080911C02882309F475CF85E39BE00E9406
:10AAB000C77680915F0A882321F08EE793E00E9499
:10AAC0000F730E9408AA60935A0870935B088093E2
:10AAD0005C0890935D080C94E26183E50E9431412B
:10AAE000882319F10E941D4120E030E0A9010E9455
:10AAF00077AF87FD0FC00E941D4120E030E04FE797
:10AB000053E40E947AB1181644F00E941D410E943D
:10AB1000E6AF05C060E070E002C06FEF70E07093D8
:10AB20002F0A60932E0A0C94E2618FEF90E09093CD
:10AB30002F0A80932E0A0C94E26110922F0A109231
:10AB40002E0A0C94E2619B9AA39881E080932602DE
:10AB500085E29BE00E94C7760E9476770C94E261C2
:10AB60000E9486210E941494149A0E947E9410924E
:10AB70002F0A10922E0A68EE73E080E090E00E94A7
:10AB800037AA9B9AA39A1092260287E19BE00E9423
:10AB9000C7760E9476770C94E26110925C0A0C945E
:10ABA000E26181E080935C0A0C94E26183E50E949B
:10ABB00031418823A1F00E941D4120E030E04AE7A6
:10ABC00054E40E944CB20E94EBAF60931D0270935C
:10ABD0001E0280931F02909320020C94E26188E58C
:10ABE0000E94314181110C947C6389E50E943141BE
:10ABF00081110C947C638AE50E94314181110C948F
:10AC00007C6385E40E94314181110C947C630E9435
:10AC10001494149A0E947E940C94E26183E50E943D
:10AC20003141882311F40C94E2610E941D4120E01F
:10AC300030E04AE754E40E944CB20E94EBAF6093CC
:10AC400056087093570880935808909359080C94AD
:10AC5000E26127EC34E039AF28AF01EA13E161EBA0
:10AC6000862E63E1962E75E6A72E73E1B72E312C62
:10AC7000E8ADF9AD8191F9AFE8AF0E943141882389
:10AC800009F45BC0F3E03F1251C00E941D416B010B
:10AC90007C0120E030E040EA51E40E9477AF87FF7A
:10ACA0003FC0A7019601F801608171818281938183
:10ACB0000E947EAF2B013C019B01AC016091791396
:10ACC00070917A1380917B1390917C130E944CB207
:10ACD0006093791370937A1380937B1390937C1312
:10ACE000A3019201F40160817181828193810E94AC
:10ACF0004CB2F4016083718382839383F501608198
:10AD00007181828193810E9417B0A30192010E94F8
:10AD10004CB20E94EBAFF501608371838283938311
:10AD2000F801C082D182E282F38207C00E941D41F5
:10AD3000F801608371838283938333940C5F1F4F88
:10AD4000F4E08F0E911C24E0A20EB11C34E033120B
:10AD50008FCF0C94E2619091C00095FFFCCF80935F
:10AD6000C600319684918111F6CF0C94E261009176
:10AD70005E0810915F080B5F1F4F6AE270E0C80128
:10AD80000E94FAB6009711F0FC011082C8010E94DF
:10AD90000F730C94E261ECE3FAE08491882341F0B4
:10ADA0009091C00095FFFCCF8093C6003196F5CFFF
:10ADB0004091440A5091450A6091460A7091470AB1
:10ADC00022E030E08CE99DE00E94078CE8E3FAE0A5
:10ADD0008491882341F09091C00095FFFCCF80932F
:10ADE000C6003196F5CF4091480A5091490A6091CA
:10ADF0004A0A70914B0A22E030E08CE99DE00E9403
:10AE0000078CE4E3FAE08491882341F09091C0003C
:10AE100095FFFCCF8093C6003196F5CF40914C0A48
:10AE200050914D0A60914E0A70914F0A22E030E035
:10AE30008CE99DE00E94078CE0E3FAE0849188238E
:10AE400041F09091C00095FFFCCF8093C6003196F1
:10AE5000F5CF4091500A5091510A6091520A709179
:10AE6000530A22E030E08CE99DE00E94078CE5E285
:10AE7000FAE08491882341F09091C00095FFFCCFC7
:10AE80008093C6003196F5CF0E9470940E9419B04D
:10AE90002091A1133091A2134091A3135091A413B8
:10AEA0000E947EAFAB01BC0122E030E08CE99DE066
:10AEB0000E94078CE1E2FAE08491882341F09091AE
:10AEC000C00095FFFCCF8093C6003196F5CF81E09E
:10AED0000E9470940E9419B02091A5133091A6137E
:10AEE0004091A7135091A8130E947EAFAB01BC0103
:10AEF00022E030E08CE99DE00E94078CEDE1FAE071
:10AF00008491882341F09091C00095FFFCCF8093FD
:10AF1000C6003196F5CF82E00E9470940E9419B06D
:10AF20002091A9133091AA134091AB135091AC1307
:10AF30000E947EAFAB01BC0122E030E08CE99DE0D5
:10AF40000E94078C8091C00085FFFCCF8AE080932F
:10AF5000C6000C94E26180E00E94C88C0C94E2610F
:10AF600081E00E94C88C0C94E2619091C00095FF32
:10AF7000FCCF8093C60081918111F7CF8091C000F2
:10AF800085FFFCCF8AE08093C600E5E1FAE084917A
:10AF9000882341F09091C00095FFFCCF8093C600BC
:10AFA0003196F5CF1E9B03C0EBE0F4E009C0E5E16C
:10AFB000F4E006C09091C00095FFFCCF8093C600DE
:10AFC00081918111F7CF8091C00085FFFCCF8AE08D
:10AFD0008093C600EDE0FAE08491882341F09091DF
:10AFE000C00095FFFCCF8093C6003196F5CF029943
:10AFF00003C0EBE0F4E009C0E5E1F4E006C09091A5
:10B00000C00095FFFCCF8093C60081918111F7CFDE
:10B010008091C00085FFFCCF8AE08093C600E5E008
:10B02000FAE08491882341F09091C00095FFFCCF15
:10B030008093C6003196F5CF1D9B03C0EBE0F4E092
:10B0400009C0E5E1F4E006C09091C00095FFFCCF97
:10B050008093C60081918111F7CF8091C00085FF58
:10B06000FCCF8AE08093C600EDEFF9E0849188235D
:10B0700041F09091C00095FFFCCF8093C6003196BF
:10B08000F5CF019903C0EBE0F4E009C0E5E1F4E09D
:10B0900006C09091C00095FFFCCF8093C6008191BF
:10B0A0008111F7CF8091C00085FFFCCF8AE08093AB
:10B0B000C600E5EFF9E08491882341F09091C0004B
:10B0C00095FFFCCF8093C6003196F5CF1C9B03C043
:10B0D000EBE0F4E009C0E5E1F4E006C09091C000C7
:10B0E00095FFFCCF8093C60081918111F7CF8091AD
:10B0F000C00085FFFCCF8AE08093C600EDEEF9E04A
:10B100008491882341F09091C00095FFFCCF8093FB
:10B11000C6003196F5CF379903C0EBE0F4E009C0E3
:10B12000E5E1F4E006C09091C00095FFFCCF80936C
:10B13000C60081918111F7CF8091C00085FFFCCFBF
:10B140008AE08093C6000C94E2618091300A80937B
:10B150004D0884E50E943141882319F10E941D4168
:10B160000E94EBAF60934D086623D9F0E0EBFEE060
:10B170008491882341F09091C00095FFFCCF80938B
:10B18000C6003196F5CFE0E4F4E08191882311F414
:10B190000C94E2619091C00095FFFCCF8093C600B3
:10B1A000F4CF84E40E943141882311F40C94E261CD
:10B1B0000E941D4120E030E0A9010E9477AF81117B
:10B1C00003C01092540A32C000914D0810E00E9452
:10B1D0001D41F801EE0FFF1FEE0FFF1FED5AFD4F4F
:10B1E0006083718382839383E0905302F0905402D2
:10B1F000009155021091560220E030E0A901B701FC
:10B20000C8010E9477AF811104C0E12CF12C00E449
:10B2100010E4C701D8018093530290935402A09385
:10B220005502B093560281E08093540A0E94954BD8
:10B230000C94E26107EC14E041E9E42E43E1F42EC2
:10B24000F80181918F010E943141882349F00E94C9
:10B250001D410E94EBAFF70160837183828393836A
:10B26000F4E0EF0EF11C24E00B3C120749F70E94BA
:10B27000E7A50C94E26107EC14E031EBE32E33E137
:10B28000F32EF80181918F010E943141882339F01A
:10B290000E941D41F7016083718382839383F4E0F0
:10B2A000EF0EF11C24E00B3C120759F70C94E261FD
:10B2B00083E50E943141882351F00E941D41609333
:10B2C000891370938A1380938B1390938C1384E566
:10B2D0000E943141882311F40C94E2610E941D41C7
:10B2E00060938513709386138093871390938813CC
:10B2F0000C94E26183E50E943141882351F00E9461
:10B300001D4160938D1370938E1380938F139093D0
:10B31000901384E50E943141882351F00E941D4121
:10B3200060937513709376138093771390937813CB
:10B3300082E40E943141882361F00E941D410E94F5
:10B34000EBAF6093C1137093C2138093C3139093B8
:10B35000C41388E50E943141882351F00E941D41A9
:10B36000609381137093821380938313909384135B
:10B370008AE50E943141882351F00E941D4160936B
:10B380007D1370937E1380937F139093801385E4D5
:10B390000E943141882311F40C94E2610E941D4106
:10B3A0006093791370937A1380937B1390937C133B
:10B3B0000C94E26107EC14E028E3E22E2AE0F22E7E
:10B3C000F80181918F010E943141882339F00E9458
:10B3D0001D41F7016083718382839383F4E0EF0E54
:10B3E000F11C24E00A3C120709F4ECC7E9CF83E51D
:10B3F0000E943141882351F00E941D416093330225
:10B4000070933402809335029093360286E40E9452
:10B410003141882381F00E941D4120E030E040E767
:10B4200052E40E947EAF60932B0270932C028093B3
:10B430002D0290932E028AE50E943141882309F45F
:10B44000C1C70E941D416093280A7093290A809306
:10B450002A0A90932B0AB6C783E50E9431418823BC
:10B4600051F00E941D416093240A7093250A809335
:10B47000260A9093270A86E40E943141882309F422
:10B48000A1C70E941D4120E030E040E752E40E9445
:10B490007EAF6093270270932802809329029093D5
:10B4A0002A0290C783E50E943141882309F48AC7A4
:10B4B0000E941D410E94E6AF6115710549F061309F
:10B4C000710559F481E080932D0A10922C0A7AC7F5
:10B4D00010922D0A10922C0A75C7E0EBFEE08491C1
:10B4E000882341F09091C00095FFFCCF8093C60067
:10B4F0003196F5CFEAEDF9E08491882341F09091FF
:10B50000C00095FFFCCF8093C6003196F5CF8091A7
:10B5100068089091690820E6289FF001299FF00DA6
:10B520001124E259F74F8191882339F09091C0009E
:10B5300095FFFCCF8093C600F6CFE8EDF9E084914B
:10B54000882341F09091C00095FFFCCF8093C60006
:10B550003196F5CF8091C00085FFFCCF8AE08093C3
:10B56000C60030C783E50E943141882309F42AC709
:10B570000E941D410E94E6AF70935E0260935D02DF
:10B5800021C783E50E943141882309F41BC70E942B
:10B590001D410E94E6AF6B017C0184E50E943141B0
:10B5A000882381F08DED90E00E94DA4A81110AC76C
:10B5B000E0914D08F0E0EE0FFF1FE75AFD4FD182FA
:10B5C000C08200C7D0925C02C0925B02FBC680E5DD
:10B5D0000E943141882309F4F5C60E941D410E9452
:10B5E000E6AFD62E062F172F83E50E943141882320
:10B5F00031F00E941D410E94E6AF7B0103C0EE24A2
:10B60000EA94FE2CC7010196039708F0DBC6EFE829
:10B61000F4E0819191918017910709F4D3C634E049
:10B62000E73CF307B1F717FDCDC60E941494CD2C6B
:10B6300060E08D2D0E9428A98FEFE816F80631F002
:10B64000EA94EF2871F000E010E00DC08D2D0E940B
:10B6500096A931E020E0892B09F030E0032F122F6A
:10B6600002C001E010E08C2D0E9496A9801791077E
:10B6700009F4A8C60E94B31E80E00E94264A0E94D8
:10B680007677F1CF83E50E943141882331F00E9423
:10B690001D410E94E6AF8B0102C00EE610E080E57E
:10B6A0000E943141882331F00E941D410E94E6AF83
:10B6B000CB0102C088EE93E06C01EE24D7FCE0944D
:10B6C000FE2C101611067CF420E030E0A901B80130
:10B6D00084E50E94D4AAC701B6010E9437AA84E576
:10B6E0000E94E5AD6FC6C701B6010E9437AA6AC6BF
:10B6F00080E50E943141882351F00E941D416093F2
:10B7000018027093190280931A0290931B0289E425
:10B710000E943141882361F00E941D410E94F82758
:10B72000609314027093150280931602909317028F
:10B7300084E40E943141882361F00E941D410E94EF
:10B740000428609310027093110280931202909368
:10B75000130283E40E943141882351F00E941D416D
:10B7600060930C0270930D0280930E0290930F026F
:10B770000E94661EE7E5F4E08191882339F09091FC
:10B78000C00095FFFCCF8093C600F6CFEAE5F4E059
:10B790008191882339F09091C00095FFFCCF809370
:10B7A000C600F6CF409118025091190260911A021A
:10B7B00070911B0222E030E08CE99DE00E94078C32
:10B7C000EEE5F4E08191882339F09091C00095FF77
:10B7D000FCCF8093C600F6CF6091140270911502E1
:10B7E00080911602909117020E94FE27AB01BC01C6
:10B7F00022E030E08CE99DE00E94078CE2E6F4E074
:10B800008191882339F09091C00095FFFCCF8093FF
:10B81000C600F6CF60911002709111028091120261
:10B82000909113020E940A28AB01BC0122E030E093
:10B830008CE99DE00E94078CE6E6F4E08191882384
:10B8400039F09091C00095FFFCCF8093C600F6CFF1
:10B8500040910C0250910D0260910E0270910F0206
:10B8600022E030E08CE99DE00E94078C8091C000CE
:10B8700085FFFCCF8AE08093C600A4C583E50E94C3
:10B880003141882319F00E941D4103C060E070E03F
:10B89000CB010E94DEA596C585E40E943141882334
:10B8A00041F00E941D410E94E6AF8B0177FF03C06B
:10B8B00009C000E010E0C12CD12CB6E1EB2EB3E4BE
:10B8C000FB2E06C0C12CD12CACE8EA2EA2E4FA2E45
:10B8D00083E50E943141882321F00E941D416B01C4
:10B8E0007C0183E40E943141882331F00E941D4194
:10B8F0000E94E6AF9B0102C025E030E0A801C7012D
:10B90000B6010E9499215EC50E9414945BC50E94F5
:10B91000388858C50E940A8455C58AE50E9431417D
:10B92000882309F497C00E941D416B017C0120E02F
:10B9300030E040E751EC0E947AB187FD3FC020E043
:10B9400030E040EA50ECC701B6010E9477AF18160C
:10B95000ACF1F7FAF094F7F8F094C092310AD09273
:10B96000320AE092330AF092340AE0EBFEE084916E
:10B97000882341F09091C00095FFFCCF8093C600D2
:10B980003196F5CFECECF9E08491882341F0909169
:10B99000C00095FFFCCF8093C6003196F5CF809113
:10B9A000C00085FFFCCF8AE08093C6008091C00074
:10B9B00085FFFCCF8AE08093C60004C5E0EBFEE083
:10B9C0008491882341F09091C00095FFFCCF809333
:10B9D000C6003196F5CFE3ECF9E08491882341F07D
:10B9E0009091C00095FFFCCF8093C6003196F5CFB3
:10B9F000EBEBF9E08491882341F09091C00095FF32
:10BA0000FCCF8093C6003196F5CF4AE050E061EF5D
:10BA10007FEF8CE99DE00E94318BE3EBF9E08491AC
:10BA2000882341F09091C00095FFFCCF8093C60021
:10BA30003196F5CF4AE050E06BEF7FEF8CE99DE067
:10BA40000E94318B8091C00085FFFCCF8AE08093FB
:10BA5000C600B8C4E0EBFEE08491882341F09091E9
:10BA6000C00095FFFCCF8093C6003196F5CFE7EA82
:10BA7000F9E08491882341F09091C00095FFFCCFBC
:10BA80008093C6003196F5CF8091C00085FFFCCF32
:10BA90008AE08093C6004091310A5091320A609149
:10BAA000330A7091340A705822E030E08CE99DE04E
:10BAB0000E94078C8091C00085FFFCCF8AE08093B4
:10BAC000C60080C480915D0290915E0290935802FE
:10BAD00080935702C090440AD090450AE090460AED
:10BAE000F090470ACF8ED8A2E9A2FAA20091480AA4
:10BAF0001091490A20914A0A30914B0A0BA31CA3CA
:10BB00002DA33EA340914C0A50914D0A60914E0ADC
:10BB100070914F0A4FA358A769A77AA78091500A3E
:10BB20009091510AA091520AB091530A8BA79CA7F9
:10BB3000ADA7BEA7C982DA82EB82FC820D831E8389
:10BB40002F83388749875A876B877C878D879E87A5
:10BB5000AF87B88B85E40E943141882359F00E9459
:10BB60001D419B01AC016BA57CA58DA59EA50E94E6
:10BB70009EAE0AC020E030E040E050E46BA57CA51A
:10BB80008DA59EA50E949DAE6BA77CA78DA79EA7A5
:10BB9000E0E3CE2EEAE0DE2EE12CF12C08EC13E4FB
:10BBA0009E01255D3F4FAE01495D5F4FBE016D5D5A
:10BBB0007F4FCE014F960E944E9B8AE50E943141F5
:10BBC000882349F00E941D419B01AC016FA178A51B
:10BBD00089A59AA51EC020E030E040E050E46FA1A6
:10BBE00078A589A59AA50E949EAE6B017C016FA3E2
:10BBF00078A789A79AA720E030E040E251E40E94AC
:10BC000077AF87FF0CC020E030E040E251E4C7018D
:10BC1000B6010E949EAE6FA378A789A79AA760E39A
:10BC2000C62E6AE0D62EE12CF12C06E913E49E0123
:10BC3000255D3F4FAE01495D5F4FBE016D5D7F4F9A
:10BC4000CE014F960E944E9B88E50E943141882389
:10BC500079F00E941D419B01AC016F8D78A189A1F3
:10BC60009AA10E949EAE6F8F78A389A39AA308C061
:10BC700080E090E0A3E5B3E48F8F98A3A9A3BAA3D3
:10BC800089E50E943141882339F00E941D416BA350
:10BC90007CA38DA39EA304C01BA21CA21DA21EA256
:10BCA00040E3C42E4AE0D42EE12CF12C0CE812E43F
:10BCB0009E01255D3F4FAE01495D5F4FBE016D5D49
:10BCC0007F4FCE014F960E944E9B8CE40E943141E3
:10BCD000882359F00E941D419B01AC016BA57CA5F6
:10BCE0008DA59EA50E949EAE0AC020E030E040EAED
:10BCF00052E46BA57CA58DA59EA50E949DAE6BA769
:10BD00007CA78DA79EA720E3C22E2AE0D22EE12C8D
:10BD1000F12C00EA11E49E01255D3F4FAE01495D23
:10BD20005F4FBE016D5D7F4FCE014F960E944E9BCF
:10BD30000E941494149A64E670E080E090E00E94FF
:10BD400037AA0E94497200E010E0F12C0E94387876
:10BD500081112AC0F3940E94B31E81E00E94264AFA
:10BD6000F110F4CF043FE1E01E0711F400E010E011
:10BD7000809101018460809301010115110531F466
:10BD80009FB7F89480910201846008C004311105C6
:10BD900041F49FB7F894809102018B7F8093020158
:10BDA0009FBF0F5F1F4FD2CF9FB7F89480910201C2
:10BDB0008B7F809302019FBF20E030E04CE852E48B
:10BDC0006BA57CA58DA59EA50E949EAE6BA77CA7AA
:10BDD0008DA79EA710E3C12E1AE0D12EE12CF12CE5
:10BDE00000EA11E49E01255D3F4FAE01495D5F4FC2
:10BDF000BE016D5D7F4FCE014F960E944E9B20E0AD
:10BE000030E048E452E46BA57CA58DA59EA50E9478
:10BE10009EAE6BA77CA78DA79EA7E12CF12C00E01E
:10BE200010E49E01255D3F4FAE01495D5F4FBE01AD
:10BE30006D5D7F4FCE014F960E944E9B1092560A29
:10BE40001092550A0E94AF728091550A9091560A3D
:10BE5000019709F47CC01092560A1092550A0E946C
:10BE60003E788091550A9091560A8230910549F1A9
:10BE7000039709F069C020E030E048E452E46BA584
:10BE80007CA58DA59EA50E949EAE6BA77CA78DA7C5
:10BE90009EA770E3C72E7AE0D72EE12CF12C00E0AC
:10BEA00010E49E01255D3F4FAE01495D5F4FBE012D
:10BEB0006D5D7F4FCE014F960E944E9B0E946F7228
:10BEC000C3CF20E030E04CE852E46BA57CA58DA503
:10BED0009EA50E949EAE6BA77CA78DA79EA7F0E3B0
:10BEE000CF2EFAE0DF2EE12CF12C00EA11E49E01C6
:10BEF000255D3F4FAE01495D5F4FBE016D5D7F4FD8
:10BF0000CE014F960E944E9B20E030E048E452E480
:10BF10006BA57CA58DA59EA50E949EAE6BA77CA758
:10BF20008DA79EA7E12CF12C00E010E49E01255D79
:10BF30003F4FAE01495D5F4FBE016D5D7F4FCE014A
:10BF40004F960E944E9B7ECF0E9462727DCF20E072
:10BF500030E040EA50E46BA57CA58DA59EA50E942B
:10BF60009EAE6BA77CA78DA79EA790E3C92E9AE0F3
:10BF7000D92EE12CF12C00E010E49E01255D3F4F0D
:10BF8000AE01495D5F4FBE016D5D7F4FCE014F96A3
:10BF90000E944E9BA80197016BA57CA58DA59EA52F
:10BFA0000E949DAE6BA77CA78DA79EA7E12CF12CCC
:10BFB00008EC13E49E01255D3F4FAE01495D5F4FE4
:10BFC000BE016D5D7F4FCE014F960E944E9BE12CCE
:10BFD000F12C0CE812E49E01255D3F4FAE01495D56
:10BFE0005F4FBE016D5D7F4FCE014F960E944E9B0D
:10BFF0009E01255D3F4FAE01495D5F4FBE016B5F06
:10C000007F4FCE0101960E944E9BE12CF12C08E45B
:10C0100013E49E01255D3F4FAE01475F5F4FBE01B8
:10C020006B5F7F4FCE0101960E944E9B20E030E077
:10C0300040E050E46BA57CA58DA59EA50E949EAE18
:10C040006BA77CA78DA79EA7E12CF12C00EA10E43A
:10C050009E01255D3F4FAE01475F5F4FBE016B5FA5
:10C060007F4FCE0101960E944E9BCE010D960E94FD
:10C07000BAA5809157029091580280935D029093E7
:10C080005E029F938F938EE999E09F938F938E0129
:10C09000015D1F4F1F930F930E9432B7C8010E948A
:10C0A000AE3E0F900F900F900F900F900F908AC19F
:10C0B00088E50E943141882339F00E941D410E9489
:10C0C000E6AF80E00E941C958AE50E9431418823FA
:10C0D00039F00E941D410E94E6AF81E00E941C954C
:10C0E00085E40E943141882309F46CC10E941D41FE
:10C0F0000E94E6AF82E00E941C9564C183E50E9425
:10C100003141811104C007EC14E0F12C10C010E0A3
:10C110000E941D410E94EBAF812F0E94BB951F5FC3
:10C120001530B1F7F0CFF394F4E0FF1679F0F80191
:10C1300081918F010E9431418823A9F30E941D4102
:10C140000E94EBAF8F2D0E94BB95EDCF82E40E9441
:10C150003141882339F00E941D410E94EBAF84E0F9
:10C160000E94BB950E9481962DC183E50E943141BA
:10C17000882309F453C00E941D410E94E6AF61303C
:10C18000710541F06230710509F048C007EC14E018
:10C19000F12C25C007EC14E0F12CF80181918F01FE
:10C1A0000E943141882341F00E941D410E94E6AF68
:10C1B0004FEF8F2D0E947D95F394F4E0FF12EDCFA9
:10C1C00082E40E943141882349F10E941D410E946E
:10C1D000E6AF4FEF20C0F394F4E0FF1689F0F801CA
:10C1E00081918F010E9431418823A9F30E941D4152
:10C1F0000E94E6AF462F6FEF8F2D0E947D95EBCF0B
:10C2000082E40E943141882349F00E941D410E942E
:10C21000E6AF462F6FEF84E00E947D950E948196E5
:10C22000D1C084E50E943141882309F487C00E946F
:10C230001D410E94EBAF60934D086623A9F1E0EB2E
:10C24000FEE08491882341F09091C00095FFFCCFDF
:10C250008093C6003196F5CFEAE6F4E08191882319
:10C2600039F09091C00095FFFCCF8093C600F6CFC7
:10C2700040E050E060914D088CE99DE00E94688BA1
:10C28000ECE6F4E08191882339F09091C00095FFAD
:10C29000FCCF8093C600F6CF8091C00085FFFCCF15
:10C2A0008AE08093C6008EC086E40E9431418823D4
:10C2B000D9F00E941D416B017C016093FF097093CE
:10C2C000000A8093010A9093020A20E030E0A9015D
:10C2D0000E947AB1181644F4C0922102D092220230
:10C2E000E0922302F0922402E0EBFEE084918823A6
:10C2F00041F09091C00095FFFCCF8093C60031962D
:10C30000F5CFEDE7F4E08191882339F09091C000FA
:10C3100095FFFCCF8093C600F6CF6091300A70E0A5
:10C320004AE050E08CE99DE00E94318B8091C00092
:10C3300085FFFCCF8AE08093C60044C0E0EBFEE0BE
:10C340008491882341F09091C00095FFFCCF8093A9
:10C35000C6003196F5CFEBE8F9E08491882341F0EF
:10C360009091C00095FFFCCF8093C6003196F5CF29
:10C37000809168089091690820E6289FF001299F24
:10C38000F00D1124E259F74F8191882339F09091F3
:10C39000C00095FFFCCF8093C600F6CFE9E8F9E036
:10C3A0008491882341F09091C00095FFFCCF809349
:10C3B000C6003196F5CF8091C00085FFFCCF8AE0A2
:10C3C0008093C6000E945841B9C1C0901B0AD0900A
:10C3D0001C0AE0901D0AF0901E0A2091500A30912C
:10C3E000510A4091520A5091530AC701B6010E9466
:10C3F0009DAE2DEC3CEC4CEC5DE30E947AB118163E
:10C4000014F00C94564CC092500AD092510AE0920B
:10C41000520AF092530A80E59AE00E94BAA560E0C1
:10C4200080E00E94B0438AC180E090E00E941C3D01
:10C430000C94534D81E090E00E941C3D0C945E4DA5
:10C4400082E090E00E941C3D0C94A74D0E94B31E18
:10C4500080E00E94264A0E9476770C9446500E9403
:10C460002641AB01BC014093FA0C5093FB0C609346
:10C47000FC0C7093FD0C85E49CE00E94EA12A2CFB4
:10C480000E941D410E94E6AF8B010C946A520E94EB
:10C4900008AA681979098A099B09693E73408105D0
:10C4A000910508F479C0EDE6FBE08491882341F022
:10C4B0009091C00095FFFCCF8093C6003196F5CFD8
:10C4C000E0914D0824E0E29FF0011124E05CF74F79
:10C4D000408151816281738121E030E08CE99DE0EF
:10C4E0000E94078CE9E6FBE08491882341F090915B
:10C4F000C00095FFFCCF8093C6003196F5CF6091C8
:10C500004D0870E04AE050E08CE99DE00E94318BDC
:10C51000E5E6FBE08491882341F09091C00095FF0F
:10C52000FCCF8093C6003196F5CFF7FE03C0E6E757
:10C53000F5E025C00E9408AA8B019C01C701B60145
:10C540006854744F8F4F9F4F601B710B820B930B7E
:10C55000A30192010E9455B3BA01A9012AE030E07B
:10C560008CE99DE00E945D8B8091C00085FFFCCF2F
:10C570000DC09091C00095FFFCCF8093C6008191C3
:10C580008111F7CF8091C00085FFFCCF3092C600AB
:10C590000E9408AA4B015C010E94B31E80E00E9429
:10C5A000264A0E947677FFEFCF16DF06EF06FF06DA
:10C5B00009F046C080914B08E0914D08F0E08F01F2
:10C5C000000F111F000F111F005C174FEE0FFF1F10
:10C5D000E85BF74F608171818823C9F0882777FD78
:10C5E0008095982F0E9419B020E030E040E85FE38A
:10C5F0000E949DAE9B01AC01F80160817181828136
:10C6000093810E947AB187FF50C00C943E548827D2
:10C6100077FD8095982F0E9419B020E030E040E827
:10C620005FE30E949EAE9B01AC01F80160817181C5
:10C63000828193810E9477AF1816BCF50C943E540A
:10C64000F7FE02C00C943E54E0914D08F0E08F01DB
:10C65000000F111F000F111F005C174FEE0FFF1F7F
:10C66000E85BF74F60817181882777FD8095982F6F
:10C670000E9419B09B01AC01F80160817181828137
:10C6800093810E949DAE0E94E6AF97FF07C09095F0
:10C690008095709561957F4F8F4F9F4F66307105E4
:10C6A0008105910514F40C943E540E9408AA6B0174
:10C6B0007C010C943E5487E59BE00E94C7768091F4
:10C6C0005F0A882321F08EE793E00E940F730E9497
:10C6D00008AA60935208709353088093540890936B
:10C6E00055080E9408AA60935A0870935B088093CB
:10C6F0005C0890935D0866CE0E94149488E50E94C1
:10C700003141882319F0179A1092350A89E50E9461
:10C710003141882319F0169A1092360A8AE50E9450
:10C720003141882319F0159A1092370A85E40E9446
:10C730003141882309F446CE149A44CEE9960FB6C7
:10C74000F894DEBF0FBECDBFDF91CF911F910F9147
:10C75000FF90EF90DF90CF90BF90AF909F908F9021
:10C760007F906F905F904F903F900895CF93DF93AD
:10C770008091640890916508039714F40E945746CD
:10C7800060E08DE59AE00E94753480916408909194
:10C790006508892B09F464C080915D0A8823E1F063
:10C7A000809168089091690820E6289FE001299F00
:10C7B000D00D1124C259D74F62E77DE0CE010E940F
:10C7C000A5B6892BF1F4BE018DE59AE00E940434F0
:10C7D00080915E0A882319F00E94A74B2BC0EFE6D8
:10C7E000FDE08491882341F09091C00095FFFCCF3B
:10C7F0008093C6003196F5CF8091C00085FFFCCFB5
:10C8000016C060E08DE59AE00E946B35EDE5FDE035
:10C810008491882341F09091C00095FFFCCF8093D4
:10C82000C6003196F5CF8091C00085FFFCCF8AE02D
:10C830008093C60080916408909165080197909359
:10C840006508809364088091680890916908019652
:10C8500064E070E00E9442B3909369088093680896
:10C860000E94B31E80E00E94264A0E94268CDF911F
:10C87000CF910C9476778F929F92AF92BF92CF9286
:10C88000DF92EF92FF920F931F93CF93DF938C0170
:10C890008C519E4F0E94182E680189E8C80ED11C49
:10C8A00021F1780181E4E81A8EEFF80AE7015701D7
:10C8B0008FE1A81AB1087AEB872E75E0972ECC1578
:10C8C000DD0599F0FE01EE19FF09EA0DFB1D9182CD
:10C8D0008082FE0178978081811102C06F97EFCF2F
:10C8E000CE014B970E94CD13F9CFC80186599F4FB7
:10C8F0000E94182EC801875B9F4FDF91CF911F9137
:10C900000F91FF90EF90DF90CF90BF90AF909F90EE
:10C910008F900C94182E8DE59AE00C94242E8DE5C2
:10C920009AE0A9CFFB01609170027091710270933F
:10C930002C0D60932B0D6091350D7091360D709319
:10C940002A0D6093290D62E060936F0265E97FE72D
:10C9500070937102609370029093280D8093270D5D
:10C96000F093260DE093250D662757FD6095762FF1
:10C970004093210D5093220D6093230D7093240D4D
:10C98000C901AA2797FDA095BA2F841B950BA60B6A
:10C99000B70B80931D0D90931E0DA0931F0DB093A8
:10C9A000200D80819181AA2797FDA095BA2F841B25
:10C9B000950BA60BB70B8093350D9093360DA09376
:10C9C000370DB093380D08950F931F93CF93DF93D6
:10C9D000EB01142F022F482F60E080E49DE00E94BD
:10C9E000BF28612F80E49DE00E9496AE11E1FE0118
:10C9F0006491662311F0111117C0112339F060E220
:10CA000080E49DE00E9496AE1150F7CF602F80E445
:10CA10009DE00E9496AE60E280E49DE0DF91CF91C0
:10CA20001F910F910C9496AE80E49DE00E9496AE0B
:10CA300021961150DCCFEF92FF920F931F93CF936B
:10CA4000DF93EB01E42E8901F90101900020E9F761
:10CA5000F22EFE1A92E1F90E482F60E080E49DE08C
:10CA60000E94BF286E2D80E49DE00E9496AEFE01DC
:10CA70006491662311F0F11019C06AE380E49DE02F
:10CA80000E9496AEFF2039F060E280E49DE00E94B3
:10CA900096AEFA94F7CFB80180E49DE0DF91CF9194
:10CAA0001F910F91FF90EF900C9495AE80E49DE064
:10CAB0000E9496AE2196FA94DACF1092990D8DE5E8
:10CAC0009AE00E94153A10923E0D08958DE59AE085
:10CAD0000C9477318DE59AE00C947E31CF93DF93FF
:10CAE000CDB7DEB7C054D1090FB6F894DEBF0FBE84
:10CAF000CDBF88E0EFEAF2E0DE01D99601900D9219
:10CB00008A95E1F788E0E7EBF2E0DE01D19601904B
:10CB10000D928A95E1F788E0EFEBF2E0DE0199965D
:10CB200001900D928A95E1F788E0E7ECF2E0DE01F2
:10CB3000919601900D928A95E1F788E0EFECF2E092
:10CB4000DE01599601900D928A95E1F788E0E7EDB4
:10CB5000F2E0DE01519601900D928A95E1F788E0AE
:10CB6000EFEDF2E0DE01199601900D928A95E1F762
:10CB700088E0E7EEF2E0DE01119601900D928A95D1
:10CB8000E1F7AE01475C5F4F60E080E49DE00E940A
:10CB90005D2AAE014F5C5F4F61E080E49DE00E9442
:10CBA0005D2AAE01475D5F4F62E080E49DE00E9438
:10CBB0005D2AAE014F5D5F4F63E080E49DE00E941F
:10CBC0005D2AAE01475E5F4F64E080E49DE00E9415
:10CBD0005D2AAE014F5E5F4F65E080E49DE00E94FC
:10CBE0005D2AAE01475F5F4F66E080E49DE00E94F2
:10CBF0005D2AAE014F5F5F4F67E080E49DE00E94D9
:10CC00005D2AC05CDF4F0FB6F894DEBF0FBECDBF0C
:10CC1000DF91CF910895CF9382E080936F020E94BD
:10CC200008AA6C507E4F8F4F9F4F60933A0D7093C0
:10CC30003B0D80933C0D90933D0D809101018460EC
:10CC400080930101CAE09FB7F8948091020184604B
:10CC5000809302019FBF84E690E00E945BAA9FB789
:10CC6000F894809102018B7F809302019FBF84E63C
:10CC700090E00E945BAAC15031F7CF910895E091F6
:10CC80007002F0917102E817F90771F09093710248
:10CC9000809370024093350D5093360D6093370D9D
:10CCA0007093380D2111B7CF089521E040E050E096
:10CCB000BA01E5CF21E040E050E0BA01E0CF8F9229
:10CCC0009F92AF92BF92CF92DF92EF92FF920F931B
:10CCD0001F93CF93DF938091350D9091360DA091E6
:10CCE000370DB091380D81309048A105B10540F065
:10CCF0001092350D1092360D1092370D1092380D9E
:10CD00006091350D7091360D8091370D9091380DF1
:10CD100025E030E040E050E00E9455B380913E0DA8
:10CD200090E0A0E0B0E0281739074A075B0710F44D
:10CD300020933E0DD0913E0D10913F0D12FB112717
:10CD400010F9C0E085E0C82ED12CE12CF12C9DE13A
:10CD5000892E912CA12CB12C01E06091350D7091A0
:10CD6000360D8091370D9091380DD11131C0209141
:10CD70006F02222369F023E065307105810591057A
:10CD800010F443E001C040E267E071E18C2F1CDE4B
:10CD9000112309F400C18091350D9091360DA091B9
:10CDA000370DB091380D0597A105B10508F0F3C016
:10CDB00032DF83E393E7DF91CF911F910F91FF90D3
:10CDC000EF90DF90CF90BF90AF909F908F906DCFFE
:10CDD000D13061F520916F02222391F0A7019601D5
:10CDE0000E9455B3213031054105510519F423E066
:10CDF00043E002C023E040E266EF70E18C2FE4DD07
:10CE0000112309F4C8C06091350D7091360D8091E1
:10CE1000370D9091380DA70196010E9455B321302E
:10CE200031054105510509F0B6C0C2CFD23061F5D8
:10CE300020916F02222391F0A70196010E9455B321
:10CE4000223031054105510519F423E043E002C0C9
:10CE500023E040E26AEE70E18C2FB6DD112309F485
:10CE60009AC06091350D7091360D8091370D90917B
:10CE7000380DA70196010E9455B3223031054105B6
:10CE8000510509F088C094CFD33061F520916F022D
:10CE9000222391F0A70196010E9455B3233031055A
:10CEA0004105510519F423E043E002C023E040E2CC
:10CEB00068ED70E18C2F88DD112309F46CC060915E
:10CEC000350D7091360D8091370D9091380DA70179
:10CED00096010E9455B3233031054105510509F0F3
:10CEE0005AC066CFD43059F520916F02222391F0B9
:10CEF000A70196010E9455B3243031054105510523
:10CF000019F423E043E002C023E040E266EC70E164
:10CF10008C2F5ADD112309F43EC06091350D7091BC
:10CF2000360D8091370D9091380DA70196010E9422
:10CF300055B3243031054105510569F539CFD53058
:10CF400051F520916F02222391F0A70196010E94D2
:10CF500055B3253031054105510519F423E043E06F
:10CF600002C023E040E26AEB70E18C2F2DDD11233B
:10CF700091F06091350D7091360D8091370D909143
:10CF8000380DA70196010E9455B3253031054105A2
:10CF9000510509F40DCF8091350D9091360DA0917A
:10CFA000370DB091380D4E97A105B10540F0809234
:10CFB000350D9092360DA092370DB092380D6091DC
:10CFC000350D7091360D8091370D9091380DA70178
:10CFD00096010E9455B380913E0D90E00396422F3A
:10CFE00050E0841795074CF48DEF820F80933E0D2F
:10CFF00000936F02DCEFD20FCFEFCF5FDF5FC43063
:10D0000008F4ABCEDF91CF911F910F91FF90EF907D
:10D01000DF90CF90BF90AF909F908F9008958F92A8
:10D020009F92AF92BF92CF92DF92EF92FF920F93B7
:10D030001F93CF93DF938091350D9091360DA09182
:10D04000370DB091380D81309048A105B10540F001
:10D050001092350D1092360D1092370D1092380D3A
:10D060006091350D7091360D8091370D9091380D8E
:10D0700025E030E040E050E00E9455B380913E0D45
:10D0800090E0A0E0B0E0281739074A075B0710F4EA
:10D0900020933E0DD0913E0D10913F0D12FB1127B4
:10D0A00010F9C0E025E0C22ED12CE12CF12C3DE19D
:10D0B000832E912CA12CB12C01E06091350D709143
:10D0C000360D8091370D9091380DD11131C02091DE
:10D0D0006F02222369F023E0653071058105910517
:10D0E00010F443E001C040E265EB70E18C2F6CDC92
:10D0F000112309F429C18091350D9091360DA0912D
:10D10000370DB091380D0597A105B10508F01CC188
:10D1100082DD83E393E7DF91CF911F910F91FF9021
:10D12000EF90DF90CF90BF90AF909F908F90BDCD4C
:10D13000D13079F520916F02222391F0A701960159
:10D140000E9455B3213031054105510519F42EE7F0
:10D150004EE302C02EE740E269EA70E18C2F34DC36
:10D16000112309F4F1C06091350D7091360D809155
:10D17000370D9091380DA70196010E9455B32130CB
:10D1800031054105510509F0DFC045DD8CE79AE71F
:10D1900030C0D230D9F520916F02222391F0A7013F
:10D1A00096010E9455B3223031054105510519F40D
:10D1B0002EE74EE302C02EE740E26FE970E18C2FCC
:10D1C00003DC112309F4C0C06091350D7091360D58
:10D1D0008091370D9091380DA70196010E9455B3AB
:10D1E000223031054105510509F0AEC014DD8DE94D
:10D1F0009BE6DF91CF911F910F91FF90EF90DF9011
:10D20000CF90BF90AF909F908F9054CDD33079F551
:10D2100020916F02222391F0A70196010E9455B33D
:10D22000233031054105510519F420E24EE302C0D7
:10D2300020E240E263E970E18C2FC6DB112309F4A0
:10D2400083C06091350D7091360D8091370D9091AE
:10D25000380DA70196010E9455B3233031054105D1
:10D26000510509F071C0D7DC8DE890E15FC0D43082
:10D2700079F520916F02222391F0A70196010E9477
:10D2800055B3243031054105510519F420E24EE330
:10D2900002C020E240E26CE770E18C2F95DB1123A5
:10D2A00009F452C06091350D7091360D8091370DA3
:10D2B0009091380DA70196010E9455B32430310595
:10D2C0004105510509F040C0A6DC88E790E12EC079
:10D2D000D530D1F520916F02222391F0A70196015C
:10D2E0000E9455B3253031054105510519F420E25E
:10D2F0004EE302C020E240E26EE670E18C2F64DB78
:10D30000112311F16091350D7091360D8091370D1B
:10D310009091380DA70196010E9455B32530310533
:10D320004105510589F477DC8AE690E1DF91CF91E0
:10D330001F910F91FF90EF90DF90CF90BF90AF9033
:10D340009F908F900C94213F8091350D9091360DD8
:10D35000A091370DB091380D4E97A105B10540F061
:10D360008092350D9092360DA092370DB092380D07
:10D370006091350D7091360D8091370D9091380D7B
:10D38000A70196010E9455B380913E0D90E003964F
:10D39000422F50E0841795074CF48DEF820F809355
:10D3A0003E0D00936F02DCEFD20FCFEFCF5FDF5F58
:10D3B000C43008F482CEDF91CF911F910F91FF907E
:10D3C000EF90DF90CF90BF90AF909F908F90089597
:10D3D000BF92CF92DF92EF92FF920F931F93CF9362
:10D3E000DF938091350D9091360DA091370DB0915E
:10D3F000380D81309048A105B10540F01092350DEF
:10D400001092360D1092370D1092380D6091350D37
:10D410007091360D8091370D9091380D25E030E0F8
:10D4200040E050E00E9455B380913E0D90E0A0E0B6
:10D43000B0E0281739074A075B0710F420933E0D28
:10D44000D0913E0D10913F0D12FB112710F9C0E055
:10D4500065E0C62ED12CE12CF12C01E06091350D58
:10D460007091360D8091370D9091380DD1112EC0ED
:10D4700020916F02222369F023E065307105810558
:10D48000910510F443E001C040E261E670E18C2FA9
:10D490009BDA112309F479C08091350D9091360DF6
:10D4A000A091370DB091380D0597A105B10508F091
:10D4B0006CC0B1DB8FE098E6DF91CF911F910F91A7
:10D4C000FF90EF90DF90CF90BF90EFCBD13071F510
:10D4D00020916F02222391F0A70196010E9455B37B
:10D4E000213031054105510519F42EE74EE302C004
:10D4F0002EE740E26AE570E18C2F66DA112309F429
:10D5000044C06091350D7091360D8091370D90912A
:10D51000380DA70196010E9455B321303105410510
:10D52000510599F578DB80EE90E8A8C0D23069F516
:10D5300020916F02222391F0A70196010E9455B31A
:10D54000223031054105510519F42EE74EE302C0A2
:10D550002EE740E263E570E18C2F36DA1123A9F063
:10D560006091350D7091360D8091370D9091380D89
:10D57000A70196010E9455B322303105410551059E
:10D5800021F449DB87EE90E879C020E030E040E20A
:10D5900051E46091110D7091120D8091130D9091D5
:10D5A000140D0E9477AF87FF73C06091350D7091A5
:10D5B000360D8091370D9091380DD33081F5209143
:10D5C0006F02222391F0A70196010E9455B32330E8
:10D5D00031054105510519F42EE74EE302C02EE74F
:10D5E00040E26CE470E18C2FEFD9111103C055E0DB
:10D5F000B52E50C06091350D7091360D8091370D6C
:10D600009091380DA70196010E9455B32330310542
:10D610004105510561F7FFDA8EEE90E82FC0D43056
:10D6200031F720916F02222391F0A70196010E9409
:10D6300055B3243031054105510519F42EE74EE369
:10D6400002C02EE740E263E470E18C2FBDD91123C4
:10D6500071F26091350D7091360D8091370D90917A
:10D66000380DA70196010E9455B3243031054105BC
:10D67000510509F0BCCFCFDA8CE19FE7DF91CF9164
:10D680001F910F91FF90EF90DF90CF90BF9012CB42
:10D6900043E0B42E6091350D7091360D8091370DB9
:10D6A0009091380DA70196010E9455B38B2D90E003
:10D6B000A0E0B0E0281739074A075B0788F025E0AB
:10D6C000B29EC00111240197AA2797FDA095BA2FF9
:10D6D0008093350D9093360DA093370DB093380D90
:10D6E0006091350D7091360D8091370D9091380D08
:10D6F000A70196010E9455B380913E0D90E00396DC
:10D70000422F50E0841795074CF48DEF820F8093E1
:10D710003E0D00936F02DCEFD20FCFEFCF5FDF5FE4
:10D72000C43008F49BCEDF91CF911F910F91FF90F1
:10D73000EF90DF90CF90BF90089580E090E0A0E858
:10D74000BFE38093110D9093120DA093130DB0932E
:10D75000140D3ECE20E044E064E180E49DE00E94B0
:10D76000F228BCD980E49DE00C94B328F3DF20E0DC
:10D7700040E050E0BA0185EF90E881CA1092490874
:10D7800010924808109247081092460810922F0AEB
:10D7900010922E0AEBCF80E49DE00C94B32820E099
:10D7A00030E04EE353E4609140087091410880916D
:10D7B0004208909143080E947AB118164CF481E017
:10D7C0009FE00E94213F84EF9EE00E94213F20C005
:10D7D000E2DF40E060E080E49DE00E94BF286BEC67
:10D7E00074E080E49DE00E9495AE42E060E080E459
:10D7F0009DE00E94BF2862ED74E080E49DE00E94FD
:10D8000095AE60ED77E080E090E00E9437AAC3DF3C
:10D81000ADCF20E030E04EE353E4609140087091DA
:10D82000410880914208909143080E947AB11816ED
:10D830006CF480EF9EE00E94213F84EE9EE00E9407
:10D84000213F88ED9EE00E94213F20C0A4DF40E000
:10D8500060E080E49DE00E94BF286BEC74E080E40F
:10D860009DE00E9495AE42E060E080E49DE00E9471
:10D87000BF2862ED74E080E49DE00E9495AE60ED0B
:10D8800077E080E090E00E9437AA85DF6FCF80913B
:10D89000970D9091980D9093490880934808809136
:10D8A000950D9091960D909347088093460810929D
:10D8B0002F0A10922E0A5ADF0C9485218091910D27
:10D8C0009091920D909349088093480880918F0D14
:10D8D0009091900D909347088093460810922F0ADC
:10D8E00010922E0A43DF0C9485218091950290912D
:10D8F00096029093490880934808809193029091F2
:10D900009402909347088093460810922F0A109231
:10D910002E0A2CDF0C948521809191029091920225
:10D92000909349088093480880918F0290919002CB
:10D93000909347088093460810922F0A10922E0A5F
:10D9400015DF0C94852180918D0290918E02909329
:10D9500049088093480880918B0290918C029093A3
:10D9600047088093460810922F0A10922E0AFEDE76
:10D970000C9485218091890290918A0290934908A4
:10D98000809348088091870290918802909347087D
:10D990008093460810922F0A10922E0AE7DE0C940C
:10D9A00085212F923F924F925F926F927F928F923A
:10D9B0009F92AF92BF92CF92DF92EF92FF920F931E
:10D9C0001F93CF93DF93CDB7DEB7A6970FB6F8942A
:10D9D000DEBF0FBECDBF80916F02811104C0809168
:10D9E0003F0D82FFC4C28DE59AE00E9409398C0187
:10D9F0008091350D9091360DA091370DB091380D75
:10DA000081309048A105B10540F01092350D10927B
:10DA1000360D1092370D1092380D6091350D7091C2
:10DA2000360D8091370D9091380D25E030E040E0C3
:10DA300050E00E9455B380913E0D90E0A0E0B0E030
:10DA4000281739074A075B0710F420933E0D2090F2
:10DA50003E0D80913F0D82FB882780F98F8F312CFE
:10DA600085E0C82ED12CE12CF12CC80101979BA395
:10DA70008AA321102DC080916F028823A9F0809184
:10DA8000350D9091360DA091370DB091380D23E0F2
:10DA90000597A105B10510F443E001C040E26CEF29
:10DAA0007FE0832D0E94E4649F8D992389F080910B
:10DAB000350D9091360DA091370DB091380D059729
:10DAC000A105B10528F4A7D883E393E7EED84FC2A8
:10DAD00061E67AE08BEC9AE00E9481108091610A05
:10DAE0008F3229F0E1E02E1669F012E001C011E05A
:10DAF000AAA0BBA0422C512C612C712CF1E0F20D9C
:10DB0000F8A351C080916F028823D9F06091350D40
:10DB10007091360D8091370D9091380DA7019601C7
:10DB20000E9455B3213031054105510519F420E219
:10DB30004EE302C020E240E268EF7FE0832D0E94C6
:10DB4000E4642F8D222389F26091350D7091360D9A
:10DB50008091370D9091380DA70196010E9455B321
:10DB6000213031054105510509F0BFCF54D80E943D
:10DB70005D65FDC1121163C140E050E0B5018DE566
:10DB80009AE00E9480359091A30A80916F029923B8
:10DB900009F49EC081110CC08F8D811176C018A12F
:10DBA000F1E0AF1AB1082FEFA216B20619F749C17A
:10DBB0006091350D7091360D8091370D9091380D33
:10DBC000A70196010E9455B3241535054605570552
:10DBD00071F5432D60E080E49DE00E94BF286EE374
:10DBE00080E49DE00E9496AE65E080E49DE00E94A6
:10DBF00096AE80916E0A882329F01092800A0EE674
:10DC00001AE002C001E61AE0B2E19B2EF801619130
:10DC10008F01662311F0911062C1992009F4BCCFE5
:10DC200060E280E49DE00E9496AE9A94F6CF432D88
:10DC300060E080E49DE00E94BF2860E280E49DE017
:10DC40000E9496AE65E080E49DE00E9496AE8091D1
:10DC50006E0A882329F01092800A0EE61AE002C0AC
:10DC600001E61AE0A2E19A2EF80161918F01662384
:10DC700011F091103AC1992009F48ECF60E280E44E
:10DC80009DE00E9496AE9A94F6CF6091350D70910A
:10DC9000360D8091370D9091380DA70196010E94A5
:10DCA00055B3241535054605570509F078CF0E9470
:10DCB0000B6661E67AE08DE59AE00E946C3910927D
:10DCC000350D1092360D1092370D1092380D4FC150
:10DCD000811104C0FF8DF1116FC061CF6091350DCE
:10DCE0007091360D8091370D9091380DA7019601F6
:10DCF0000E9455B32415350546055705A1F5209119
:10DD00009B0D29A310E0412F60E080E49DE00E947C
:10DD1000BF2860E280E49DE00E9496AE1F5F143051
:10DD200091F7432D60E080E49DE00E94BF286EE300
:10DD300080E49DE00E9496AE2FE63AE0FEE68F2E4C
:10DD4000FAE09F2E01E010E0F40151914F015111D2
:10DD5000D2C014E1101B60E280E49DE00E9496AE08
:10DD60001150C9F7B7CF432D60E080E49DE00E94D9
:10DD7000BF2860E280E49DE00E9496AE80916E0A2A
:10DD8000882329F01092810A0EE61AE002C001E60B
:10DD90001AE0E3E19E2EF80161918F01662311F0F4
:10DDA0009110DFC0992009F495CF60E280E49DE0F6
:10DDB0000E9496AE9A94F6CF6091350D7091360D13
:10DDC0008091370D9091380DA70196010E9455B3AF
:10DDD000241535054605570509F0E1CE0E940B666E
:10DDE00081E69AE09F938F9381EF9FE09F938F93BB
:10DDF0008E010F5F1F4F1F930F930E9432B70F903A
:10DE00000F900F900F900F900F907E01F5E0EF0EA6
:10DE1000F11CF7018081882349F0992787FD9095AF
:10DE20000E946FB6F70181937F01F3CFC8010E9472
:10DE3000AE3E8DEE9FE00E94213F98DC98C01F5FB0
:10DE4000AFCE6091350D7091360D8091370D909168
:10DE5000380DA70196010E9455B3812F90E0A0E0F4
:10DE6000B0E0281739074A075B0788F0E5E01E9FF6
:10DE7000C00111240197AA2797FDA095BA2F80937E
:10DE8000350D9093360DA093370DB093380D6091FA
:10DE9000350D7091360D8091370D9091380DA70199
:10DEA00096010E9455B380913E0D90E00396422F5B
:10DEB00050E08417950764F48DEF820F80933E0D38
:10DEC00081E080936F027CEF272E220E33243A9458
:10DED00033942394F3E0F31508F0CBCD48C080E4ED
:10DEE0009DE00E9496AE9A9491CE80E49DE00E94BF
:10DEF00096AE9A94B9CE432D602F80E49DE02DA379
:10DF00003EA35CA30E94BF285CA1652F80E49DE036
:10DF10000E9496AE0F5F1F4F2DA13EA10431110547
:10DF200009F012CF49010CE211E080913F0D82FD12
:10DF300005C080919B0D99A1981741F001501109DE
:10DF40000115110591F72F5F3F4FFCCE61E070E0A6
:10DF500080E090E02DA33EA30E9437AA2DA13EA110
:10DF6000EDCF80E49DE00E9496AE9A9414CFA696E1
:10DF70000FB6F894DEBF0FBECDBFDF91CF911F91DA
:10DF80000F91FF90EF90DF90CF90BF90AF909F9058
:10DF90008F907F906F905F904F903F902F9008955B
:10DFA0008F929F92AF92BF92CF92DF92EF92FF92A9
:10DFB0000F931F93CF93DF938091350D9091360D82
:10DFC000A091370DB091380D81309048A105B10571
:10DFD00040F01092350D1092360D1092370D1092C0
:10DFE000380D6091350D7091360D8091370D9091FF
:10DFF000380D25E030E040E050E00E9455B38091BC
:10E000003E0D90E0A0E0B0E0281739074A075B0713
:10E0100010F420933E0DD0913E0D10913F0D12FB58
:10E02000112710F9C0E095E0C92ED12CE12CF12C7C
:10E0300027E2822E912CA12CB12C01E06091350DAC
:10E040007091360D8091370D9091380DD11134C0FB
:10E0500020916F02222371F023E065307105810564
:10E06000910510F443E001C040E268ED7FE08C2FA1
:10E070000E94E464112309F4C8C18091350D909188
:10E08000360DA091370DB091380D0597A105B1055A
:10E0900008F0BBC10E940B6683E393E7DF91CF9149
:10E0A0001F910F91FF90EF90DF90CF90BF90AF90B6
:10E0B0009F908F900C945566D130D9F520916F02C6
:10E0C000222399F0A70196010E9455B32130310512
:10E0D0004105510519F420E24EE302C020E240E27E
:10E0E00068EC7FE08C2F0E94E464112309F48DC159
:10E0F0006091350D7091360D8091370D9091380DEE
:10E10000A70196010E9455B3213031054105510503
:10E1100009F07BC10E940B66DF91CF911F910F9197
:10E12000FF90EF90DF90CF90BF90AF909F908F9037
:10E13000C5CBD230D9F520916F02222399F0A701E7
:10E1400096010E9455B3223031054105510519F45D
:10E1500020E24EE302C020E240E269EB7FE08C2F38
:10E160000E94E464112309F450C16091350D70914F
:10E17000360D8091370D9091380DA70196010E94C0
:10E1800055B3223031054105510509F03EC10E94C9
:10E190000B66DF91CF911F910F91FF90EF90DF9071
:10E1A000CF90BF90AF909F908F9071CBD330D9F527
:10E1B00020916F02222399F0A70196010E9455B386
:10E1C000233031054105510519F420E24EE302C028
:10E1D00020E240E26AEA7FE08C2F0E94E46411238F
:10E1E00009F413C16091350D7091360D8091370D92
:10E1F0009091380DA70196010E9455B32330310547
:10E200004105510509F001C10E940B66DF91CF91D4
:10E210001F910F91FF90EF90DF90CF90BF90AF9044
:10E220009F908F9079CBD430D9F520916F02222323
:10E2300099F0A70196010E9455B32430310541059C
:10E24000510519F420E24EE302C020E240E26AE9FF
:10E250007FE08C2F0E94E464112309F4D6C0609102
:10E26000350D7091360D8091370D9091380DA701C5
:10E2700096010E9455B3243031054105510509F03E
:10E28000C4C00E940B66DF91CF911F910F91FF9048
:10E29000EF90DF90CF90BF90AF909F908F9053CB37
:10E2A000D530D9F520916F02222399F0A70196016C
:10E2B0000E9455B3253031054105510519F420E27E
:10E2C0004EE302C020E240E26AE87FE08C2F0E9429
:10E2D000E464112309F499C06091350D7091360DF5
:10E2E0008091370D9091380DA70196010E9455B38A
:10E2F000253031054105510509F087C00E940B66A4
:10E30000DF91CF911F910F91FF90EF90DF90CF9011
:10E31000BF90AF909F908F90E8CAD630D9F52091EA
:10E320006F02222399F0A70196010E9455B326306F
:10E3300031054105510519F420E24EE302C020E207
:10E3400040E26BE77FE08C2F0E94E464112309F424
:10E350005CC06091350D7091360D8091370D9091B4
:10E36000380DA70196010E9455B3263031054105AD
:10E37000510509F04AC00E940B66DF91CF911F91B1
:10E380000F91FF90EF90DF90CF90BF90AF909F9054
:10E390008F90F0CAD730C9F520916F02222399F0EF
:10E3A000A70196010E9455B327303105410551055B
:10E3B00019F420E24EE302C020E240E262E77FE08F
:10E3C0008C2F0E94E464112301F16091350D70914E
:10E3D000360D8091370D9091380DA70196010E945E
:10E3E00055B3273031054105510579F40E940B667C
:10E3F000DF91CF911F910F91FF90EF90DF90CF9021
:10E40000BF90AF909F908F90B9C98091350D90913A
:10E41000360DA091370DB091380D8897A105B10543
:10E4200040F08092350D9092360DA092370DB0924B
:10E43000380D6091350D7091360D8091370D9091AA
:10E44000380DA70196010E9455B380913E0D90E0D2
:10E450000396422F50E0841795074CF48DEF820FFE
:10E4600080933E0D00936F02DCEFD20FCFEFCF5FB2
:10E47000DF5FC43008F4E2CDDF91CF911F910F919F
:10E48000FF90EF90DF90CF90BF90AF909F908F90D4
:10E49000089581D941E060E080E49DE00E94BF28BA
:10E4A00069EF74E080E49DE00E9495AE42E060E098
:10E4B00080E49DE00E94BF2869E075E080E49DE073
:10E4C0000C9495AE68D942E060E080E49DE00E9443
:10E4D000BF286CE175E080E49DE00C9495AE1F933D
:10E4E000CF93DF9358D940E060E080E49DE00E9444
:10E4F000BF286CE275E080E49DE00E9495AE42E0AA
:10E5000060E080E49DE00E94BF286AE375E080E45B
:10E510009DE00E9495AE10E043E0612F80E49DE015
:10E520000E94BF286FE573E080E49DE00E9495AEF5
:10E53000CAE0D0E00E94B31E81E00E94264A65E551
:10E5400070E080E090E00E9437AA2197209791F731
:10E550001F5F143109F7DF91CF911F9108951F9329
:10E56000CF93DF9318D940E060E080E49DE00E9403
:10E57000BF2866E475E080E49DE00E9495AE42E02D
:10E5800060E080E49DE00E94BF286AE375E080E4DB
:10E590009DE00E9495AE10E043E0612F80E49DE095
:10E5A0000E94BF286FE573E080E49DE00E9495AE75
:10E5B000CAE0D0E00E94B31E81E00E94264A6EE6C7
:10E5C00070E080E090E00E9437AA2197209791F7B1
:10E5D0001F5F143109F7DF91CF911F910895809348
:10E5E0002E0D10922D0D0895E2E7F2E0019000202B
:10E5F000E9F73197E257F2401E161F0634F01092E9
:10E60000860282E080936F02089580E2E431F10592
:10E61000B4F7DF01AE58BD4F8C933196F7CF209100
:10E620008C0D211108C044E150E0BC0182E792E06A
:10E630000E9423B7D9CF089510925F0A60E08DE55C
:10E640009AE00E946B350E948A9481EE9FE00E94BE
:10E65000213F81E080931F0A87E595E0E0DF8DEDA3
:10E660009FE00C94213FAF92BF92CF92DF92EF9246
:10E67000FF920F931F93CF93DF931092990D809188
:10E68000350D9091360DA091370DB091380D813038
:10E690009048A105B10540F01092350D1092360D4D
:10E6A0001092370D1092380D6091350D7091360D26
:10E6B0008091370D9091380D25E030E040E050E03A
:10E6C0000E9455B380913E0D90E0A0E0B0E0281785
:10E6D00039074A075B0710F420933E0DD0913E0D99
:10E6E00010913F0D12FB112710F9C0E045E0C42E38
:10E6F000D12CE12CF12CAA24A394D11137C0809104
:10E700006F028823A9F08091350D9091360DA0916C
:10E71000370DB091380D23E00597A105B10510F430
:10E7200043E001C040E265E871E18C2F0E94E4649F
:10E730001123E1F08091350D9091360DA091370DA8
:10E74000B091380D0597A105B10580F40E940B66C4
:10E7500085EF90E8DF91CF911F910F91FF90EF909F
:10E76000DF90CF90BF90AF900C9455660E94D7A5D4
:10E770004091350D5091360D6091370D7091380DE7
:10E78000811104C080915F0A882399F1D130C9F5C5
:10E7900080916F028823A9F0CB01BA01A7019601ED
:10E7A0000E9455B3213031054105510519F42EE77A
:10E7B0004EE302C02EE740E260E871E18C2F0E9438
:10E7C000E4641123F1F06091350D7091360D809164
:10E7D000370D9091380DA70196010E9455B3213055
:10E7E00031054105510569F40E940B6683E39CE7FE
:10E7F0003EC2D13031F480916F0281119BC2111160
:10E80000AFC22091600A6091350D7091360D8091F4
:10E81000370D9091380D222309F4F1C02091480C56
:10E82000222309F4B9C020915F0A2223E9F1D230F2
:10E8300009F076C020916F02222399F0A70196017A
:10E840000E9455B3223031054105510519F420E2EB
:10E850004EE302C020E240E26CE671E18C2F0E94A0
:10E86000E464112309F4E2C06091350D7091360D16
:10E870008091370D9091380DA70196010E9455B3F4
:10E88000223031054105510509F0D0C00E940B66C8
:10E89000DF91CF911F910F91FF90EF90DF90CF907C
:10E8A000BF90AF900C946A65D230D1F520916F0281
:10E8B000222399F0A70196010E9455B32230310519
:10E8C0004105510519F420E24EE302C020E240E286
:10E8D0006FE571E18C2F0E94E464112309F4A6C056
:10E8E0006091350D7091360D8091370D9091380DF6
:10E8F000A70196010E9455B322303105410551050B
:10E9000009F094C00E940B66DF91CF911F910F9187
:10E91000FF90EF90DF90CF90BF90AF900C94666522
:10E92000D33009F083C020916F02222399F0A70110
:10E9300096010E9455B3233031054105510519F464
:10E9400020E24EE302C020E240E264E571E18C2F58
:10E950000E94E464112309F469C06091350D70913F
:10E96000360D8091370D9091380DA70196010E94C8
:10E9700055B3233031054105510509F057C00E94B8
:10E980000B66DF91CF911F910F91FF90EF90DF9079
:10E99000CF90BF90AF9050CED23011F003E047C07F
:10E9A00020916F02222399F0A70196010E9455B38E
:10E9B000223031054105510519F42EE74EE302C01E
:10E9C0002EE740E266E471E18C2F0E94E46411239B
:10E9D00029F36091350D7091360D8091370D90912E
:10E9E000380DA70196010E9455B32230310541052B
:10E9F0005105A1F60E940B6681ED9CE638C1D2302C
:10EA000069F620916F02222311F3A70196010E945B
:10EA100055B3223031054105510519F42EE74EE377
:10EA200002C02EE740E26BE371E1CECF04E08091BB
:10EA30005F0A8111DCC00D1348C080916F028823EA
:10EA4000F9F06091350D7091360D8091370D9091F0
:10EA5000380DA70196010E9455B3802F90E0A0E0E9
:10EA6000B0E0281739074A075B0719F420E24EE3A4
:10EA700002C020E240E26DE271E18C2F0E94E4646A
:10EA8000112319F16091350D7091360D8091370D7C
:10EA90009091380DA70196010E9455B3802F90E008
:10EAA000A0E0B0E0281739074A075B0771F40E941D
:10EAB0000B66DF91CF911F910F91FF90EF90DF9048
:10EAC000CF90BF90AF900C94096CBB24B394B00E60
:10EAD000BD1248C080916F028823F9F06091350D16
:10EAE0007091360D8091370D9091380DA7019601E8
:10EAF0000E9455B38D2F90E0A0E0B0E028173907B1
:10EB00004A075B0719F420E24EE302C020E240E22C
:10EB10006DE171E18C2F0E94E464112319F1609181
:10EB2000350D7091360D8091370D9091380DA701FC
:10EB300096010E9455B38B2D90E0A0E0B0E028171D
:10EB400039074A075B0771F40E940B66DF91CF918A
:10EB50001F910F91FF90EF90DF90CF90BF90AF90FB
:10EB60000C94CF6B32E0B32EB00EBD123FC080913B
:10EB70006F028823F9F06091350D7091360D809108
:10EB8000370D9091380DA70196010E9455B38D2F36
:10EB900090E0A0E0B0E0281739074A075B0719F4B6
:10EBA0002EE74EE302C02EE740E264E171E18C2FD4
:10EBB0000E94E4641123D1F06091350D7091360DFF
:10EBC0008091370D9091380DA70196010E9455B3A1
:10EBD0008B2D90E0A0E0B0E0281739074A075B07CB
:10EBE00029F40E940B668FE098E641C00D5F0D137B
:10EBF0004AC080916F028823F9F06091350D7091C1
:10EC0000360D8091370D9091380DA70196010E9425
:10EC100055B3802F90E0A0E0B0E0281739074A07ED
:10EC20005B0719F42EE74EE302C02EE740E26CE0EA
:10EC300071E18C2F0E94E464112329F16091350D5C
:10EC40007091360D8091370D9091380DA701960186
:10EC50000E9455B3802F90E0A0E0B0E0281739075C
:10EC60004A075B0781F40E940B668FE596E6DF9109
:10EC7000CF911F910F91FF90EF90DF90CF90BF90B9
:10EC8000AF900C945A66BB24B394B00E6091350DCE
:10EC90007091360D8091370D9091380DA701960136
:10ECA0000E9455B38B2D90E0A0E0B0E02817390703
:10ECB0004A075B0788F025E0B29EC0011124019746
:10ECC000AA2797FDA095BA2F8093350D9093360D06
:10ECD000A093370DB093380D6091350D7091360DBE
:10ECE0008091370D9091380DA70196010E9455B380
:10ECF00080913E0D90E00396422F50E084179507D7
:10ED00004CF48DEF820F80933E0DA0926F02DCEFEA
:10ED1000D20FCFEFCF5FDF5FC43008F4EECCDF91CE
:10ED2000CF911F910F91FF90EF90DF90CF90BF9008
:10ED3000AF900895CB01BA01A70196010E9455B387
:10ED4000213031054105510519F42EE74EE302C08B
:10ED50002EE740E268E771E18C2F0E94E4644FCD1A
:10ED60006091350D7091360D8091370D9091380D71
:10ED7000A70196010E9455B3213031054105510587
:10ED800009F03FCD0E940B6680ED9FE670CF209189
:10ED90008C0D211108C044E150E0BC0182E792E0F3
:10EDA0000E9496B621CC0895F2DF81E080938C0D0D
:10EDB0000C94B66B10928C0D0895CF92DF92EF9267
:10EDC000FF92CF93C0910301C2FBCC27C0F981E031
:10EDD000C8278091030181FFC260C0903A0DD09096
:10EDE0003B0DE0903C0DF0903D0D0E9408AAC61628
:10EDF000D706E806F90620F48091000186FF39C0A5
:10EE0000C0933F0D80913F0D817090913F0D91FD1A
:10EE100082609091390D891721F18130F1F028F04D
:10EE2000823089F08330A1F01CC0913021F49091A0
:10EE30009B0D9F5F05C09230A1F490919B0D915066
:10EE400090939B0D0EC0992391F3933051F4F5CF1D
:10EE5000923069F3913029F4F0CF933041F3992344
:10EE600061F38093390DCF91FF90EF90DF90CF90B9
:10EE70000895C460C5CF0E94AA6BE4E0F1E08081F0
:10EE80008B7F808380818D7F80839FB7F894E5E0BE
:10EE9000F1E08081846080839FBF9FB7F894808178
:10EEA000826080839FBFE1E0F1E080818F7B80837F
:10EEB0009FB7F894E2E0F1E08081806480839FBF97
:10EEC00060E08FE00E9428A99FB7F894E5E0F1E0A8
:10EED0008081816080839FBF8091030180958170D4
:10EEE0008093340D6ADF10929B0D0895CF92DF92CC
:10EEF000EF92FF9262DF80910301817091E0892798
:10EF00002091340D8217B9F082E080936F028091D6
:10EF10000301817089278093340D0E94AA6B809130
:10EF2000340D882309F490C08DE59AE00E94A83042
:10EF30008AEC9EE02CDFC090300DD090310DE09037
:10EF4000320DF090330D0E9408AAC616D706E806C7
:10EF5000F90608F086C040919B0D442361F181E0E1
:10EF600080936F02552747FD5095652F752F80912F
:10EF7000350D9091360DA091370DB091380D840F5D
:10EF8000951FA61FB71F8093350D9093360DA09344
:10EF9000370DB093380D10929B0D0E9408AA685649
:10EFA000754C8F4F9F4F6093050D7093060D8093A6
:10EFB000070D9093080D80913F0D82FF0EC00E94B7
:10EFC00008AA6856754C8F4F9F4F6093050D70933C
:10EFD000060D8093070D9093080DE0917002F0915B
:10EFE00071021995C090050DD090060DE090070DA7
:10EFF000F090080D0E9408AAC616D706E806F90682
:10F0000038F48091700290917102855F904819F5F3
:10F0100080916F02823011F40E94CB6B80916F025D
:10F02000882319F0815080936F020E9408AA6C59BE
:10F030007F4F8F4F9F4F6093300D7093310D8093B2
:10F04000320D9093330D0DC08DE59AE00E9473311F
:10F050008DEB9EE06FCF0E94B66B82E080936F02D3
:10F06000D7CFFF90EF90DF90CF90089581E0089583
:10F0700080913F0D82FB882780F908950F931F939D
:10F08000CF93DF930E94CB6B40E060E080E49DE093
:10F090000E94BF2865E675E080E49DE00E9495AE81
:10F0A00041E061E080E49DE00E94BF2868E775E0F0
:10F0B00080E49DE00E9495AE42E061E080E49DE046
:10F0C0000E94BF286CE775E080E49DE00E9495AE49
:10F0D00043E061E080E49DE00E94BF2860E975E0C4
:10F0E00080E49DE00E9495AE41E060E080E49DE018
:10F0F0000E94BF2860EA75E080E49DE00E9495AE22
:10F1000000919B0D112707FD1095C1E0D0E0809183
:10F11000550A9091560A892B09F071C00E94B31EBE
:10F1200081E00E94264A20919B0D332727FD3095D0
:10F13000C801821B930B97FF03C09195819591099C
:10F1400005970CF44DC0201731070CF421970217D6
:10F1500013070CF42196C430D1052CF4209729F420
:10F16000C1E0D0E002C0C3E0D0E041E060E080E474
:10F170009DE00E94BF2861E973E080E49DE00E9469
:10F1800095AE42E060E080E49DE00E94BF2861E926
:10F1900073E080E49DE00E9495AE43E060E080E48F
:10F1A0009DE00E94BF2861E973E080E49DE00E9439
:10F1B00095AE4C2F60E080E49DE00E94BF2860EA9D
:10F1C00075E080E49DE00E9495AE00919B0D1127B3
:10F1D00007FD109564E670E080E090E00E9437AA99
:10F1E00047DF882309F493CFD093560AC093550A7A
:10F1F00064EF71E080E090E00E9437AA88CF0E941F
:10F20000CB6BDF91CF911F910F910C94B66BFC01EA
:10F21000808190E02AE030E0B9010E9442B3482F9B
:10F22000CB01B9010E9442B3805D8093090D405D1E
:10F2300040930A0D10920B0D89E09DE0089520E0A7
:10F2400030E040E251E4FC01608171818281938170
:10F250000E944CB20E94E6AF77FD02C02BE201C0D3
:10F260002DE22093090D9B0177FF04C0222733274D
:10F27000261B370BC90168EE73E00E9442B3CB0135
:10F28000EAE0F0E0BF010E9442B3805D80930A0D86
:10F29000C90164E670E00E9442B3CB01BF010E9445
:10F2A00042B3805D80930B0DC901BF010E9442B340
:10F2B000282FCB01BF010E9442B3805D80930C0DCB
:10F2C0008EE280930D0D205D20930E0D10920F0D98
:10F2D00089E09DE008958F929F92AF92BF92CF9266
:10F2E000DF92EF92FF92FC0180809180A280B38038
:10F2F00020E030E048EC52E4C501B4010E944CB279
:10F300006B017C0120E030E0A9010E947AB118165F
:10F310001CF4C701B60103C0C701B60190580E9492
:10F32000E6AF6B017C0120E030E0A901C501B4012A
:10F330000E9477AF87FF12C08DE28093090DC7014D
:10F34000B60128EE33E040E050E00E9477B3CA01F6
:10F35000B9012AE030E040E050E036C0C701B60114
:10F3600020E137E240E050E00E9477B3AAE08A2E25
:10F37000912CA12CB12CCA01B901A50194010E94C4
:10F3800077B3662391F0605D6093090DC701B60104
:10F3900028EE33E040E050E00E9477B3CA01B901A3
:10F3A000A50194010E9477B313C080E28093090DF8
:10F3B000C701B60128EE33E040E050E00E9477B389
:10F3C000CA01B901A50194010E9477B3662311F027
:10F3D000605D01C060E260930A0DC701B60124E6DA
:10F3E00030E040E050E00E9477B3FAE08F2E912C9D
:10F3F000A12CB12CCA01B901A50194010E9477B3D7
:10F40000605D60930B0DC701B601A50194010E94D8
:10F4100077B3662381F0605D60930E0DCA01B90178
:10F42000A50194010E9477B3605D60930D0D8EE29B
:10F4300080930C0D15C0CA01B901A50194010E9469
:10F4400077B3662329F0605D60930D0D8EE203C0F3
:10F4500080E280930D0D80930C0D80E280930E0D61
:10F4600010920F0D89E09DE0FF90EF90DF90CF901C
:10F47000BF90AF909F908F900895FC0120813181C3
:10F4800037FF07C08DE28093090D31952195310931
:10F4900014C02436310574F0C90164E670E00E949E
:10F4A00042B3CB016AE070E00E9442B3805D80937A
:10F4B000090D06C080E28093090D2A30310564F001
:10F4C000EAE0F0E0C901BF010E9442B3CB01BF01F5
:10F4D0000E9442B3805D01C080E280930A0DC901A1
:10F4E0006AE070E00E9442B3805D80930B0D109241
:10F4F0000C0D89E09DE008958F929F92AF92BF928C
:10F50000CF92DF92EF92FF920F931F93CF93DF93EF
:10F510006091140270911502809116029091170269
:10F520000E94FE276093190D70931A0D80931B0D96
:10F5300090931C0D60911002709111028091120243
:10F54000909113020E940A286093150D7093160D76
:10F550008093170D9093180D8091350D9091360D75
:10F56000A091370DB091380D81309048A105B105BB
:10F5700040F01092350D1092360D1092370D10920A
:10F58000380D6091350D7091360D8091370D909149
:10F59000380D25E030E040E050E00E9455B3809106
:10F5A0003E0D90E0A0E0B0E0281739074A075B075E
:10F5B00010F420933E0DD0913E0D10913F0D12FBA3
:10F5C000112710F9C0E0B5E0CB2ED12CE12CF12CA5
:10F5D00003E1802E912CA12CB12C01E06091350D1E
:10F5E0007091360D8091370D9091380DD11134C046
:10F5F00020916F02222371F023E0653071058105AF
:10F60000910510F443E001C040E26BE270E18C2F01
:10F610000E94E464112309F4E2C08091350D9091B9
:10F62000360DA091370DB091380D0597A105B105A4
:10F6300008F0D5C00E940B668FE098E6DF91CF916D
:10F640001F910F91FF90EF90DF90CF90BF90AF9000
:10F650009F908F900C945566D130D9F520916F0210
:10F660002223B9F0A70196010E9455B388E498E0DF
:10F67000213031054105510521F4FFDE9C014EE3A7
:10F6800003C0FBDE9C0140E264E270E18C2F0E942B
:10F690001B65112309F4A3C06091350D7091360DDF
:10F6A0008091370D9091380DA70196010E9455B3B6
:10F6B000213031054105510509F091C00E940B66CA
:10F6C00023E331E040E050E068E478E08DE190E150
:10F6D00078C0D230D9F520916F022223B9F0A7016A
:10F6E00096010E9455B386E498E022303105410529
:10F6F000510521F4C2DE9C014EE303C0BEDE9C0135
:10F7000040E269E170E18C2F0E941B65112309F42E
:10F7100066C06091350D7091360D8091370D9091D6
:10F72000380DA70196010E9455B3223031054105DD
:10F73000510509F054C00E940B6623E930E040E017
:10F7400050E066E478E085E190E13BC0D33009F019
:10F7500046C020916F022223B9F0A70196010E94B2
:10F7600055B38EE29AE0233031054105510521F46D
:10F7700084DE9C014EE303C080DE9C0140E26BE02E
:10F7800070E18C2F0E941B65112349F16091350DAA
:10F790007091360D8091370D9091380DA70196012B
:10F7A0000E9455B32330310541055105C1F40E9433
:10F7B0000B662FEF30E040E050E06EE27AE081E04F
:10F7C00090E1DF91CF911F910F91FF90EF90DF902B
:10F7D000CF90BF90AF909F908F900C949264809147
:10F7E000350D9091360DA091370DB091380D44979D
:10F7F000A105B10540F08092350D9092360DA09292
:10F80000370DB092380D6091350D7091360D8091A5
:10F81000370D9091380DA70196010E9455B3809144
:10F820003E0D90E00396422F50E0841795074CF46C
:10F830008DEF820F80933E0D00936F02DCEFD20FAD
:10F84000CFEFCF5FDF5FC43008F4C8CEDF91CF9138
:10F850001F910F91FF90EF90DF90CF90BF90AF90EE
:10F860009F908F9008958F929F92AF92BF92CF9268
:10F87000DF92EF92FF920F931F93CF93DF938091CC
:10F88000350D9091360DA091370DB091380D813026
:10F890009048A105B10540F01092350D1092360D3B
:10F8A0001092370D1092380D6091350D7091360D14
:10F8B0008091370D9091380D25E030E040E050E028
:10F8C0000E9455B380913E0D90E0A0E0B0E0281773
:10F8D00039074A075B0710F420933E0DD0913E0D87
:10F8E00010913F0D12FB112710F9C0E085E0C82EE2
:10F8F000D12CE12CF12C92E2892E912CA12CB12C4F
:10F9000001E06091350D7091360D8091370D909129
:10F91000380DD11134C020916F02222371F023E001
:10F92000653071058105910510F443E001C040E2A6
:10F930006DE67FE08C2F0E94E464112309F49CC1E2
:10F940008091350D9091360DA091370DB091380D05
:10F950000597A105B10508F08FC10E940B6683E3EE
:10F9600093E7DF91CF911F910F91FF90EF90DF9080
:10F97000CF90BF90AF909F908F900C945566D130F0
:10F98000D9F520916F022223B9F0A70196010E94B8
:10F9900055B38DE592E0213031054105510521F443
:10F9A0006CDD9C014EE303C068DD9C0140E267E62C
:10F9B0007FE08C2F0E941B65112309F45DC16091CB
:10F9C000350D7091360D8091370D9091380DA7014E
:10F9D00096010E9455B3213031054105510509F0CA
:10F9E0004BC10E940B6627EE33E04AE050E06DE524
:10F9F00072E081E69FE03DC0D23009F048C020911E
:10FA00006F022223B9F0A70196010E9455B388E442
:10FA100098E0223031054105510521F42EDD9C018D
:10FA20004EE303C02ADD9C0140E26AE57FE08C2FB3
:10FA30000E941B65112309F41FC16091350D70915F
:10FA4000360D8091370D9091380DA70196010E94D7
:10FA500055B3223031054105510509F00DC10E9411
:10FA60000B6623E331E040E050E068E478E083E5B2
:10FA70009FE0DF91CF911F910F91FF90EF90DF906A
:10FA8000CF90BF90AF909F908F900C949264D330A2
:10FA9000D9F520916F022223B9F0A70196010E94A7
:10FAA00055B386E498E0233031054105510521F432
:10FAB000E4DC9C014EE303C0E0DC9C0140E26FE427
:10FAC0007FE08C2F0E941B65112309F4D5C0609143
:10FAD000350D7091360D8091370D9091380DA7013D
:10FAE00096010E9455B3233031054105510509F0B7
:10FAF000C3C00E940B6623E930E040E050E066E4BA
:10FB000078E08BE49FE0B5CFD430D9F520916F0237
:10FB10002223B9F0A70196010E9455B38EE29AE024
:10FB2000243031054105510521F4A7DC9C014EE349
:10FB300003C0A3DC9C0140E261E47FE08C2F0E94C3
:10FB40001B65112309F498C06091350D7091360D35
:10FB50008091370D9091380DA70196010E9455B301
:10FB6000243031054105510509F086C00E940B661D
:10FB70002FEF30E040E050E06EE27AE087E39FE074
:10FB800078CFD530D9F520916F022223B9F0A701A3
:10FB900096010E9455B38BE592E025303105410571
:10FBA000510521F46ADC9C014EE303C066DC9C0134
:10FBB00040E262E37FE08C2F0E941B65112309F471
:10FBC0005BC06091350D7091360D8091370D90912D
:10FBD000380DA70196010E9455B325303105410526
:10FBE000510509F049C00E940B6627EE33E04AE058
:10FBF00050E06BE572E08DE29FE03BCFD630E1F55F
:10FC000020916F02222399F0A70196010E9455B31B
:10FC1000263031054105510519F420E24EE302C0BA
:10FC200020E240E26DE17FE08C2F0E94E46411232A
:10FC300019F16091350D7091360D8091370D9091CD
:10FC4000380DA70196010E9455B3263031054105B4
:10FC5000510591F40E940B6688E19FE0DF91CF91FE
:10FC60001F910F91FF90EF90DF90CF90BF90AF90DA
:10FC70009F908F900C94213F8091350D9091360D7F
:10FC8000A091370DB091380D8397A105B10540F0D3
:10FC90008092350D9092360DA092370DB092380DAE
:10FCA0006091350D7091360D8091370D9091380D22
:10FCB000A70196010E9455B380913E0D90E00396F6
:10FCC000422F50E0841795074CF48DEF820F8093FC
:10FCD0003E0D00936F02DCEFD20FCFEFCF5FDF5FFF
:10FCE000C43008F40ECEDF91CF911F910F91FF9099
:10FCF000EF90DF90CF90BF90AF909F908F9008953E
:10FD0000FC01808191818436910524F164E670E0E4
:10FD10000E9442B3CB012AE030E0B9010E9442B315
:10FD2000805D8093090D80819181B9010E9442B369
:10FD3000CB01B9010E9442B3805D80930A0D80819E
:10FD40009181B9010E9442B3805D80930B0D1092A6
:10FD50000C0D23C08A309105BCF02AE030E0B901D7
:10FD60000E9442B3CB01B9010E9442B3805D8093EF
:10FD7000090D80819181B9010E9442B3805D809319
:10FD80000A0D10920B0D09C06AE070E00E9442B3A8
:10FD9000805D8093090D10920A0D89E09DE0089521
:10FDA000CF92EF920F93E7E4CE2EF5E5EF2E06E427
:10FDB00023E142E162E580E49DE00E94AA290F91DF
:10FDC000EF90CF900895CF93DF93FC016491EC0105
:10FDD0002196662331F080E49DE00E94972ACE01AF
:10FDE000F4CFDF91CF9108950F931F93CF93DF93BB
:10FDF0008C01EB0141E061E080E49DE00E94BF28BE
:10FE0000C801E1DF6AE380E49DE00E9496AEFE0156
:10FE100001900020E9F76C2F6E1B6C5E41E080E4DE
:10FE20009DE00E94BF28BE0180E49DE0DF91CF915C
:10FE30001F910F910C9495AECF92DF92EF92FF92AB
:10FE40000F931F938091350D9091360DA091370D32
:10FE5000B091380D0097A105B10509F442C0BC016D
:10FE6000882777FD8095982F0E9419B02091110D59
:10FE70003091120D4091130D5091140D0E944CB20F
:10FE80009B01AC016091500A7091510A8091520A15
:10FE90009091530A0E949EAE6093500A7093510A4B
:10FEA0008093520A9093530A1092350D1092360D9A
:10FEB0001092370D1092380DA0E3CA2EAAE0DA2E68
:10FEC000E12CF12C00E81FE320E53AE04CE45AE095
:10FED00068E47AE084E49AE00E944E9B81E080939B
:10FEE0006F0280916F02882339F080E59AE0A7D9EC
:10FEF000BC018AE390E178DF80913F0D82FF0EC064
:10FF000021E040E050E0BA0188EE99E61F910F91A0
:10FF1000FF90EF90DF90CF900C943F661F910F9170
:10FF2000FF90EF90DF90CF900895CF93DF931F92D3
:10FF30001F92CDB7DEB78091350D9091360DA0910F
:10FF4000370DB091380DB7FF08C01092350D1092E3
:10FF5000360D1092370D1092380D80911D0D909135
:10FF60001E0DA0911F0DB091200D4091350D5091A7
:10FF7000360D6091370D7091380D84179507A607DF
:10FF8000B70744F48093350D9093360DA093370D49
:10FF9000B093380D80916F028823A9F08091210DD4
:10FFA0009091220D2091350D3091360D820F931FC7
:10FFB0009A838983CE01019660DABC018091270D76
:10FFC0009091280D11DF80913F0D82FF1DC0E091BF
:10FFD000250DF091260D8091210D9091220D2091FB
:10FFE000350D3091360D820F931F918380834091A0
:10FFF000290D50912A0D60E070E021E080912B0DD9
:020000021000EC
:1000000090912C0D0E943F660F900F90DF91CF9141
:1000100008954F925F926F927F928F929F92AF92CC
:10002000BF92CF92DF92EF92FF920F931F93CF93E5
:10003000DF934C015B017A018091350D9091360D73
:10004000A091370DB091380D892B8A2B8B2B09F499
:100050007BC00E944D41E501CC0FDD1FCC0FDD1FA1
:100060008E010C5B154F6091350D7091360D882710
:1000700077FD8095982F0E9419B02091110D309135
:10008000120D4091130D5091140D0E944CB2F801C5
:1000900020813181428153810E949EAE2B013C011F
:1000A00020E030E0A9010E9477AFF80187FD05C08C
:1000B000408251826282738204C010821182128255
:1000C0001382B701882777FD8095982F0E9419B079
:1000D0006B017C018E010C5B154F9B01AC01F8019B
:1000E00060817181828193810E947AB118162CF40B
:1000F000F801C082D182E282F3821092350D109213
:10010000360D1092370D1092380DCA55DA4F20E097
:1001100030E040E752E4688179818A819B810E94C6
:100120007EAFD0E3CD2EDAE0DD2E7B018C0120E521
:100130003AE04CE45AE068E47AE084E49AE00E9411
:100140004E9B81E080936F0280916F02882359F06B
:10015000C501880F991F880F991F8C5B954F6FD829
:10016000BC01C40141DE80913F0D82FF18C021E037
:1001700040E050E0BA0188EE99E6DF91CF911F91FF
:100180000F91FF90EF90DF90CF90BF90AF909F9036
:100190008F907F906F905F904F900C943F66DF91AF
:1001A000CF911F910F91FF90EF90DF90CF90BF9074
:1001B000AF909F908F907F906F905F904F90089539
:1001C00046ED50E060E070E084E390E122CF46EC41
:1001D00050E061E070E086E390E11BCF49EC50E035
:1001E00062E070E088E390E114CF8F929F92AF922B
:1001F000BF92CF92DF92EF92FF920F931F93CF9314
:10020000DF93CDB7DEB728970FB6F894DEBF0FBEE9
:10021000CDBF80912F0D882321F0815080932F0D29
:1002200003C081E080936F0280916F02882309F4FC
:1002300056C280919A0D8F5F80939A0D8E3129F46A
:100240000E94AA6B10929A0D0EC06AE00E9421B320
:10025000911109C020E044E064E180E49DE00E9447
:10026000CF290E946E6520E030E040E05FE36091BE
:1002700040087091410880914208909143080E9483
:100280009EAE0E94E6AF78876F83609148087091B8
:100290004908882777FD8095982F0E9419B020E0A3
:1002A00030E040E05FE30E949EAE0E94E6AF7E83B6
:1002B0006D8340E060E080E49DE00E94BF2862E042
:1002C00080E49DE00E9496AECE010796D6D8BC0190
:1002D00080E49DE00E9495AE6FE280E49DE00E9484
:1002E00096AECE0105960CDDBC0180E49DE00E9437
:1002F00095AE85E19FE067DD60E973E080E49DE015
:100300000E9495AE40E06AE080E49DE00E94BF2834
:1003100062EA75E080E49DE00E9495AE2CEA35EC3F
:1003200047E257E360914C0A70914D0A80914E0A62
:1003300090914F0A0E949EAE69837A838B839C833F
:10034000CE0101960E946B79BC0180E49DE00E9481
:1003500095AE60E280E49DE00E9496AE41E060E0F0
:1003600080E49DE00E94BF2820E030E040E05FE3B1
:1003700060913A0870913B0880913C0890913D084B
:100380000E949EAE0E94E6AF78876F836091460818
:1003900070914708882777FD8095982F0E9419B0A3
:1003A00020E030E040E05FE30E949EAE0E94E6AFB6
:1003B0007E836D8360E080E49DE00E9496AECE0176
:1003C00007965BD8BC0180E49DE00E9495AE6FE289
:1003D00080E49DE00E9496AECE01059691DCBC01C2
:1003E00080E49DE00E9495AE82E19FE0ECDC60E954
:1003F00073E080E49DE00E9495AE41E06AE080E415
:100400009DE00E94BF2860E973E080E49DE00E94C7
:1004100095AE66E080E49DE00E9496AE8DE592E0A8
:100420002CD8BC0180E49DE00E9495AE65E280E49A
:100430009DE00E9496AE6DE873E080E49DE00E942E
:1004400095AE42E060E080E49DE00E94BF288FE02E
:100450009FE0B9DC80915F0A8823A9F18091480C64
:10046000882319F18091F20C9091F30CA091F40C77
:10047000B091F50C0097A105B105B9F0BC01CD0113
:100480006D597F4F8F4F9F4F24E630E040E050E0A2
:100490000E9455B36091FA0C7091FB0C8091FC0C9A
:1004A0009091FD0C0E9455B301C020E030E03A83EA
:1004B0002983CE0101960E943D7ABC0180E49DE033
:1004C0000E9495AE03C08BE09FE07DDC65E280E496
:1004D0009DE00E9496AE6CE873E080E49DE00E948F
:1004E00095AE42E06AE080E49DE00E94BF2860E9AA
:1004F00073E080E49DE00E9495AE67E080E49DE0BB
:100500000E9496AE8091520890915308A091540891
:10051000B0915508892B8A2B8B2BE1F10E9408AAF8
:1005200020E6C22E2AEED22EE12CF12CA701960154
:100530000E9455B349015A016091520870915308C5
:100540008091540890915508A70196010E9455B3D7
:10055000C401821B930B6CE370E00E942EB3182F32
:100560006983CE0101960E940779BC0180E49DE079
:100570000E9495AE6AE380E49DE00E9496AE1983E6
:10058000CE0101960E940779BC0180E49DE00E94A3
:1005900095AE03C085E09FE016DC60E973E080E47F
:1005A0009DE00E9495AE43E060E080E49DE00E9403
:1005B000BF286EE773E082E792E00E9405B7892BBF
:1005C00009F074C06EE67AE085E59DE00E9405B70B
:1005D000892BD1F0E5E5FDE0DF010D900020E9F782
:1005E000AD014150510945555D4060E070E0CF01DB
:1005F0000E94D5B66EE67AE085E59DE00E940EB7D2
:1006000010928B0D10928A0DEEE6FAE00190002018
:10061000E9F7EF56FA40759708F445C000918A0D46
:1006200010918B0DC12CD12C80918A0D90918B0D46
:100630009801281B390B2431310534F00196909331
:100640008B0D80938A0D38C0C114D104B9F7F8011D
:10065000E35AF54F7F019189602F681B43E09111A8
:1006600015C080E49DE00E94BF28D70150966C9190
:1006700080E49DE00E9496AE10928B0D10928A0D40
:1006800000E010E0CC24C394D12CCECF80E49DE0D8
:100690000E94BF28F701608980E49DE00E9496AE29
:1006A0000F5F1F4FC1CF65E57DE002C062E772E0DA
:1006B00080E49DE00E9495AE02E712E0D8018D91A2
:1006C0008D0180322CF460E280E49DE00E9496AEC1
:1006D000B2E006381B0791F78AE080932F0D8091D6
:1006E0003F0D82FB882780F990912E0D992399F078
:1006F00090912D0D992339F0811119C010922D0D73
:1007000010922E0D14C0882391F00E940B6681E098
:1007100080932D0D0CC0882351F021E040E050E083
:10072000BA0183E393E70E943F660E94AA6B80911F
:100730005D0290915E022091350D3091360D843628
:10074000910534F4820F931F853691054CF416C041
:100750008436910599F0820F931F8436910574F4C5
:100760001092350D1092360D1092370D1092380DF3
:1007700084E690E090935E0280935D0220915D029A
:1007800030915E028091350D9091360D2436310501
:1007900069F48B3091051CF0865A9F4F09C0863F43
:1007A000EFEF9E078CF482599F4F02C0820F931F78
:1007B00090935E0280935D021092350D1092360D7B
:1007C0001092370D1092380D80915D0290915E026B
:1007D0008A3091051CF48AE090E005C0883E934081
:1007E00034F087EE93E090935E0280935D0228964A
:1007F0000FB6F894DEBF0FBECDBFDF91CF911F9132
:100800000F91FF90EF90DF90CF90BF90AF909F90AF
:100810008F900895CF93DF93C0EBDEE0FE018491CB
:10082000882341F09091C00095FFFCCF8093C600D3
:100830003196F5CFE5E8F4E18491882341F0909179
:10084000C00095FFFCCF8093C6003196F5CF809114
:10085000C00085FFFCCF8AE08093C600FE01849132
:10086000E0EBFEE0882349F09091C00095FFFCCFBB
:100870008093C60031968491F5CF4091A113509199
:10088000A2136091A3137091A4138DE794E10E94C9
:100890008A3E4091A5135091A6136091A7137091C1
:1008A000A8138AE794E10E948A3E4091A9135091CF
:1008B000AA136091AB137091AC1387E794E10E9487
:1008C0008A3E4091AD135091AE136091AF13709179
:1008D000B01384E794E10E948A3E8091C00085FFB6
:1008E000FCCF8AE08093C600FE018491E0EBFEE03D
:1008F000882349F09091C00095FFFCCF8093C600FB
:1009000031968491F5CFEAE5F4E18491882341F0B2
:100910009091C00095FFFCCF8093C6003196F5CF33
:100920008091C00085FFFCCF8AE08093C600FE0165
:100930008491E0EBFEE0882349F09091C00095FFA0
:10094000FCCF8093C60031968491F5CF4091B113CE
:100950005091B2136091B3137091B41381E594E197
:100960000E948A3E4091B5135091B6136091B7131F
:100970007091B8138EE494E10E948A3E4091B913BD
:100980005091BA136091BB137091BC138BE494E146
:100990000E948A3E4091BD135091BE136091BF13D7
:1009A0007091C01388E494E10E948A3E8091C00057
:1009B00085FFFCCF8AE08093C600FE018491E0EBC6
:1009C000FEE0882349F09091C00095FFFCCF809312
:1009D000C60031968491F5CFEAE2F4E18491882350
:1009E00041F09091C00095FFFCCF8093C6003196F6
:1009F000F5CF8091C00085FFFCCF8AE08093C600D0
:100A0000FE018491E0EBFEE0882349F09091C00064
:100A100095FFFCCF8093C60031968491F5CF40912D
:100A2000911350919213609193137091941381E2FA
:100A300094E10E949C3E40919513509196136091D1
:100A40009713709198138EE194E10E949C3E40911F
:100A5000991350919A1360919B1370919C138BE1A1
:100A600094E10E949C3E40919D1350919E13609191
:100A70009F137091A01388E194E10E949C3E8091A5
:100A8000C00085FFFCCF8AE08093C600FE01849100
:100A9000E0EBFEE0882349F09091C00095FFFCCF89
:100AA0008093C60031968491F5CFE3EEF3E1849113
:100AB000882341F09091C00095FFFCCF8093C60041
:100AC0003196F5CF8091C00085FFFCCF8AE08093FE
:100AD000C600FE018491E0EBFEE0882349F090918E
:100AE000C00095FFFCCF8093C60031968491F5CF6E
:100AF0004091891350918A1360918B1370918C13DC
:100B00008AED93E10E948A3E4091851350918613AD
:100B1000609187137091881387ED93E10E948A3E5C
:100B20008091C00085FFFCCF8AE08093C600FE0163
:100B30008491E0EBFEE0882349F09091C00095FF9E
:100B4000FCCF8093C60031968491F5CFE4E2F3E1C7
:100B50008491882341F09091C00095FFFCCF809351
:100B6000C6003196F5CF8091C00085FFFCCF8AE0AA
:100B70008093C600FE018491E0EBFEE0882349F0FB
:100B80009091C00095FFFCCF8093C6003196849170
:100B9000F5CF40918D1350918E1360918F1370910A
:100BA00090138BE193E10E948A3E4091751350911E
:100BB0007613609177137091781388E193E10E9426
:100BC0008A3E4091C1135091C2136091C31370913A
:100BD000C41385E193E10E949C3E409181135091A2
:100BE0008213609183137091841382E193E10E94D8
:100BF0008A3E40917D1350917E1360917F137091D6
:100C000080138FE093E10E948A3E409179135091C6
:100C10007A1360917B1370917C138CE093E10E94B6
:100C20008A3E8091C00085FFFCCF8AE08093C60099
:100C3000FE018491E0EBFEE0882349F09091C00032
:100C400095FFFCCF8093C60031968491F5CFEAEFF3
:100C5000F2E18491882341F09091C00095FFFCCF90
:100C60008093C6003196F5CF8091C00085FFFCCF00
:100C70008AE08093C600FE018491E0EBFEE08823C9
:100C800049F09091C00095FFFCCF8093C60031964B
:100C90008491F5CF4091380A5091390A60913A0A0F
:100CA00070913B0A81EF92E10E948A3E40913C0A9A
:100CB00050913D0A60913E0A70913F0A8EEE92E19A
:100CC0000E948A3E4091400A5091410A6091420A36
:100CD0007091430A8BEE92E10E948A3E8091C0009F
:100CE00085FFFCCF8AE08093C600FE018491E0EB93
:100CF000FEE0882349F09091C00095FFFCCF8093DF
:100D0000C60031968491F5CFEDEDF2E18491882310
:100D100041F09091C00095FFFCCF8093C6003196C2
:100D2000F5CF8091C00085FFFCCF8AE08093C6009C
:100D3000FE018491E0EBFEE0882349F09091C00031
:100D400095FFFCCF8093C60031968491F5CF4091FA
:100D500018025091190260911A0270911B0283EDE2
:100D600092E10E948A3E6091140270911502809176
:100D70001602909117020E94FE27AB01BC0180ED84
:100D800092E10E948A3E609110027091110280915E
:100D90001202909113020E940A28AB01BC018DEC53
:100DA00092E10E948A3E8091C00085FFFCCF8AE0DC
:100DB0008093C600FE018491E0EBFEE0882349F0B9
:100DC0009091C00095FFFCCF8093C600319684912E
:100DD000F5CFE9E9F2E18491882341F09091C000D8
:100DE00095FFFCCF8093C6003196F5CF8091C0006F
:100DF00085FFFCCF8AE08093C600FE018491E0EB82
:100E0000FEE0882349F09091C00095FFFCCF8093CD
:100E1000C60031968491F5CF40913302509134024F
:100E200060913502709136028FE892E10E948A3E0D
:100E300020E030E040E752E460912B0270912C02F8
:100E400080912D0290912E020E944CB2AB01BC0108
:100E50008CE892E10E948A3E4091280A5091290A2A
:100E600060912A0A70912B0A89E892E10E948A3ED9
:100E70008091C00085FFFCCF8AE08093C600FE0110
:100E80008491E0EBFEE0882349F09091C00095FF4B
:100E9000FCCF8093C60031968491F5CFEDE5F2E169
:100EA0008491882341F09091C00095FFFCCF8093FE
:100EB000C6003196F5CF8091C00085FFFCCF8AE057
:100EC0008093C600FE018491E0EBFEE0882349F0A8
:100ED0009091C00095FFFCCF8093C600319684911D
:100EE000F5CF4091240A5091250A6091260A70910D
:100EF000270A83E592E10E948A3E20E030E040E745
:100F000052E4609127027091280280912902909109
:100F10002A020E944CB2AB01BC0180E592E10E9422
:100F20008A3E8091C00085FFFCCF8AE08093C60096
:100F3000FE018491E0EBFEE0882349F09091C0002F
:100F400095FFFCCF8093C60031968491F5CFE6EFF4
:100F5000F1E18491882341F09091C00095FFFCCF8E
:100F60008093C6003196F5CF8091C00085FFFCCFFD
:100F70008AE08093C600FE018491E0EBFEE08823C6
:100F800049F09091C00095FFFCCF8093C600319648
:100F90008491F5CF40912D0A50E060E070E08CEE36
:100FA00091E10E949C3E8091C00085FFFCCF8AE0C9
:100FB0008093C600FE018491E0EBFEE0882349F0B7
:100FC0009091C00095FFFCCF8093C600319684912C
:100FD000F5CF8091540A8823A1F1E9EDF1E18491E4
:100FE000882341F09091C00095FFFCCF8093C6000C
:100FF0003196F5CF8091C00085FFFCCF8AE08093C9
:10100000C600FE01C491E0EBFEE0CC2349F08091E4
:10101000C00085FFFCCFC093C6003196C491F5CFC8
:1010200040915302509154026091550270915602C2
:101030008FEC91E10E948A3E8091C00085FFFCCF39
:1010400011C0E3EBF1E18491882341F09091C0005D
:1010500095FFFCCF8093C6003196F5CF8091C000FC
:1010600085FFFCCF8AE08093C600DF91CF91089581
:10107000AF92BF92CF92DF92EF92FF920F931F93A6
:10108000CF93DF93CDB7DEB7E0970FB6F894DEBF0E
:101090000FBECDBF80E1EFEEF2E0DE019196019050
:1010A0000D928A95E1F780E1EFEFF2E0DE015196D3
:1010B00001900D928A95E1F780E1EFE0F3E0DE0127
:1010C000119601900D928A95E1F76E0181E2C80EAA
:1010D000D11C81EAE82E83E1F82E8E010F5E1F4FAE
:1010E00061EB73E1AE014F5F5F4F91E9A92E93E190
:1010F000B92E20E030E0F60181919191A191B1915A
:101100006F01F70181939193A193B1937F01F8014E
:1011100081919191A191B1918F01FB018193919363
:10112000A193B193BF01FA0181919191A191B191E4
:10113000AF01F50181939193A193B1935F012F5F6B
:101140003F4F24303105B9F60E94E7A580E090E8D2
:10115000ABE3B5E48093891390938A13A0938B1328
:10116000B0938C138093851390938613A093871369
:10117000B093881310928D1310928E1310928F13C8
:101180001092901380E29EE4A0E0B0E08093C1133F
:101190009093C213A093C313B093C413109275130A
:1011A00010927613109277131092781380E090E0EB
:1011B000A0EAB1E48093811390938213A0938313E8
:1011C000B09384138DEC9CECACECBEE380937D1368
:1011D00090937E13A0937F13B093801380E090E0F0
:1011E000A0EAB0E48093791390937A13A0937B13D1
:1011F000B0937C131092400A1092410A1092420A56
:101200001092430A10923C0A10923D0A10923E0A34
:1012100010923F0A1092380A1092390A10923A0A34
:1012200010923B0A82ED90E09093980D8093970D79
:1012300082E390E09093960D8093950D1092940D1B
:101240001092930D8FEF90E09093920D8093910DFB
:1012500084E690E09093900D80938F0D10928E0D08
:1012600010928D0D83E393EBA3E2B2E48093180216
:1012700090931902A0931A02B0931B0260E070E0F1
:101280008CE990E40E94F827609314027093150291
:10129000809316029093170265E87BE28CEA92E451
:1012A0000E9404286093100270931102809312022E
:1012B000909313020E94661E80E090E0A0E8BFE3D6
:1012C00080930C0290930D02A0930E02B0930F0234
:1012D00010922D0A80E090E0A0E4B0E48093330205
:1012E00090933402A0933502B093360240E050E070
:1012F00064E372E440932B0250932C0260932D021E
:1013000070932E021092280A1092290A10922A0A2B
:1013100010922B0A1092240A1092250A1092260A83
:101320001092270A40E050E060E071E44093270209
:10133000509328026093290270932A021092540A53
:101340008093530290935402A0935502B093560297
:101350000E94954BE0EBFEE08491882341F0909150
:10136000C00095FFFCCF8093C6003196F5CFE1E930
:10137000F1E18491882341F09091C00095FFFCCF6A
:101380008093C6003196F5CF8091C00085FFFCCFD9
:101390008AE08093C600E0960FB6F894DEBF0FBED9
:1013A000CDBFDF91CF911F910F91FF90EF90DF9014
:1013B000CF90BF90AF9008951F920F920FB60F92EB
:1013C00011240BB60F922F933F934F935F936F931C
:1013D0008F939F93EF93FF936091C60020911D0E12
:1013E00030911E0EC90101968F77992740911F0EEB
:1013F0005091200E8417950741F0F901E356F24F02
:10140000608390931E0E80931D0EFF91EF919F912C
:101410008F916F915F914F913F912F910F900BBEE4
:101420000F900FBE0F901F9018959A01AB012115D8
:1014300081EE38074105510549F182E08093C000F3
:1014400060E079E08DE390E00E9477B321503109AC
:1014500041095109CA01B90122E030E040E050E001
:101460000E9477B33093C5002093C4008091C100DF
:1014700080618093C1008091C10088608093C10029
:101480008091C10080688093C10008951092C000CF
:1014900020E130E0E7CF20911F0E3091200E8091A7
:1014A0001D0E90911E0E8217930771F0F901E356FD
:1014B000F24F80812F5F3F4F2F7733273093200EDD
:1014C00020931F0E90E008958FEF9FEF0895809175
:1014D0001F0E9091200E90931E0E80931D0E089566
:1014E0004F925F926F927F928F929F92AF92BF9234
:1014F000CF92DF92EF92FF920F931F93CF93DF93E0
:10150000CDB7DEB7A0970FB6F894DEBF0FBECDBF44
:101510005C014115510561057105E9F420E030E0F9
:1015200040E350E060E070E0A0960FB6F894DEBFB4
:101530000FBECDBFDF91CF911F910F91FF90EF9024
:10154000DF90CF90BF90AF909F908F907F906F90E3
:101550005F904F905BC08E010F5F1F4FC12CD12C4D
:1015600076014801422E512C612C712C8FEFC81A44
:10157000D80AE80AF80ACB01BA01A30192010E9435
:1015800055B3CA01F80161938F01A901BC0141154E
:1015900051056105710551F7F1E0CF1AD108E10855
:1015A000F108F401EC0DFD1D80818A3010F440E358
:1015B00001C047E3480F552747FD5095652F752F0C
:1015C00020E030E0C50122D081E0C81AD108E1084E
:1015D000F108EFEFCE16DE06EE06FE0611F7A09636
:1015E0000FB6F894DEBF0FBECDBFDF91CF911F9134
:1015F0000F91FF90EF90DF90CF90BF90AF909F90B2
:101600008F907F906F905F904F90089521153105D6
:1016100039F48091C00085FFFCCF4093C600089547
:101620002A30310509F424C05BCF9A01462F552793
:1016300047FD5095652F752FE9CFCF93DF93EC01D0
:1016400020E030E04DE050E060E070E0DFDF20E0DF
:1016500030E04AE050E060E070E0CE01DF91CF91F1
:10166000D5CF9A01AB01662757FD6095762FCECF77
:10167000CF92DF92EF92FF92CF93DF93EC016A015A
:101680007B0177FF0FC020E030E04DE250E060E0EA
:1016900070E0BCDFF094E094D094C094C11CD11CE5
:1016A000E11CF11C2AE0B701A601CE01DF91CF9128
:1016B000FF90EF90DF90CF9013CF2115310539F4D3
:1016C0008091C00085FFFCCF4093C600089508CFED
:1016D0009A01462F50E060E070E0EFCFCF93DF93A8
:1016E000EC019A01AB0160E070E0E7DFCE01DF9131
:1016F000CF91A3CF8F929F92AF92BF92CF92DF9262
:10170000EF92FF921F93CF93DF93EC016A017B016D
:10171000122F20E030E0A901C701B6010E9477AF87
:1017200087FF0CC020E030E04DE250E060E070E068
:10173000CE016CDFF7FAF094F7F8F094B12C60E08A
:1017400070E080E09FE3B11641F020E030E040E23D
:1017500051E40E947EAFB394F6CF9B01AC01C70168
:10176000B6010E949EAE6B017C010E94EBAF4B0163
:101770005C010E9417B09B01AC01C701B6010E9439
:101780009DAE6B017C012AE0B501A401CE01A8DE6B
:10179000112361F0EFE5F3E08191882339F0909116
:1017A000C00095FFFCCF8093C600F6CF112319F13E
:1017B00020E030E040E251E4C701B6010E944CB2A3
:1017C0006B017C010E94E6AF4B01AA2497FCA09418
:1017D000BA2CB501A401CE014BDFC501B4010E94B2
:1017E00019B09B01AC01C701B6010E949DAE6B010F
:1017F0007C011150DBCFDF91CF911F91FF90EF90D3
:10180000DF90CF90BF90AF909F908F90089572CF50
:10181000CF93DF931F92CDB7DEB7698341E050E0ED
:10182000BE016F5F7F4F04960E94C2160F90DF913A
:10183000CF910895FB0101900020E9F7AF014150DD
:101840005109461B570B04960C94C2168091390E11
:10185000811109C08091380E811105C08091370E29
:10186000811101C00895E0EBFEE08491882341F0EE
:101870009091C00095FFFCCF8093C6003196F5CFC4
:10188000E0EFF4E18491882341F09091C00095FF4E
:10189000FCCF8093C6003196F5CF8091390E882316
:1018A000F1F060913A0E70913B0E80913C0E909158
:1018B0003D0E0E9419B02091A1133091A2134091C6
:1018C000A3135091A4130E947EAFAB01BC018CEE18
:1018D00094E10E948A3E8CED94E10E94C77680914B
:1018E000380E8823F1F060913E0E70913F0E80918A
:1018F000400E9091410E0E9419B02091A513309195
:10190000A6134091A7135091A8130E947EAFAB017C
:10191000BC0188ED94E10E948A3E88EC94E10E942B
:10192000C7768091370E8823F1F06091420E709156
:10193000430E8091440E9091450E0E9419B0209163
:10194000A9133091AA134091AB135091AC130E948C
:101950007EAFAB01BC0184EC94E10E948A3E84EB33
:1019600094E10E94C7768091C00085FFFCCF8AE099
:101970008093C6001092390E1092380E1092370ED6
:1019800008951092390E1092380E1092370E089565
:1019900080939B020895EFE6F0E08081826080836F
:1019A00008951F920F920FB60F9211240BB60F924B
:1019B0000F931F932F933F934F935F936F937F9357
:1019C0008F939F93AF93BF93EF93FF9380916A0E92
:1019D00090916B0E892B09F084C190916D0E8091CE
:1019E0006C0E981771F0E0916C0E8DE4E89FF00199
:1019F0001124E259F14FDF01A45BBF4F81E08C93CA
:101A000002C0E0E0F0E0F0936B0EE0936A0E3097D6
:101A100009F461C1DF01A45BBF4F81E08C93109298
:101A20004D0E10924E0E10924F0E1092500E60AD51
:101A300071AD61349CE9790728F461329EE479073D
:101A400048F002C060E47CE97695679576956795E5
:101A500084E007C0613197E2790730F076956795A9
:101A600082E080934A0E07C080934A0E603271056F
:101A700010F460E270E060527109611588E0780747
:101A8000D0F0872F9927880F991F880F991F8150B1
:101A9000974EFC01329645915491AA27659F90017B
:101AA000649F210D3A1F06942A1F3A1F1124FC013E
:101AB000859194911DC0CB01969587958C7F81501F
:101AC0009B4EFC01459154910296FC0185919491A5
:101AD000FB01E770FF278E9F90018F9F300D9E9F27
:101AE000300D1124E3E036952795EA95E1F7CA0118
:101AF000821B930B8436910598F4EEEBF5E081910F
:101B0000882339F09091C00095FFFCCF8093C600E8
:101B1000F6CF4AE050E08CE99DE0E0DD84E690E01D
:101B20009093490E8093480E80914A0E992787FD25
:101B300090959093470E8093460EE0916A0EF09137
:101B40006B0E64AD75AD70934C0E60934B0E6134AB
:101B50009CE9790728F461328EE4780748F002C0E6
:101B600060E47CE9769567957695679584E007C093
:101B7000613197E2790730F07695679582E080933E
:101B80004A0E08C081E080934A0E6032710510F45D
:101B900060E270E060527109611588E07807E0F05A
:101BA000872F9927880F991F880F991F8150974E6B
:101BB000FC01329625913491AA27639FA001629F70
:101BC000410D5A1F06944A1F5A1F1124FC012591EA
:101BD0003491241B350B1EC0CB01969587958C7FC5
:101BE00081509B4EFC01259134910296FC01459158
:101BF0005491FB01E770FF274E9FC0014F9F900D4E
:101C00005E9F900D1124F3E096958795FA95E1F784
